:020000040000FA
:100000000000000082EF12F0086A800E3B6E00D004
:10001000196A1A6A1B6A1C6A0A9ADAD9D8A01200ED
:10002000D30FD8B40A8A2D0FC60FF7E20A0FF5E3F3
:10003000156E146A136A126A0A0E116E9EEC03F0B2
:1000400015501124196E12501A6E000ED8B0010E00
:100050001A2613501B6E000ED8B0010E1B2614502A
:100060001C6E000ED8B0010E1C26080607E0B0D9A1
:10007000D8A01200C60F02E20A0FDAE20AAA0BD0D9
:10008000191E1A1E1B1E1C1E192AD8B41A2AD8B4EF
:100090001B2AD8B41C2A1950D8801200086A196E7D
:1000A0001A6A00960850D8B40086040E076E1A38F3
:1000B00005D81A5003D8193801D819500F0BF60F6C
:1000C000D8B0070F0A0F23D031D803D0086A196EB1
:1000D0001A6A00960850D8B40086050E076E270EDF
:1000E000166E100E0CD8030E166EE80E08D8166A9F
:1000F000640E05D8166A0A0E02D8195008D0156E7B
:100100001A50126E1950116E4CEC03F01150116E12
:10011000074E0096085002E0075C07E21150D8A491
:10012000009600B602D0300F45D112001AAE120070
:1001300019501A10D8B41200191E1A1E194A1A2A78
:100140002D0E38D13D6E26AE02D02D0E33D9283E6D
:1001500004D0273E02D0264A262A336A346A356AFA
:10016000366A268E6A0E2526D89026322732283205
:100170003632353234323332253EF6D72850255CBC
:100180002826255E2750265C2726265E086A38D852
:100190002E0E10D93E6AD8903334286E3434276E30
:1001A0003534266E3634256E3E36D89028362736BE
:1001B000263625363E36335028263450D8B0343CC7
:1001C00027263550D8B0353C26263650D8B0363C98
:1001D0002526D8B03E3ED8902836273626362536F6
:1001E0003E363E50300FE6D828C033F027C034F0FA
:1001F00026C035F025C036F03D2ECCD7D890120061
:100200000096085003E100860A0E086E28C014F01C
:1002100027C013F026C012F025C011F0076A1C6A2F
:100220001B6A1A6A0A0E196E1EEC03F0072A0750A1
:10023000085CF5E11950D8A4009600A602D0082C5D
:1002400003D01950300FB6D8082EE0D7120005C0E1
:1002500011F006C012F0010E156E166AEA6802C0AF
:10026000E9FF000028D814E3152EFBD7FF0E162651
:10027000F8E21126D8A01226D8A01200200E156E82
:10028000030E166EEED7EA6802C0E9FF14D8FEE24C
:1002900054D81F6A080E166E51D80DD8D8B01F3E1C
:1002A0001532162EF9D722AA1F6A22BA159E46D8F1
:1002B000D88015501200120EE9260950EF1202C024
:1002C000E9FFEF1422BC0918FF0F12001D6EEA6847
:1002D000E2680250E96E120FE16E800E0A16080EF7
:1002E0001E6ED890D8B00A3E11D81D321E2EFAD7F5
:1002F000000022BA0A300AD800D000D000D0D8803E
:1003000005D80650166E055053D9120022AE0BD0F8
:10031000EF50091022AC0918EF6EE7500910D8A071
:100320000918E76E0BD0EF500910D8A0091822BCAD
:100330000918EF6E091CE71601D00A8C22501F0B1A
:10034000000F126E2150110FD8B0122A0AAC3DD105
:100350000A9C116E020E0AEC04F037D171B271984A
:10036000718802C011F009C012F0156A166A000007
:1003700000D00000A4BA0FD0E8681526162211227A
:100380001222D8A012001548163CF1D7D00E156ED7
:10039000030E166EEED77450D8801200A66AA68E91
:1003A0000900F55002E002D8FBD71200A4A8FED73E
:1003B000736E120001BA8AD701A202D001B036D002
:1003C00001A205D001B003D001B2EE6E1200EED74B
:1003D0003BAE03D0EE50D88012003B50080ABEE07E
:1003E0003B50030AD8B433D73B50050AD8B44BD797
:1003F000008800A8009800BA03D0008A35D829E206
:100400000094080E166E40D81536162EFCD700B490
:1004100007D000B801D04AD845D841D800B819D87B
:1004200043D8D89015501CD0008800A8009800BC74
:1004300005D0FE0B0A6E008CD89012D000BE05D0FD
:100440001D6E008E11D805E21D5012D802E200A8E0
:1004500007D02CD827D8009C009E009A009424D85E
:100460001F80D8A01F90120017D80A5000BA0109A7
:10047000156E080E166E153617D801E217D812D869
:100480000ED8162EF8D710D80DD800D00000D8906E
:1004900081BCD88004D8120007D804D807D8819E20
:1004A000939E06D0938E04D0938C02D08A9C939C0A
:1004B0001200A86EA66AA684550EA76EAA0EA76E95
:1004C000A682A6B2FED7A694A94AAA2AA68E120090
:1004D000A96EA66AA680A850A94AAA2AA68E1200CA
:1004E000E836E836FC0B0109C2128009C216C0507A
:1004F000F80B0309C06E640E67D8C282C2B2FED781
:10050000C4CF26F0C350256E1200080E1D6E1E6E5D
:10051000EA6803C0E9FF04500AB480D90AA480D96C
:10052000E26803C0E1FF0250120FE96E0950EF12BA
:1005300002C0E9FF116A126A1D500FE00AB231D8F9
:10054000EF500914FF0F113612360AA22AD81D2EB9
:10055000F5D71E500AB043D111501200080E1D6E7F
:10056000EA6803C0E9FF04500AB458D90AA458D96C
:10057000E26803C0E1FF0250120FE96E091CEF169A
:100580001D500EE00AB02BD902C0E9FF1232113221
:10059000EF500910D8A00918EF6E03D81D2EF6D71A
:1005A00012000450E71A000000D0E71A1200166A81
:1005B000156EFF0E1526162200D0D8A01200030ECD
:1005C000126EE60E02D8F5D7126AFE0F116E000009
:1005D00000D000D0E86A125AD8A01200110600D04C
:1005E00000D0F5D70009D8B412001F6E11C0E9FF82
:1005F00012C0EAFF126A116A1FBE07D0EE50116ED8
:100600001FA21200EF50126E120004D8EF14D8A4EB
:10061000112A1200010E1FB0E8441FB2E8441FB2B5
:10062000E8441FB4E8381200010F1E6E0A0E156E62
:10063000166A32D81E2EFDD7195012002F6A306A62
:10064000316A326A210E176E15D02F3630363136A8
:10065000323619502F5C1A5030581B5031581C50EC
:10066000325808E3326E19502F5E1A50305A1B5020
:10067000315AD8801136123613361436172EE5D774
:1006800032C01CF031C01BF030C01AF02F50196E70
:100690001200126A166A156E1A6A196A100EF36E43
:1006A000123419361A361550195C16501A5805E3CB
:1006B0001550195E16501A5AD88011361236F32E7C
:1006C000EFD71150120020501A18800BF46E20AE94
:1006D00005D01F1E201E1F2AD8B4202A1AAE05D00E
:1006E000191E1A1E192AD8B41A2A156A116A126A12
:1006F000166A1A5002E1195018E0100EF36ED890E5
:100700001F362036153616361A50165C02E119507F
:10071000155C07E31950155ED8A016061A50165E30
:10072000D88011361236F32EEAD7F4AE05D0111E5A
:10073000121E112AD8B4122A1150120014C032F01D
:1007400013C031F012C030F011C02FF03150190237
:10075000F3CF13F0F4CF14F030501A02F3501326F5
:10076000F45014222F501B02F3501326F45014227D
:1007700032501902F350142631501A02F350142645
:1007800030501B02F35014262F501C02F350142635
:100790002F501902F3CF11F0F4CF12F0305019029C
:1007A000F3501226F4501322000E14222F501A0276
:1007B000F3501226F4501322000E1422120015508A
:1007C0001D02F3CF19F0F4CF1AF016501D02F350AA
:1007D0001A2615501E02F3501A2619501200156AD7
:1007E000166A04D01232113215361636FF0FFAE2AD
:1007F00016C012F01550116E1200116E12BE02D802
:1008000011501200111E121E114A122A1200D89005
:1008100012321132FF0FFBE211501200EF1203D01F
:10082000FF0AEF1601D0FF0AE988E92AEC16120048
:10083000A66AA68E0900F55002E0EE6EFBD7120004
:10084000F34E02D0E652FCD7E6CFEEFFE82EFCD7FF
:100850001200A66AA68EEE500900F55C02E1F5666C
:10086000FAD712003FC01FF03F8C0ED8D90E3A6E57
:100870005B0E396E5E0E386E7D0E376EC7EC06F07D
:100880001FAC3F9C3650120034BE06D13352D8B450
:1008900003D13FC01DF03F8C7E0E335C1E6E7E0E7A
:1008A000336E3A6A396A386A7F0E376EF30E365CF9
:1008B000040ED8A0050E355C350ED8A0360E345C7B
:1008C00002E36FD903D0332A6CD91E0636C011F06B
:1008D00035C012F034C013F033C014F0710E3A6E0C
:1008E0005F0E396E550E386E800E376E5CD911C0B2
:1008F0003AF012C039F013C038F014C037F0C7EC2A
:1009000006F0C60E3A6EF50E396E1F0E386E800E6A
:10091000376E49D936C015F035C016F034C017F01F
:1009200033C018F011C036F012C035F013C034F0E7
:1009300014C033F08A0E3A6E120E396E790E386E8C
:100940007D0E376EC7EC06F0F60E3A6E460E396E27
:10095000550E386E7E0E376E26D915C03AF016C089
:1009600039F017C038F018C037F0ABD936C015F0E1
:1009700035C016F034C017F033C018F01450336E81
:10098000376E1350346E386E1250356E396E11500A
:10099000366E3A6EFCD936C025F035C026F034C02C
:1009A00027F033C028F015C03AF016C039F017C050
:1009B00038F018C037F0EBD911C03AF012C039F056
:1009C00013C038F014C037F0E2D925C03AF026C081
:1009D00039F027C038F028C037F037663706E1D83D
:1009E00011C03AF012C039F013C038F014C037F01B
:1009F000DAD81E5252E036C025F035C026F034C099
:100A000027F033C028F01EC033F0000E33BEFF0EB7
:100A1000346E356E366E7CEC07F036C011F035C0A2
:100A200012F034C013F033C014F0830E3A6E800E0F
:100A3000396EDE0E386E720E376EA9D925C03AF0C7
:100A400026C039F027C038F028C037F0ACD836C0FF
:100A500025F035C026F034C027F033C028F011C08F
:100A600036F012C035F013C034F014C033F03A6AD7
:100A7000800E396E310E386E7E0E376E88D925C0E5
:100A80003AF026C039F027C038F028C037F08BD8AC
:100A90001DBC03D03F9C01D03F8A36501200385015
:100AA0003418426E42BE34D038BE19D03750335C51
:100AB000D8A0000CD8A4010C3850345CD8A0000C8D
:100AC000D8A4010C3950355CD8A0000CD8A4010C76
:100AD0003A50365CD8A0000CD8A4010C000C33505E
:100AE000375CD8A0000CD8A4010C3450385CD8A0D6
:100AF000000CD8A4010C3550395CD8A0000CD8A447
:100B0000010C36503A5CD8A0000CD8A4010C000CA3
:100B100034AE010C000C34503818426E42BE34D052
:100B200034BE19D03350375CD8A0000CD8A4010CC7
:100B30003450385CD8A0000CD8A4010C3550395C76
:100B4000D8A0000CD8A4010C36503A5CD8A0000CF8
:100B5000D8A4010C000C3750335CD8A0000CD8A4EA
:100B6000010C3850345CD8A0000CD8A4010C3950CA
:100B7000355CD8A0000CD8A4010C3A50365CD8A043
:100B8000000CD8A4010C000C38AE010C000C3A6A21
:100B9000396A7E0E376E800E34AE000E386E03D882
:100BA00044D1800E381A3750335C3E6E11E23E6CF1
:100BB000335037C033F0376E345038C034F0386EAD
:100BC000355039C035F0396E36503AC036F03A6E8D
:100BD0001A0E3E6074D0375272E03D6A3450416E56
:100BE0003818406E348E388E080E3E5E08E33AC0E8
:100BF0003DF039C03AF038C039F0386AF5D73E26B2
:100C000007E0D890383239323A323D323E2EF9D7A9
:100C100040AE33D03A50365E3950355A3850345A97
:100C200007E2D880000E365635563456800E411AEB
:100C30003D6C04E03606000E355A345A040E3E6E02
:100C400034660DD035C034F036C035F03DC036F0D6
:100C50003D6A080E335E29E33E2EF2D726D034BE1D
:100C600008D0D8903D36363635363436332EF7D761
:100C70001CD03DAE22D03D6A0FD03A5036263950B6
:100C800035223850342206E33432353236323D32A2
:100C9000334A0DD03DAE11D0363E0FD0353E0DD08B
:100CA000343E0BD0D8803690EFD7336A02D03F82E3
:100CB0003368366A356A800E346E41AE349E3650E3
:100CC00012003450316E3818406E375051E03352B4
:100CD00052E0335E7F0E03E2332603E24BD033262D
:100CE0004CE236C02FF035C030F0318E388E180E01
:100CF000416E366A356A346A0BD03A502F5C3950EF
:100D0000305811E3306E316A3A502F5E0BD004E256
:100D10003850315CF2E007E33A502F5E3950305AD8
:100D20003850315AD8803636353634362F3630364C
:100D30003136412EECD734BE07D033521BE040325F
:100D40003306412A4036E3D707E23A502F5E395046
:100D5000305A3850315A17E3363E15D0353E13D04D
:100D6000343E11D0343235323632333E0CD005D0D9
:100D70003F8604D03F84336A02D03F823368366AAC
:100D8000356A800E346E40AE349E365012003450B8
:100D9000316E3818406E3350D8A437503AE03326BD
:100DA0007E0E03E3335E03E336D0335E31E336C0B9
:100DB0002FF035C030F0318E388E366A356A346A9D
:100DC000180E416E313230322F3206E33A50362659
:100DD0003950352238503422343235323632412EB1
:100DE000F1D734BE07D0363635363436335210E0BC
:100DF0003306313416E3363E14D0353E12D0343E3D
:100E000010D0D880343235323632333E0AD003D057
:100E10003F84336A02D03F823368366A356A800E77
:100E2000346E40AE349E3650120033C041F0345020
:100E300036C034F0366E3636413236323F6A363698
:100E4000413602E33F843F7E06E13F80416A366AD5
:100E5000356A346A0BD0412803E0D880363206D098
:100E6000D890363202E13F8201D03F863FB604D0AF
:100E70003FA20FD03FB407D07F0E366EFF0E356E07
:100E8000346E336E23D0800E366E01D0366A000E7B
:100E9000F6D73FB0FBD7336A9F0E4160EBD77E0E8B
:100EA0004164F4D79E0E415C07E0D890363235326B
:100EB00034323332412AF6D73FA408D0D880000E0E
:100EC000335634563556365636AEE0D733501200C8
:100ED000336E000E33BEFF0E346E356E366E0CD0A0
:100EE000000E34BEFF0E356E366E06D0336E346A99
:100EF000356A366A409E0AD0409E36AE07D0D8800A
:100F0000000E3356345635563656408E960E416E88
:100F1000365209E0080E412634C033F035C034F0B3
:100F200036C035F011D035520FE1080E415E345015
:100F300007E1080E415E335002E1365010D0336AAB
:100F4000356E33C034F0336A35BE06D0D8903336B0
:100F5000343635364106F8D740AE359E415033C061
:100F600036F0336E355034C035F0346E12002450F4
:100F70004D544B3136312C302A3238003A2042431E
:100F8000545241434B20000024505542582C3430D9
:100F90002C474C4C2C302C302C302C302A35430034
:100FA00024505542582C34302C5A44412C302C308B
:100FB0002C302C302A34340024505542582C3430F4
:100FC0002C4753562C302C302C302C302A353900FD
:100FD00024505542582C34302C4753412C302C305F
:100FE0002C302C302A34450024505542582C3430B3
:100FF0002C524D432C302C302C302C302A343700DE
:1010000024505542582C34302C4747412C312C3138
:101010002C302C302A35410024505542582C343085
:101020002C5654472C312C312C302C302A3545008D
:1010300024504D544B3331342C302C302C312C3146
:101040002C302C302C302C302C302C302C302C30C0
:101050002C302C302C302C302C302C302C302A32B0
:10106000380024504D544B3130312A333200474E32
:101070004747412C3132303030302E3030302C3335
:101080003531352E393237392C4E2C30313934390F
:101090002E3231362C452C312C31302C312E322C45
:1010A0003230302E302C4D2C2D33342E322C4D2C12
:1010B0002C303030302A000047505654472C333003
:1010C000392E36322C542C202C4D2C302E31332CF2
:1010D0004E2C302E322C4B2C412A32330000212151
:1010E00021214E4F20454E4F5547482053415445EE
:1010F0004C49544553002121212147505320434F4F
:101100004D4D554E49434154494F4E204552524F43
:101110005220202000005445535420444520000014
:1011200042414C4C4F4F4E205041594C4F4144206E
:1011300056200000204259204F4D3342430054793D
:1011400070652048454C5020666F7220496E666F6E
:1011500000004543484F00004D5943004D5943415D
:101160004C4C000054520000545241434500545826
:101170004400545844454C415900554E5000554E7A
:1011800050524F544F00444953500000444953506B
:101190004C41590048454C5000005345524750536C
:1011A00000005454455854005441494C00005359D0
:1011B0004D424F4C0000484F4C440000484F4C44B7
:1011C0004F4646005458540054585441494C00006E
:1011D0005645520056455253494F4E0043574944D5
:1011E0000000435742415400435754454D500000BE
:1011F00050524553530050524553535552450000E9
:10120000465251004652455155454E4359005246AB
:101210005251000044455600444556494154494FF7
:101220004E0042415544000053504545440044425D
:10123000495453005342495453004241545600000C
:1012400054454D500000494E54454D5000004558FE
:1012500054454D500000504F55540000504F5745D5
:101260005200494453500000435753500000534F1D
:101270004C415200534F4C415243454C4C00555346
:101280004F4C000049534F4C00005355505600003E
:1012900043574C0043574C4F43004C4F4341544F2E
:1012A00052004C4F433130005245460044415441B6
:1012B0000000534C454550005445535400004341F1
:1012C0004C49425241544500534554500000475048
:1012D000530055424C4F5800415052530000525455
:1012E000545900004F4646534554000054454C00A5
:1012F00054454C454D4554525900524441544100C7
:1013000052415700455849540000436F6D6D616E5E
:1013100064206973206E6F742076616C69640000CC
:1013200031202D206F6E626F6172642074656D7064
:101330002E2032202D2065787465726E616C2074C9
:10134000656D702E2033202D2052432074656D7002
:10135000657261747572650034202D206261746558
:10136000727920766F6C746167652035202D20734B
:10137000797374656D20766F6C74616765203620B3
:101380002D20736F6C617220766F6C7461676520BD
:1013900037202D20636861726765206375727265FE
:1013A0006E74000038202D206169722070726573A0
:1013B000737572652039202D206865617264207311
:1013C000617474656C6974657300436831202D2005
:1013D0000000436832202D200000436833202D2078
:1013E0000000436834202D200000436835202D2064
:1013F000000043414C494252415445204F4E0000A9
:10140000534554204652455155454E4359204F4E61
:1014100020504F5254412E3220544F203132303020
:1014200020487A007479706520552870292C204452
:10143000286F776E292C20532861766529207265E4
:1014400073702E2045286E6429004D5943616C6CE1
:101450002000504F574552204F55543A20005443D6
:10146000584F204652455155454E43593A200000A9
:101470005254545920262043572046524551554531
:101480004E43593A2000415052532046524551553F
:10149000454E43593A200000525454593A20000016
:1014A000444556494154494F4E3A20005350454512
:1014B000443A20004441544120424954533A2000C8
:1014C00053544F5020424954533A200042415456FD
:1014D0006F6C746167653A200000535550706C79E9
:1014E000566F6C746167653A200054454D506572C3
:1014F00061747572653A2000494E7465726E616C54
:1015000054454D50657261747572653A20004558B6
:101510007465726E616C54454D506572617475727C
:10152000653A2000435749443A200000435753503E
:101530003A20000043574C4F433A20004357424162
:10154000543A2000435754454D503A2000004C4F28
:101550004341544F523A20004C4F4331303A20001F
:10156000415052533A200000554E50726F746F2014
:101570000000545844656C61793A20005458546115
:10158000696C3A20000053594D424F4C3A200000FC
:1015900054526163653A20005441494C3A2000009E
:1015A000457665727920000054544558543A20001D
:1015B000484F4C444F46463A2000434F4E54494E04
:1015C000554F5553205452414E534D495353494F53
:1015D0004E004543484F3A200000534F4C41523A89
:1015E0002000536F6C6172566F6C746167653A20AE
:1015F0000000536F6C617243757272656E743A20AD
:1016000000005155454354454C00505245535355E5
:1016100052453A200000534C4545503A200053456E
:10162000524750533A200000343830302042640092
:101630003936303020426400313932303020426453
:10164000000054656C656D657472793A20005465CC
:101650006C656D6574727920646174613A20000074
:101660004E4F524D414C00002C204368323A20002E
:101670002C204368333A20002C204368343A200061
:101680002C204368353A20004D61782064657669E6
:101690006174696F6E206973203130303020487A70
:1016A00000004D6178206261756472617465206923
:1016B000732031303030204264004D617820646105
:1016C00074612062697473206973203800004D6171
:1016D000782073746F70206269747320697320328C
:1016E000000056455253494F4E3A204243504C2039
:1016F000762E0000564261743A20000054656D70E9
:101700003A2000004E6F6D696E616C20506F7574E9
:101710003A20000055202D205057522055702C2083
:1017200044202D2050575220446F776E2C204520A6
:101730002D20457869742C2053202D205361766527
:101740000000436F6D6D616E647320287769746863
:10175000206578616D706C65293A200044495350CA
:101760002020202020202D20446973706C61792076
:10177000616C6C20736574696E6773004D594361C9
:101780006C6C202020202D20286D7963616C6C20EA
:101790004F4D3342432D313129005452616365204E
:1017A000202020202D2028786D69742F6F666629EF
:1017B00020666F7220646562756767696E67206F67
:1017C0006E6C7900545844656C61792020202D207E
:1017D000747864656C6179206E20303C6E3C3130E9
:1017E0003020286E2078203130206D732900545825
:1017F0005461696C202020202D2054582074616988
:101800006C2074696D6520286E2078203130206D41
:1018100073290000554E50726F746F2020202D20C8
:1018200028756E70726F746F2061707273207620ED
:1018300077696465312D3129202D20332064696753
:101840006973206D6178000053594D424F4C202040
:1018500020202D203220415052532073796D626F29
:101860006C73202D2064656661756C74206973202B
:1018700042414C4C4F4F4E20282F4F2900004652DA
:1018800051202020202020202D2066726571756552
:101890006E637920666F72204150525320696E202A
:1018A000487A0000524652512020202020202D202E
:1018B0006672657175656E637920666F7220525429
:1018C0005459202620435720696E20487A005254EC
:1018D00054592020202020202D204F4E206F722090
:1018E0004F464600415052532020202020202D20DA
:1018F0004F4E206F72204F46460044455620202010
:10190000202020202D20646576696174696F6E2027
:10191000696E20487A004241554420202020202032
:101920002D20626175647261746520666F72205249
:10193000545459207472616E736D697474696E6762
:101940000000444249545320202020202D206E7551
:101950006D626572206F6620646174616269747380
:101960000000534249545320202020202D206E7522
:101970006D626572206F662073746F706269747334
:1019800020312E35203D2031350042415456202053
:10199000202020202D2073656E64206261746572A2
:1019A0007920766F6C7461676520285254545929E8
:1019B000202D20594553206F72204E4F0000535563
:1019C00050562020202020202D2073656E64207327
:1019D0007570706C7920766F6C7461676520285221
:1019E00054545929202D20594553206F72204E4FB1
:1019F000000054454D502020202020202D207365CC
:101A00006E6420696E626F782074656D70657261B6
:101A10007475726520285254545929202D20594537
:101A200053206F72204E4F00494E54454D50202098
:101A300020202D2073656E6420726164696F636875
:101A400069702074656D70657261747572652028A7
:101A50005254545929202D20594553206F72204E3D
:101A60004F00455854454D50202020202D207365AF
:101A70006E642065787465726E616C2074656D703B
:101A80006572617475726520285254545929202D4D
:101A900020594553206F72204E4F0000504F55542F
:101AA0002020202020202D206F75747075742070E8
:101AB0006F77657220696E206D5700005245462091
:101AC0002020202020202D20584F206F72205443AA
:101AD000584F206672657175656E637920696E2056
:101AE000487A20286D696E2E203130303030303009
:101AF000302C206D61782E20333230303030303051
:101B0000000055424C4F5820202020202D204F4EC1
:101B1000203D2055424C4F582C204F4646203D201A
:101B20005155454354454C005052455353757265C9
:101B300020202D204F4E203D20424D503138302066
:101B400070726573656E742C204F4646203D206E82
:101B50006F742070726573656E740000484F4C445A
:101B60006F66662020202D20686F6C64206F66668B
:101B70002074696D6520696E206D696E757465737A
:101B80000000435749442020202020202D20736549
:101B90006E64204357206964656E74696669657276
:101BA000204F4E206F72204F46460000435742415F
:101BB0005420202020202D2073656E6420626174E3
:101BC00065727920766F6C746167652028435729A8
:101BD000202D20594553206F72204E4F000043574F
:101BE00054454D50202020202D2073656E642074B4
:101BF000656D706572617475726520284357292080
:101C00002D20594553206F72204E4F00435753509B
:101C10002020202020202D207370656564206F66B1
:101C2000204357206964656E74696669657220692E
:101C30006E2057504D0043574C202020202020205C
:101C40002D2073656E6420515241206C6F632E20ED
:101C5000616E6420616C74697475646520696E20BE
:101C60004357202D20594553206F72204E4F0000BE
:101C70004C4F4341544F522020202D2073656E64F9
:101C800020515241206C6F6361746F72202D205976
:101C90004553206F72204E4F00004C4F433130208F
:101CA000202020202D2073656E6420313020636851
:101CB00061722E206F6620515241206C6F632E207E
:101CC0004F4E203D2031302C204F4646203D2036BF
:101CD0002063686172616B7465727300534F4C418D
:101CE0005263656C6C202D206D6F756E7465642079
:101CF0002D204F4E206F72206E6F74206D6F756EA9
:101D0000746564202D204F46460055534F4C2020CB
:101D1000202020202D2073656E6420736F6C61720B
:101D200020766F6C74616765202D20594553206FB4
:101D300072204E4F000049534F4C2020202020207D
:101D40002D2073656E6420736F6C617220637572F1
:101D500072656E7420594553206F72204E4F0000FB
:101D60004543484F2020202020202D204F4E206F1B
:101D700072204F464600534C4545502020202020DD
:101D80002D20737769746368207468652047505309
:101D9000207265636569766572202D204F4E206F35
:101DA00072204F4646005345524750532020202072
:101DB0002D206261756472617465206F66204750E2
:101DC0005320726563656976657220283438303037
:101DD000206F722039363030206F72203139323026
:101DE0003029000043414C494252415445202D20A6
:101DF00063616C6962726174652031323030487A97
:101E00000000444154412020202020202D206964DE
:101E1000656E74696669636174696F6E206F6620B0
:101E200074686520726164696F206368697000007E
:101E3000475053202020202020202D204F4E202DA1
:101E400020666F72206E6F726D616C206D6F6465BD
:101E50002C204F4646202D20666F722074657374C7
:101E6000696E6720776974686F75742047505320D6
:101E700072656365697665720000564552202020C0
:101E8000202020202D20736F667477617265207684
:101E9000657273696F6E00004558495420202020F8
:101EA00020202D20656E64206F6620636F6D6D614C
:101EB0006E6420696E74657270726574657200007C
:101EC0005441494C20287461696C207465787420F1
:101ED0006576657279206E292D286F6E2C6F666687
:101EE0002C6E292D6E3D30206973206F666620614F
:101EF0006E6420313C6E3C39206576657279206EC7
:101F00002D7468206D65737361676500545445587E
:101F10005420202020202D207461696C2074657865
:101F200074202D20313030206368617273206D6120
:101F300078005461696C207465787420636F6D6DEE
:101F4000616E64733A005C55202020202020202000
:101F50002D2073656E642062617465727920766FDE
:101F60006C74616765005C562020202020202020B2
:101F70002D2073656E642073797374656D20766FA0
:101F80006C74616765005C53202020202020202095
:101F90002D2073656E6420736F6C617220766F6C98
:101FA0007461676500005C492020202020202020EB
:101FB0002D2073656E6420736F6C6172206375727F
:101FC00072656E7400005C542020202020202020A8
:101FD0002D2073656E6420696E7465726E616C206D
:101FE00074656D7065726174757265005C5820204F
:101FF0002020202020202D2073656E6420657874B9
:1020000065726E616C2074656D7065726174757255
:1020100065005C5720202020202020202D20736583
:102020006E6420726164696F636869702074656DA5
:10203000706572617475726500005C50202020200C
:10204000202020202D2073656E64207072657373CC
:10205000757265005C4620202020202020202D2045
:1020600073656E642074656D7065726174757265F8
:102070002066726F6D207072657373757265207360
:10208000656E736F72005C4220202020202020208B
:102090002D2073656E64206E756D626572206F66AB
:1020A00020726563656976656420736174656C6C24
:1020B0006974657300005C5A2020202020202020B5
:1020C0002D20736F6674776172652076657273690F
:1020D0006F6E000054454C656D65747279202D203B
:1020E0004F4E206F72204F4646005241572020200D
:1020F000202020202D207365742072617720746564
:102100006C656D6574726963206461746120283048
:102110002D39393929004176616C6961626C65201D
:1021200076616C75657320666F722074656C656D81
:10213000657472793A0031202D206F6E626F617282
:10214000642074656D70657261747572650032200B
:102150002D2065787465726E616C2074656D706594
:10216000726174757265000033202D20726164699C
:102170006F636869702074656D70657261747572E3
:10218000650034202D2062617465727920766F6C51
:1021900074616765000035202D2073797374656D57
:1021A00020766F6C74616765000036202D20736F98
:1021B0006C617263656C6C20766F6C74616765002E
:1021C00037202D206368617267696E6720637572BE
:1021D00072656E74000038202D2061697220707263
:1021E000657373757265000039202D206865617212
:1021F000642073617474656C6974657300003020C9
:102200002D206368616E6E656C206E6F742075732F
:1022100065640000526164696F2063686970206EB4
:102220006F7420636F6E6E65637465640000526145
:1022300064696F206368697020636F6D6D756E6986
:10224000636174696F6E206572726F72000043681B
:102250006970205265766973696F6E3A200050612B
:1022600072743A205369000050617274204275699B
:102270006C643A203078000044657363726970744E
:10228000696F6E2049643A2030780000437573749A
:102290006F6D65722049643A20307800524F4D20AE
:1022A00049643A203078000024504D544B3130328C
:1022B0002A33310053617665643A20004E6F7420F2
:1022C0007361766564202D2041637475616C20769E
:1022D000616C75653A2000004E6F20636F6D6D75FF
:1022E0006E69636174696F6E0000424354524143EA
:1022F0004B2000002C3030303030303030004E6F0A
:102300007468696E6700496E742E54656D700000C4
:102310004578742E54656D70000052432E54656DDF
:1023200070004261742E566F6C7400005379732EE6
:10233000566F6C740000536F6C2E566F6C740000F7
:10234000536F6C2E43757272000050726573737513
:102350007265000053617474656C69746573000084
:102360003A5041524D2E00003A554E49542E00002D
:102370003A45514E532E00003A424954532E3030C4
:102380003030303030302C42414C4C4F4F4E204595
:1023900058504552494D454E54002C4E432C4E4307
:1023A0002C4E432C4E432C4E432C4E432C4E432C50
:1023B0004E43000054656D70496E0000302C302E85
:1023C000312C2D34300054656D7045780000546513
:1023D0006D7052430000302C302E3030322C3000E3
:1023E000302C302E30312C300000302C312C2D315F
:1023F00030300000302C312C353000000800000057
:10240000090000000A0000000B0000000C000000A2
:102410000D0000000E00000010000000120000007F
:1024200014000000170000001A0000001E00000049
:1024300022000000270000002D00000036000000F0
:10244000460000005E0000007F0000007F000000EA
:102450007F00000008000000090000000A000000E2
:102460000B0000000C0000000D0000000E0000003A
:10247000100000001200000014000000170000000F
:102480001A0000001E0000002200000027000000CB
:102490002D00000036000000460000005E00000035
:1024A0007F0000007F0000007F00000008000000A7
:1024B000090000000A0000000B0000000C000000F2
:1024C0000D0000000E0000001000000012000000CF
:1024D00014000000170000001A0000001E00000099
:1024E00022000000270000002D0000003600000040
:1024F000460000005E0000007F0000007F0000003A
:102500007F000000400E3F6E006A7086A00E756E60
:10251000010E766E200E726E900E716E0F01386B8A
:10252000396B3A6B796A786A606A0001AB0E926E19
:102530009A0E936E1D0E946EF40ED36ED26AC00E78
:102540009B6E796A786AF26AF16AF06A816A010EB2
:10255000C26E080EC16EAB0EC06E0B0E0F01386F4F
:10256000396B080E3A6FE00E426F416F100E406FEC
:102570009E0E9C6E9D6AA06A040E9F6EA26A070E54
:10258000D56E460ECD6ECC6ABD6A2F0EBA6E140E95
:10259000516F4E6B4A6BC66A6C6AAC98AC84B88655
:1025A000060EB06E800EAF6EAB9E7086729872840F
:1025B000060E766E800E756E718E0301176B186BAA
:1025C000196B156B166B00EE8AF0EF6A00EE90F057
:1025D000EF6A00EE9BF0EF6A00EEA6F0EF6A00EE05
:1025E000B1F0EF6A00EEBCF0EF6A00EEC7F0EF6A00
:1025F00000EED2F0EF6A0601786B776B766B756B45
:102600007A6B796B636BB56B706B6F6BB86B010E2C
:10261000B76FB981030118910601B99503014B6B9E
:102620004C6B4E6F2C0E4D6F010E0601946F2C0EED
:10263000936F640E956F996B030117931A6B0601E4
:10264000B997B999AA6A3A0EA96E69EC02F003012A
:102650002F6F69EC02F0306F000189EC47F0030145
:1026600012510001E8BC12D1030112510001E8B877
:102670001ED0800E026E400E096E226A9BC621F0AB
:10268000066A056A200E016EA66AA68E0F0EF76E08
:102690006E0EF66E0900F55003E066EC01F0FAD715
:1026A0000D0E66EC01F00A0E66EC01F0EFD0800E24
:1026B000026E400E096E226A9BC621F0066A056A08
:1026C000200E016EB50E66EC01F0620E66EC01F0B4
:1026D000060E66EC01F0110E66EC01F0020E66ECDF
:1026E00001F0000E66EC01F0080E66EC01F0040E3D
:1026F00066EC01F0250E66EC01F0950E66EC01F03B
:10270000B50E66EC01F0620E66EC01F0060E66ECAA
:1027100001F0090E66EC01F00D0E66EC01F0000E02
:1027200066EC01F0000E66EC01F0000E66EC01F0C4
:10273000000E66EC01F0000E66EC01F0FF0E66EC98
:1027400001F0FF0E66EC01F0000E66EC01F0000EE9
:1027500066EC01F0000E66EC01F0000E66EC01F094
:10276000000E66EC01F0000E66EC01F0070E66EC60
:1027700001F0210E66EC01F0AF0E66EC01F0800E68
:10278000026E400E096E226A9BC621F0066A056A37
:10279000200E016EB50E66EC01F0620E66EC01F0E3
:1027A000060E66EC01F0110E66EC01F0000E66EC10
:1027B00001F0000E66EC01F0170E66EC01F04B0E16
:1027C00066EC01F0640ED7EC02F0800E026E400E53
:1027D000096E226A9BC621F0066A056A200E016E08
:1027E000B50E66EC01F0620E66EC01F0060E66ECCA
:1027F00001F0570E66EC01F0080E66EC01F0000ED9
:1028000066EC01F0010E66EC01F0000E66EC01F0E2
:10281000000E66EC01F0000E66EC01F0500E66EC66
:1028200001F04F0E66EC01F0540E66EC01F0530E11
:1028300066EC01F0AC0E66EC01F0850E66EC01F082
:10284000800E026E400E096E226A9BC621F0066A57
:10285000056A200E016EB50E66EC01F0620E66ECA4
:1028600001F0060E66EC01F0570E66EC01F0000E6A
:1028700066EC01F0000E66EC01F05D0E66EC01F016
:102880001D0E66EC01F0640ED7EC02F0949A8B8A70
:1028900094928B925A0E03015C630AD05A0E5D63C8
:1028A00007D05A0E5E6304D05F515A0A000102E05D
:1028B000000E01D0010E3C6E000E030112B7010E96
:1028C0003C16000119E003012C6B2B6B010E030178
:1028D0002C5D000106E310E12D0E03012B5D0001CC
:1028E0000BE2070E166ED00ED8EC02F003012B2B74
:1028F000000E2C230001EAE39482949A8B8A640EE2
:10290000D7EC02F0949A8B8A020E166E580ED8EC11
:1029100002F0949A8B9A46C65CF645C65BF644C6AE
:102920005AF643C659F6C2EC4AF0C80ED7EC02F08C
:10293000070E0501E06F020EE16F010EE26FE36F1B
:102940005CC6E4F55BC6E5F55AC6E6F559C6E7F59B
:10295000000168EC50F0140ED7EC02F0040E0501F3
:10296000E06F200EE16FE26BE36BE46B000168EC5B
:1029700050F0140ED7EC02F0080E0501E06F130EB4
:10298000E16F040EE26F150EE36F210EE46F200E6F
:10299000E56F080EE66F0B0EE76FE86B000168EC61
:1029A00050F013EC5BF092EC26F0080E06013E2589
:1029B00003011C6F050E0501E06F110EE16F200E83
:1029C000E26F010EE36F510EE46F1CC3E5F50001E9
:1029D00048EC50F0060E0501E06F110EE16F200E7D
:1029E000E26F020EE36F0D0EE46FE56BE66B000124
:1029F00048EC50F0050E0501E06F110EE16F220E5C
:102A0000E26F010EE36FE46B080EE56F000148EC26
:102A100050F061C62CF6060161510001E8BE08D0F5
:102A2000180E0601615D000103E3170E0601616FD8
:102A3000000199EC25F00601626B0001AAEC25F07B
:102A4000050E0501E06F110EE16FE26B010EE36F01
:102A5000E46FE56F000148EC50F00C0E0501E06FEB
:102A6000110EE16F200EE26F080EE36F180EE46F97
:102A7000010EE56FE66B080EE76F020EE86F800E41
:102A8000E96FEA6BF00EEB6F100EEC6F000148EC93
:102A900050F00D0E0501E06F110EE16F200EE26F98
:102AA000090EE36F220EE46FE56B820EE66F030EF4
:102AB000E76FEE0EE86FA20EE96F020EEA6F5D0E91
:102AC000EB6F020EEC6FED6B000148EC50F00C0E5A
:102AD0000501E06F110EE16F200EE26F080EE36F4B
:102AE000420EE46FA40EE56F030EE66FD60EE76F9D
:102AF000030EE86FE96BF50EEA6F010EEB6F800EC7
:102B0000EC6F000148EC50F0100E0501E06F110E63
:102B1000E16F210EE26F0C0EE36FE46BA20EE56F26
:102B2000810EE66F260EE76FAF0EE86F3F0EE96F7E
:102B3000EE0EEA6FC80EEB6FC70EEC6FDB0EED6F9B
:102B4000F20EEE6F020EEF6F080EF06F000148EC10
:102B500050F0100E0501E06F110EE16F210EE26FD3
:102B60000C0EE36FE46F070EE56F030EE66F150EB4
:102B7000E76FFC0EE86F0F0EE96FEA6BA20EEB6FCA
:102B8000810EEC6F260EED6FAF0EEE6F3F0EEF6F06
:102B9000EE0EF06F000148EC50F0100E0501E06FF2
:102BA000110EE16F210EE26F0C0EE36F180EE46F51
:102BB000C80EE56FC70EE66FDB0EE76FF20EE86F2B
:102BC000020EE96F080EEA6F070EEB6F030EEC6F53
:102BD000150EED6FFC0EEE6F0F0EEF6FF06B000138
:102BE00048EC50F0080E0501E06F110EE16F220E67
:102BF000E26F040EE36FE46B080EE56F7F0EE66F85
:102C0000E76B3D0EE86F000148EC50F00B0E05013C
:102C1000E06F110EE16F230EE26F070EE36FE46BBE
:102C20002C0EE56F0E0EE66F0B0EE76F040EE86FCD
:102C30000C0EE96F730EEA6F030EEB6F000148ECA8
:102C400050F07BEC25F0D6EC25F0320ED7EC02F0FC
:102C5000C2EC25F078EC68F07BEC25F0BCEC26F0BB
:102C6000350E0601606F00017FEC6CF0EAEF29F091
:102C7000719E9482030112510001E8AA02D017EC60
:102C80005DF0030114510001E8AA02D0DBEC55F01D
:102C9000030112350001D8A058D00EEC45F000EE2B
:102CA000E8F0EE50FEE1ED520F0EF76E7C0EF66E80
:102CB00018EC04F0020E016E086A1A6A0E0E196E04
:102CC00069EC00F02E0EEE6E020E016E010E086E23
:102CD0008C0E67EC00F0EF6A06018F6B040E0301A7
:102CE0001C6F000100EEE8F003011C51E926000E04
:102CF000EA22EF500C6E0C5200010FE000EEE8F0FB
:102D000003011C51E926000EEA22EF500C6E060169
:102D10008F1B03011C2B0001E4D700EEE8F0EE50FE
:102D2000FEE1ED522A0EEE6E020E016E086E0601F5
:102D30008F514FEC00F00D0EEE6E0A0EEE6EEF6A44
:102D40000001BBEC26F054EC65F0030112510001C8
:102D5000E8BC67D282949494640ED7EC02F0948419
:102D6000030E166EE80ED8EC02F0030112510001BA
:102D7000E8A837D2800E026E400E096E226A9BC60A
:102D800021F0066A056A200E016EB50E66EC01F0B0
:102D9000620E66EC01F0060E66EC01F03B0E66EC8E
:102DA00001F02C0E66EC01F0000E66EC01F0010E55
:102DB00066EC01F0060E66EC01F0000E66EC01F028
:102DC000000E66EC01F0000E66EC01F0900E66EC71
:102DD00001F0020E66EC01F0000E66EC01F0E80E68
:102DE00066EC01F0030E66EC01F0000E66EC01F0FB
:102DF000000E66EC01F0100E66EC01F0800E026E23
:102E0000400E096E226A9BC621F0066A056A200EF2
:102E1000016E270E66EC01F0000E66EC01F0000E6C
:102E200066EC01F0000E66EC01F0000E66EC01F0BD
:102E3000000E66EC01F0000E66EC01F0000E66EC90
:102E400001F0000E66EC01F0000E66EC01F0000EE1
:102E500066EC01F02C0E66EC01F0010E66EC01F060
:102E6000000E66EC01F0000E66EC01F04F0E66EC11
:102E700001F0C10E66EC01F0030E66EC01F0000EED
:102E800066EC01F0800E026E400E096E226A9BC64F
:102E900021F0066A056A200E016E860E66EC01F0CE
:102EA000020E66EC01F0000E66EC01F0000E66EC1E
:102EB00001F0FE0E66EC01F0000E66EC01F0000E73
:102EC00066EC01F0000E66EC01F0640E66EC01F0B9
:102ED000400E66EC01F0010E66EC01F0000E66ECAF
:102EE00001F0930E66EC01F0950E66EC01F0800E99
:102EF000026E400E096E226A9BC621F0066A056AC0
:102F0000200E016EB50E66EC01F0620E66EC01F06B
:102F1000060E66EC01F03B0E66EC01F0000E66EC6E
:102F200001F0000E66EC01F0410E66EC01F0C90EF6
:102F300066EC01F0640ED7EC02F0800E026E400EDB
:102F4000096E226A9BC621F0066A056A200E016E90
:102F5000B50E66EC01F0620E66EC01F0060E66EC52
:102F600001F0160E66EC01F0080E66EC01F0000EA2
:102F700066EC01F0010E66EC01F0030E66EC01F068
:102F8000030E66EC01F0000E66EC01F0510E66ECEB
:102F900001F0080E66EC01F0000E66EC01F0000E88
:102FA00066EC01F0840E66EC01F0150E66EC01F0A3
:102FB000800E026E400E096E226A9BC621F0066AE0
:102FC000056A200E016EB50E66EC01F0620E66EC2D
:102FD00001F0060E66EC01F0160E66EC01F0000E34
:102FE00066EC01F0000E66EC01F01C0E66EC01F0E0
:102FF0005A0E66EC01F0640ED7EC02F0800E026E01
:10300000400E096E226A9BC621F0066A056A200EF0
:10301000016EB50E66EC01F0620E66EC01F0060E74
:1030200066EC01F0110E66EC01F0020E66EC01F0A8
:10303000000E66EC01F0080E66EC01F0040E66EC82
:1030400001F0250E66EC01F0950E66EC01F0B50E70
:1030500066EC01F0620E66EC01F0060E66EC01F023
:10306000090E66EC01F00D0E66EC01F0000E66EC48
:1030700001F0000E66EC01F0000E66EC01F0000EAF
:1030800066EC01F0000E66EC01F0FF0E66EC01F05C
:10309000FF0E66EC01F0000E66EC01F0000E66EC2F
:1030A00001F0000E66EC01F0000E66EC01F0000E7F
:1030B00066EC01F0000E66EC01F0070E66EC01F024
:1030C000210E66EC01F0AF0E66EC01F0800E026E90
:1030D000400E096E226A9BC621F0066A056A200E20
:1030E000016EB50E66EC01F0620E66EC01F0060EA4
:1030F00066EC01F0110E66EC01F0000E66EC01F0DA
:10310000000E66EC01F0170E66EC01F04B0E66EC5B
:1031100001F0640ED7EC02F000EEE8F00F0EF76E4F
:10312000880EF66E18EC04F0EF6A16EC6CF0640E84
:10313000D7EC02F000EEE8F00F0EF76EA00EF66E80
:1031400018EC04F0EF6A16EC6CF0640ED7EC02F0A9
:1031500000EEE8F00F0EF76EB80EF66E18EC04F005
:10316000EF6A16EC6CF0640ED7EC02F000EEE8F0BB
:103170000F0EF76ED00EF66E18EC04F0EF6A16EC38
:103180006CF0640ED7EC02F000EEE8F00F0EF76E74
:10319000E80EF66E18EC04F0EF6A16EC6CF0640EB4
:1031A000D7EC02F000EEE8F0100EF76E000EF66EAF
:1031B00018EC04F0EF6A16EC6CF0640ED7EC02F039
:1031C00000EEE8F0100EF76E180EF66E18EC04F034
:1031D000EF6A16EC6CF0640ED7EC02F0CBEC62F008
:1031E0000BD000EEE8F0100EF76E300EF66E18EC15
:1031F00004F0EF6A16EC6CF0640ED7EC02F08DEC84
:103200006BF00301183100010CE3300E0601606F12
:1032100000017FEC6CF0010E166EF40ED8EC02F09B
:10322000A4D53D0E0601606F2CC661F6000199EC35
:1032300025F0A2D1030156530001D8B49DD1030E4D
:103240000601995D000106E2EA0E166E600ED8ECEA
:1032500002F092D103011731000103E3010E0301D3
:10326000566F030112510001E8A486D003011251E8
:103270000001E8B81ED0800E026E400E096E226A70
:103280009BC621F0066A056A200E016EA66AA68E0C
:103290000F0EF76E6E0EF66E0900F55003E066EC49
:1032A00001F0FAD70D0E66EC01F00A0E66EC01F0A3
:1032B0005ED0800E026E400E096E226A9BC621F01F
:1032C000066A056A200E016EB50E66EC01F0620E0C
:1032D00066EC01F0060E66EC01F0570E66EC01F0AC
:1032E000080E66EC01F0000E66EC01F0010E66ECD3
:1032F00001F0000E66EC01F0000E66EC01F0000E2D
:1033000066EC01F0500E66EC01F04F0E66EC01F039
:10331000540E66EC01F0530E66EC01F0AC0E66EC58
:1033200001F0850E66EC01F0800E026E400E096E13
:10333000226A9BC621F0066A056A200E016EB50E50
:1033400066EC01F0620E66EC01F0060E66EC01F030
:10335000570E66EC01F0000E66EC01F0000E66EC14
:1033600001F05D0E66EC01F01D0E66EC01F0640EDE
:10337000D7EC02F094928B92A20ED36ED2889B9CD3
:10338000C290020E0301565D000109E303015607D6
:10339000010E166ED50ED8EC02F00001F2D7010E28
:1033A0000301246FD50E236F14510001E8A605D048
:1033B000200E0301235F000E245B03011231000184
:1033C00005E3400E0301235F000E245B0301123569
:1033D000000105E3730E0301235F000E245B03016C
:1033E00014510001E8AA07D0060E0301235F000E66
:1033F000245B000112D0030114510001E8AC0DD090
:10340000750E0301235F000E245B1435000105E3F4
:10341000750E0301235F000E245B24C316F0030125
:103420002351D8EC02F09B8CD298F40ED36EC2805C
:1034300012510001E8A611D023EC53F006017ABF27
:1034400008D07A53000109E10F0E0601795D0001F1
:1034500004E2D89003015637562B030112510001A4
:10346000E8A485D09482640ED7EC02F003011251D7
:103470000001E8B81ED0800E026E400E096E226A6E
:103480009BC621F0066A056A200E016EA66AA68E0A
:10349000100EF76E620EF66E0900F55003E066EC52
:1034A00001F0FAD70D0E66EC01F00A0E66EC01F0A1
:1034B0005ED0800E026E400E096E226A9BC621F01D
:1034C000066A056A200E016EB50E66EC01F0620E0A
:1034D00066EC01F0060E66EC01F0570E66EC01F0AA
:1034E000080E66EC01F0000E66EC01F0010E66ECD1
:1034F00001F0000E66EC01F0000E66EC01F0000E2B
:1035000066EC01F0200E66EC01F04E0E66EC01F068
:10351000550E66EC01F0520E66EC01F07B0E66EC87
:1035200001F0C30E66EC01F0800E026E400E096ED3
:10353000226A9BC621F0066A056A200E016EB50E4E
:1035400066EC01F0620E66EC01F0060E66EC01F02E
:10355000570E66EC01F0000E66EC01F0000E66EC12
:1035600001F05D0E66EC01F01D0E66EC01F0070E39
:10357000166ED00ED8EC02F0AA6A2D0EA96E69EC78
:1035800002F00301566F5553000102E00301550795
:1035900000013CD9010E0601945D000108E305E13C
:1035A0002C0E0601935D000102E3000E01D0010E16
:1035B0003C6E000E030117B3010E3C16000106E03D
:1035C000030117810001A2EC23F00AD1030112319B
:1035D000000102E3BEEC23F0030E0601995D000139
:1035E000D8A0FED0030114510001E8AA02D0F5ECE6
:1035F00022F003011235000102E363EC63F00301E2
:1036000056530001D8B4BAD0130E166E880ED8ECFB
:1036100002F0FCD8010E0601945D000108E305E10B
:10362000F40E0601935D000102E3000E01D0010ECD
:103630003C6E000E030117B3010E3C16000106E0BC
:10364000030117810001A2EC23F00DD003011451F6
:103650000001E8AA02D0F5EC22F0030112350001C6
:1036600002E336EC63F0030112510001E8A486D0B6
:10367000030112510001E8B81ED0800E026E400E08
:10368000096E226A9BC621F0066A056A200E016E49
:10369000A66AA68E0F0EF76E6E0EF66E0900F55036
:1036A00003E066EC01F0FAD70D0E66EC01F00A0EAD
:1036B00066EC01F05ED0800E026E400E096E226A4A
:1036C0009BC621F0066A056A200E016EB50E66ECF7
:1036D00001F0620E66EC01F0060E66EC01F0570E8A
:1036E00066EC01F0080E66EC01F0000E66EC01F0ED
:1036F000010E66EC01F0000E66EC01F0000E66ECC7
:1037000001F0000E66EC01F0500E66EC01F04F0E79
:1037100066EC01F0540E66EC01F0530E66EC01F01D
:10372000AC0E66EC01F0850E66EC01F0800E026EC8
:10373000400E096E226A9BC621F0066A056A200EB9
:10374000016EB50E66EC01F0620E66EC01F0060E3D
:1037500066EC01F0570E66EC01F0000E66EC01F02D
:10376000000E66EC01F05D0E66EC01F01D0E66ECDD
:1037700001F0640ED7EC02F094928B92000E0301DC
:1037800014BD010E3C6E000E14BB010E3C16000170
:1037900027E003015653000105E02E0E166EE00EE1
:1037A000D8EC02F0E2EC26F0B3EC67F0000E030177
:1037B00014BF010E3C6E5653000102E1000E01D011
:1037C000010E3C1608E03A0E166E980ED8EC02F088
:1037D000F8EC67F005D0070E166ED00ED8EC02F0AC
:1037E000010E03015553D8A4000E3C6E000E14BB0D
:1037F000010E3C16000107E0AA6A2B0EA96E69ECC7
:1038000002F00301556F00011AEF19F00301125184
:103810000001E8AC4DD003EE60F0100EF76E6E0EB6
:10382000F66E18EC04F0EF6A03EEB6F0100EF76EC9
:10383000B80EF66E18EC04F00D0EEE6E0A0EEE6E7B
:10384000EE6A06018F6B03011A6B000103EE60F054
:1038500003011A51EB500C6E2A0E0C5CD8A4010E19
:103860003C6E4F0E1A5D010ED8B0000E3C160001E2
:103870000CE003EE60F003011A51EB500C6E0601F0
:103880008F1B03011A2B0001E0D703EE60F0EE500E
:10389000FEE1ED52020E016E086E06018F514FECF3
:1038A00000F00D0EEE6E0A0EEE6EEF6A0001F2D021
:1038B0000601A46BB99BB99D000104EE0CF0240E27
:1038C000EE6E470EEE6EEF6A800E026E800E096E8F
:1038D000226A9BC621F00B0E066EB80E056E27EC11
:1038E00001F0D8A0E8EF22F02408F9E127EC01F07C
:1038F000D8A0E8EF22F003011C6F020E1A6F510EE0
:1039000003011A5D00011BE2800E026E800E096E3B
:10391000226A9BC621F043EC01F003011C6F04EE08
:103920000CF01A51E926000EEA221CC3EFFF2A0E02
:103930001C5D000104E003011A2B0001E0E3800E8E
:10394000026E800E096E226A9BC621F043EC01F0E4
:1039500003011C6F0D6A1A290C6ED8B40D2A0C5085
:103960000C0FE96E040E0D20EA6E1CC3EFFF800EF3
:10397000026E800E096E226A9BC621F043EC01F0B4
:103980001C6F0D6A020E1A250C6ED8B00D2A0C5051
:103990000C0FE96E040E0D20EA6E1CC3EFFF0D6ADA
:1039A000030E1A250C6ED8B00D2A0C500C0FE96EC0
:1039B000040E0D20EA6EEF6A04010D510C6E470EE5
:1039C0000C5C010ED8A4000E3C6E0F510C6E470E1D
:1039D0000C5C010ED8A4000E3C1610510C6E470E64
:1039E0000C5C010ED8A4000E3C1611510C6E410E59
:1039F0000C5C010ED8A4000E3C1600010EE003EE94
:103A000060F014EE0CF0FF0EE75204E0E6CFEEFF9C
:103A1000E82EFAD7EF6A0601B98B04010D510C6E3E
:103A2000470E0C5C010ED8A4000E3C6E0F510C6EBC
:103A3000560E0C5C010ED8A4000E3C1610510C6EF4
:103A4000540E0C5C010ED8A4000E3C1611510C6EE5
:103A5000470E0C5C010ED8A4000E3C1600010EE0CF
:103A600003EEB6F014EE0CF0FF0EE75204E0E6CFE2
:103A7000EEFFE82EFAD7EF6A0601B98D010E0601B6
:103A8000B9BD000E3C6E010EB9BB000E3C12000128
:103A900001E012D704EE0CF013EEB6F0550EE7522B
:103AA00004E0E6CFEEFFE82EFAD7EF6A0501A46B3B
:103AB000A36BA66BA56B03011B6B0001FCEC26F04E
:103AC00005EEADF0EECFF3FFEFCFF4FFF450F310BF
:103AD00006E103013A6B396B386B000121D005EE2A
:103AE000ADF004EC00F00501A36F1AC0A4F5A4C565
:103AF00012F0A3C511F0000E14EC03F003013A6FAD
:103B0000A4C512F0A3C511F0010E14EC03F0396F37
:103B1000A4C512F0A3C511F0020E14EC03F0386F27
:103B200003011B6B000102EC27F005EEADF0EECFB8
:103B3000F3FFEFCFF4FFF450F31002E0000E01D0DA
:103B4000010E3C6E000E030112B9010E3C12000181
:103B500007E0300E03013D6F3C6F3B6F000121D049
:103B600005EEADF004EC00F00501A56F1AC0A6F556
:103B7000A6C512F0A5C511F0000E14EC03F0030168
:103B80003D6FA6C512F0A5C511F0010E14EC03F0AF
:103B90003C6FA6C512F0A5C511F0020E14EC03F09F
:103BA0003B6F0601986B04EE0CF013EE60F0550EBF
:103BB000E75204E0E6CFEEFFE82EFAD7EF6A030102
:103BC0001B6B0001FDEC26F00501AD510C6E300EB3
:103BD0000C5C0001D8B499EF22F00601A46B03013C
:103BE0001B6B000102EC27F001EE7FF015EEADF04B
:103BF000020EE6CFEEFFE82EFCD73A0EEE6E15EE83
:103C0000ADF0030EF36E020E20EC04F03A0EEE6EF1
:103C100015EEADF0050EF36E020E20EC04F0EF6A27
:103C200003011B6B000100EC27F00501AD510301FE
:103C30000E6F4E0E0E5D000107E10301188301EEC9
:103C40008FF0EF6A000110D0530E03010E5D0001EA
:103C500009E10301189301EE8FF02D0EEE6EEF6A6D
:103C6000000102D00301168703011B6B000101EC68
:103C700027F001EE8FF0EE50FEE1ED5215EEADF0C3
:103C8000080EE6CFEEFFE82EFCD7EF6A0501AD5136
:103C90000301426F0501AE510301436F0501AF51AE
:103CA0000301446F0501B0510301456F266A0A0EF6
:103CB000256E2A6A44C329F00F0E2916000E2A1613
:103CC00026C01EF025C01DF02AC016F029C015F030
:103CD000DFEC03F0256E1AC026F02A6A45C329F0EE
:103CE0000F0E2916000E2A16295025262A502622A4
:103CF0004B51255C116E000E2658126EFEEC03F03F
:103D00000C6E12C00DF00D5204E1030E0C5C0001AC
:103D100025E3266A0A0E256E2A6A44C329F00F0E8F
:103D20002916000E2A1626C01EF025C01DF02AC036
:103D300016F029C015F0DFEC03F0256E1AC026F04E
:103D40002A6A45C329F00F0E2916000E2A1625509F
:103D5000292403014B6F000106EF1CF0266A0A0EAE
:103D6000256E2A6A44C329F00F0E2916000E2A1662
:103D700026C01EF025C01DF02AC016F029C015F07F
:103D8000DFEC03F0256E1AC026F02A6A45C329F03D
:103D90000F0E2916000E2A162550292403014B6FF9
:103DA0000501B1510C6E2E0E0C5C000102E0030106
:103DB00016870501B2510301466F0501B351030196
:103DC000476F0F0E42151C6F1C5176EC07F03A6AD4
:103DD000396A200E386E820E376EC7EC06F036C098
:103DE00027F635C026F634C025F633C024F60F0E6C
:103DF00043151C6F1C5168EC07F027C63AF026C625
:103E000039F025C638F024C637F0D3EC05F036C0BB
:103E100027F635C026F634C025F633C024F60F0E3B
:103E200044151C6F1C51640DF3CF23F3F4CF24F31E
:103E30000F0E45151C6F1C510A0DF3CF1CF31C51BE
:103E40002327000E24230F0E46151C6F1C51232719
:103E5000000E24233A6A396A160E386E880E376EC1
:103E600024C334F023C333F078EC07F061EC06F0A0
:103E700036C028F035C027F034C026F033C025F016
:103E800027C63AF026C639F025C638F024C637F0E2
:103E900028C036F027C035F026C034F025C033F0F6
:103EA000D3EC05F036C027F635C026F634C025F62B
:103EB00033C024F618510001E8B218D0366A356ACA
:103EC000800E346E7F0E336E27C63AF026C639F068
:103ED00025C638F024C637F0C7EC06F036C027F602
:103EE00035C026F634C025F633C024F603011B6B1B
:103EF0000001FEEC26F00501AD5103010F6F450EE8
:103F00000F5D000107E10301189501EE9FF0EF6AD4
:103F1000000110D0570E03010F5D000109E10301FC
:103F2000188501EE9FF02D0EEE6EEF6A000102D0B3
:103F30000301168703011B6B0001FFEC26F001EE65
:103F40009FF0EE50FEE1ED5215EEADF0090EE6CF1A
:103F5000EEFFE82EFCD7EF6A0501AD510C6E0F0E97
:103F60000C140301486F266A48C325F026500A0D39
:103F7000F3CF26F025500A0DF3CF25F0F450262676
:103F80000501AE510C6E2A6A0CC029F00F0E2916DD
:103F9000000E2A16255029240301486F266A48C3BB
:103FA00025F026500A0DF3CF26F025500A0DF3CF49
:103FB00025F0F45026260501AF510C6E2A6A0CC07C
:103FC00029F00F0E2916000E2A1625502924030168
:103FD000486F0501B0510C6E0F0E0C140301496FB0
:103FE000266A49C325F026500A0DF3CF26F0255046
:103FF0000A0DF3CF25F0F45026260501B1510C6EC1
:104000002A6A0CC029F00F0E2916000E2A16255018
:1040100029240301496F4C51495D116E126AD8A0E1
:104020001206FEEC03F00C6E12C00DF00D5204E10E
:10403000030E0C5C000105E349C34CF3000106EFDD
:104040001CF049C34CF30501B3510C6E0F0E0C1458
:1040500003014A6F485176EC07F036C028F035C0AE
:1040600027F034C026F033C025F0495176EC07F034
:1040700036C02CF035C02BF034C02AF033C029F004
:10408000366A356A200E346E820E336E2CC03AF0DA
:104090002BC039F02AC038F029C037F0C7EC06F041
:1040A00036C02CF035C02BF034C02AF033C029F0D4
:1040B0004A5176EC07F02CC03AF02BC039F02AC0F8
:1040C00038F029C037F0D3EC05F036C02CF035C0FD
:1040D0002BF034C02AF033C029F03A6A396A160E40
:1040E000386E880E376E2CC036F02BC035F02AC0E3
:1040F00034F029C033F061EC06F036C02CF035C046
:104100002BF034C02AF033C029F028C03AF027C081
:1041100039F026C038F025C037F02CC036F02BC05F
:1041200035F02AC034F029C033F0D3EC05F036C0A6
:104130002BF635C02AF634C029F633C028F6266A95
:104140004AC325F026500A0DF3CF26F025500A0D5C
:10415000F3CF25F0F45026260501B4510C6E2A6ADF
:104160000CC029F00F0E2916000E2A1625502924FE
:1041700003014A6F18510001E8A418D0366A356A65
:10418000800E346E7F0E336E2BC63AF02AC639F09D
:1041900029C638F028C637F0C7EC06F036C02BF633
:1041A00035C02AF634C029F633C028F603011B6B4C
:1041B0000001FCEC26F005EEA7F015EEADF0320E96
:1041C000E75204E0E6CFEEFFE82EFAD7EF6A05EEFD
:1041D000A7F004EC00F00601996F030112510001F1
:1041E000E8BC1BD003011B6B0001FAEC26F001EECA
:1041F000AFF015EEADF0320EE75204E0E6CFEEFF81
:10420000E82EFAD7EF6A01EEAFF004EC00F00601F9
:10421000936F1AC094F600013FD0270E0601945DFB
:10422000000118E305E1100E0601935D000112E3A1
:1042300030C312F003012F51116EFE0DF3CF2FF397
:10424000F4CF30F31250FE0DF35030271150FF0D14
:10425000F350302703012F510601932703013051FA
:1042600006019423010E945D000106E308E12D0E82
:104270000601935D000103E20301306B2F6B000127
:1042800001EEAFF0020E016E086A94C61AF093C6F2
:1042900019F069EC00F0EF6A03014D510601935DDE
:1042A000116E03014E5106019459126EFEEC03F09B
:1042B0000C6E12C00DF0070E0D5C00010BE303E164
:1042C000D10E0C5C07E394C64EF393C64DF3000188
:1042D00006EF1CF094C64EF393C64DF3266A39C31D
:1042E00025F00F0E2516000E26162A6A0A0E296ED4
:1042F0002E6A38C32DF00F0E2D16000E2E162AC072
:104300001EF029C01DF02EC016F02DC015F0DFECF8
:1043100003F0296E1AC02AF0255029240301396FB1
:10432000140E395D000105E26C0E0301392700010E
:1043300003D0300E030139270001266A3BC325F064
:104340000F0E2516000E26162A6A0A0E296E2E6AF0
:104350003AC32DF00F0E2D16000E2E162AC01EF099
:1043600029C01DF02EC016F02DC015F0DFEC03F0B3
:10437000296E1AC02AF02550292403013B6F200E14
:104380003B27266A3CC325F00F0E2516000E261685
:104390002A6A0A0E296E2E6A3DC32DF00F0E2D16C5
:1043A000000E2E162AC01EF029C01DF02EC016F0D9
:1043B0002DC015F0DFEC03F0296E1AC02AF025504D
:1043C00029243D6F1C0E3D27200E4227200E432737
:1043D00018510001E8A203D0200E03014527640E06
:1043E0000301485D000ED8B0010E3C6E0A0E485D18
:1043F000010ED8B0000E3C12000103E0200E0301B4
:104400004627030118510001E8A403D0200E030140
:104410004727640E0301485D00010FE36E0E0301A0
:10442000485D000105E2080E03014827000103D0A2
:10443000480E0301485F00010DD00A0E0301485DDC
:10444000000105E31C0E03014827000103D0760E8E
:10445000030148270A0E0301495D000105E2580ED9
:1044600003014927000103D01C0E03014927000165
:104470001EC60CF01FC60DF00DC01DF60CC01CF6BC
:1044800020C60CF021C60DF00DC01FF60CC01EF6A4
:1044900022C60CF023C60DF00DC021F60CC020F68C
:1044A00094C623F693C622F622C60CF023C60DF05E
:1044B00020C60EF021C60FF00E500C5C0F500D58A8
:1044C00002E3000E01D0010E3C6E20C60CF021C6A6
:1044D0000DF01EC60EF01FC60FF00E500C5C0F50F4
:1044E0000D5802E3000E01D0010E3C161EC60CF062
:1044F0001FC60DF01CC60EF01DC60FF00E500C5C52
:104500000F500D5802E3000E01D0010E3C1610E0D2
:104510000301439B050E0601945D000108E305E1DC
:10452000DD0E0601935D000102E303011783000124
:104530004ED00601A42B0A0EA45D000141E3170E24
:104540000601616F000199EC25F000EEE8F00D0E18
:10455000EE6E100EF76EDE0EF66E18EC04F00D0E19
:10456000EE6EEE6A030114510001E8AA05D00301C2
:104570001B6B0001AEEC28F000EEE8F010EE4FF0FF
:10458000060EE6CFEEFFE82EFCD713EE60F0550ED8
:10459000E75204E0E6CFEEFFE82EFAD7EF6A030118
:1045A0001235000106E3BBEC26F054EC65F0E2ECBA
:1045B00026F00601A46BD60E166ED80ED8EC02F0CB
:1045C00000012CC661F699EC25F05CEF1CF012009E
:1045D00082949494640ED7EC02F09484030E166EC9
:1045E000E80ED8EC02F05CEF1CF01C0E03014A2729
:1045F00042C358F043C359F044C35AF045C35BF07B
:1046000046C35CF047C35DF05E6A48C30CF449C31F
:104610000DF44AC30EF439C30FF43BC310F43DC389
:1046200011F450C312F44FC313F4100E0601932576
:1046300003012D6F270E0601942103012E6F2EC357
:1046400012F02DC311F0200E166E590E156E4CECA3
:1046500003F0256E12C026F0210E25240C6E0CC02E
:1046600014F42EC312F02DC311F0200E166E590E45
:10467000156E4CEC03F01AC02EF319C02DF32EC3A7
:1046800012F02DC311F0166A5B0E156E4CEC03F0A0
:10469000256E12C026F0210E25240C6E0CC015F4D8
:1046A0002EC312F02DC311F0166A5B0E156E4CEC82
:1046B00003F01AC026F019C025F0210E25240C6E37
:1046C0000CC016F47D0E0401176F0D0E186F060155
:1046D000986BB9510001E8B602D04DEC56F0E2EC0F
:1046E00026F0D3EF28F082949494640ED7EC02F075
:1046F00094840601982B060E985D000121E300EEDC
:10470000E8F00D0EEE6E100EF76EF60EF66E18EC6B
:1047100004F00D0EEE6EEF6A0601986B0301145162
:104720000001E8AA05D003011B6B0001AEEC28F0E4
:1047300003011235000104E3BBEC26F054EC65F0F4
:1047400006EF1CF0BBEC26F0030114891487149DBE
:104750000601915176EC07F03A6A396A400E386EDC
:104760007F0E376EC7EC06F015EC07F08C6F34C087
:104770008DF6010E166EF40ED8EC02F00001939A3D
:104780008A9AB9D9BCEC26F0350E06015F6F00019C
:104790006ED903011A6B060E03011A5D00010EE2C9
:1047A00000EE4FF003011A51EB500C6E200E0C5C22
:1047B000000104E003011A2B0001EDE305EEADF06A
:1047C000110EF76E160EF66E18EC04F010EE4FF0A8
:1047D00003011A510001E6CFEEFFE82EFBD72F0EA2
:1047E000EE6E410EEE6E4D0EEE6EEE6A03011A6B2A
:1047F000000105EEADF003011A51EB500C6E0C52A6
:1048000000010DE005EEADF003011A51EB50060179
:10481000606F0001F1D803011A2B0001E9D70601EE
:104820008D51050DF3CF16F08C51050DF3CF15F01A
:10483000F4501626D9EC02F0030114510001E8A649
:104840002CD004EE0CF013EE60F0550EE75204E0AD
:10485000E6CFEEFFE82EFAD7EF6AE7EC4CF0010E58
:10486000166EF40ED8EC02F003011A6B000105EE8F
:10487000ADF003011A51EB500C6E0C5200010DE02B
:1048800005EEADF003011A51EB500601606F000117
:10489000B3D803011A2B0001E9D703011731000136
:1048A00033E3030114510001E8AA2BD0010E166E68
:1048B000F40ED8EC02F0E2EC26F004EE0CF0210E3F
:1048C000EE6E11EE8FF0070EE6CFEEFFE82EFCD76E
:1048D0000EC3EEFF4FC3EEFF11EE9FF0080EE6CFC2
:1048E000EEFFE82EFCD70FC3EEFF50C3EEFF0D0E18
:1048F000EE6EEF6A0301119D00014CEC27F0D9EC3C
:1049000028F063EC63F077D00601B981030113311D
:10491000000132E361EC52F0010E166EF40ED8EC99
:1049200002F005EEADF0200EEE6E550EEE6E10EEBE
:10493000A6F00A0EE75204E0E6CFEEFFE82EFAD723
:10494000560EEE6EEE6A03011A6B000105EEADF035
:1049500003011A51EB500C6E0C5200010DE005EEF4
:10496000ADF003011A51EB500601606F000144D80D
:1049700003011A2B0001E9D7030113510001E8A23A
:1049800039D01FEC51F09B510C6E2D0E0C5C02E1E6
:104990004E0E9B6F030E166EE80ED8EC02F005EE7D
:1049A000ADF0200EEE6E540EEE6E10EE9BF00A0E81
:1049B000E75204E0E6CFEEFFE82EFAD7430EEE6EA4
:1049C000EE6A03011A6B000105EEADF003011A5106
:1049D000EB500C6E0C5200010DE005EEADF0030142
:1049E0001A51EB500601606F000106D803011A2B23
:1049F0000001E9D7C7D81200200E0601605D000152
:104A00000FE106018D51050DF3CF16F08C51050D08
:104A1000F3CF15F0F4501626D9EC02F00001120085
:104A2000410E0601605D000112E2266A4E0E06018B
:104A30006025256ED8B0262A2E0E255C646FAA6AE2
:104A400064C6A9FF69EC02F05F6F000110D0266A0E
:104A50005E0E06016025256ED8B0262A410E255C23
:104A6000646FAA6A64C6A9FF69EC02F05F6F020E68
:104A700006015F5D000126E37BD806015F3100017E
:104A80000FE306018D51030DF3CF16F08C51030D8A
:104A9000F3CF15F0F4501626D9EC02F0000106D041
:104AA0008DC616F006018C51D8EC02F0000197D8A3
:104AB0008DC616F006018C51D8EC02F0D8905F3309
:104AC0000001D5D7D89006018C35156E8D35166E40
:104AD000D9EC02F000011200050E0501E06F110E85
:104AE000E16F200EE26F010EE36FE46B8A0EE56F5B
:104AF000000148EF50F0050E0501E06F110EE16F67
:104B0000200EE26F010EE36FE46B880EE56F00018B
:104B100048EF50F0050E0501E06F110EE16F200E19
:104B2000E26F010EE36FE46B890EE56F000148EF61
:104B300050F00601619F050E0501E06F110EE16F57
:104B4000220EE26F010EE36FE46F61C6E5F500012E
:104B500048EF50F0050E0501E06F110EE16FE26BBA
:104B6000010EE36FE46B62C6E5F5000148EF50F01B
:104B7000020E0501E06F340EE16F070EE26F0001D7
:104B800048EF50F0020E0501E06F340EE16F010EA8
:104B9000E26F000148EF50F0020E0501E06F340EA5
:104BA000E16F050EE26F000148EF50F0060E0501BF
:104BB000E06F310EE16F010EE26F300EE36FE46BD8
:104BC000E56BE66B000148EF50F0020E0501E06F67
:104BD000340EE16F030EE26F000148EF50F0020E59
:104BE0000501E06F340EE16F080EE26F000148EF3F
:104BF00050F0020E0501E06F340EE16F060EE26F19
:104C0000000148EF50F0020E0501E06F340EE16F35
:104C1000020EE26F000148EF50F0060E0501E06F52
:104C2000110EE16F200EE26F020EE36F0D0EE46FC6
:104C3000030EE56FE80EE66F000148EF50F0060E38
:104C40000501E06F110EE16F200EE26F020EE36FBF
:104C50000D0EE46FE56BE66B000148EF50F038C6CF
:104C600028F037C627F036C626F035C625F050C6E0
:104C700034F04FC633F070EC07F036C02CF035C07E
:104C80002BF034C02AF033C029F0660E366E356E34
:104C9000060E346E7F0E336E2CC03AF02BC039F006
:104CA0002AC038F029C037F0C7EC06F036C02CF027
:104CB00035C02BF034C02AF033C029F02952D8B4C3
:104CC0003F84D8A4290628C03AF027C039F026C06E
:104CD00038F025C037F02CC036F02BC035F02AC094
:104CE00034F029C033F0C7EC06F015EC07F00601EC
:104CF000696F34C06AF66AC65EF669C65DF6070E6D
:104D00000501E06F110EE16F200EE26F030EE36FFD
:104D10000A0EE46FE56B5EC6E6F55DC6E7F50001D9
:104D200048EF50F0070E0501E06F110EE16F200E05
:104D3000E26F030EE36F0A0EE46FE56BE66BE76B61
:104D4000000148EF50F0080E0501E06F130EE16F0F
:104D5000040EE26F150EE36F210EE46F200EE56F77
:104D6000080EE66F0B0EE76FE86B140ED7EC02F03F
:104D7000000168EF50F0B0DE100E0F01406FAA6A1C
:104D80003E0EA96E69EC02F00601476F69EC02F075
:104D9000486F69EC02F0496F69EC02F04A6FE80E67
:104DA00047253F6F030E4821406F000E4921416F98
:104DB000000E4A21426F000113EC5BF050DF640EDD
:104DC000D7EF02F0AA6A310EA96E69EC02F0060173
:104DD0003F6F69EC02F0406F69EC02F0416F69ECE3
:104DE00002F0426F000187DE13EC5BF09BDF640E84
:104DF000D7EF02F033D832D831D830D82FD82ED8C8
:104E00002DD82CD82BD803011A6B000104EE0CF01E
:104E100003011B51E926000EEA22EF500C6E2C0E06
:104E20000C5C000112E004EE0CF003011B51E926BA
:104E3000000EEA22EFCF0CF005EEADF01A510CC0D7
:104E4000EBFF1A2B1B2B0001E0D7F36A05EEADF048
:104E500003011A51F3CFEBFF0001120004EE0CF036
:104E600003011B51E926000EEA22EF500C6E2C0EB6
:104E70000C5CD8A4010E3C6E500E1B5D010ED8B028
:104E8000000E3C16000104E003011B2B0001E6D7D5
:104E900003011B2B000112000301179D00015BECB5
:104EA00046F0BCEC29F000EEE8F010EE58F0080EE9
:104EB000E75204E0E6CFEEFFE82EFAD7EF6A610E84
:104EC0004E6E030111510001E8A801D04E90BCECD8
:104ED00044F000EEE8F010EE4FF0080EE75204E068
:104EE000E6CFEEFFE82EFAD7EF6ABCEC44F04EB006
:104EF0003AD0030111510001E8A411D0600E4E6EAA
:104F000000EEE8F010EE61F0080EE75204E0E6CFA4
:104F1000EEFFE82EFAD7EF6ABCEC44F001D013D0D4
:104F2000030111510001E8A60ED000EEE8F010EEEA
:104F30006AF0080EE75204E0E6CFEEFFE82EFAD75B
:104F4000EF6ABCEC44F0610E4E6E00EEE8F010EE3D
:104F500073F0080EE75204E0E6CFEEFFE82EFAD732
:104F6000EF6ABCEC44F0030E4B6E59D9F00E4B6E59
:104F700056D10301376B366B2C6B780E2B6F630E9B
:104F80000301365D0001D8B0E8D02CC3AAFF2BC3C3
:104F9000A9FF69EC02F04B6E0D0E4B5CD8B4DDD06E
:104FA0005C0E4B5CD8A4D1D003012B2B000E2C231C
:104FB0001B6B2CC3AAFF2BC3A9FF69EC02F04B6E3D
:104FC0004B9A550E4B5C00010EE100EEE8F010EE3E
:104FD000A6F00A0EE75204E0E6CFEEFFE82EFAD77D
:104FE000EF6ABCD8B1D0560E4B5C0EE100EEE8F093
:104FF00010EEB1F00A0EE75204E0E6CFEEFFE82E25
:10500000FAD7EF6AABD8A0D0570E4B5C0EE100EE9A
:10501000E8F010EEBCF00A0EE75204E0E6CFEEFF37
:10502000E82EFAD7EF6A9AD88FD0580E4B5C0EE173
:1050300000EEE8F010EEC7F00A0EE75204E0E6CF0B
:10504000EEFFE82EFAD7EF6A89D87ED05A0E4B5C75
:1050500016E100EEE8F0020E016E086A1A6A0E0E02
:10506000196E69EC00F02E0EEE6E020E016E010E4E
:10507000086E8C0E67EC00F0EE6A70D865D0540EA6
:105080004B5C0EE100EEE8F010EE9BF00A0EE752EA
:1050900004E0E6CFEEFFE82EFAD7EF6A5FD854D0EF
:1050A000530E4B5C0EE100EEE8F010EE90F00A0EAD
:1050B000E75204E0E6CFEEFFE82EFAD7EF6A4ED8CB
:1050C00043D0490E4B5C0EE100EEE8F010EE8AF0A2
:1050D000050EE75204E0E6CFEEFFE82EFAD7EF6ABE
:1050E0003DD832D0500E4B5C0EE100EEE8F010EEF1
:1050F000D2F00A0EE75204E0E6CFEEFFE82EFAD730
:10510000EF6A2CD821D0460E4B5C0EE100EEE8F0A1
:1051100010EEDDF00A0EE75204E0E6CFEEFFE82ED7
:10512000FAD7EF6A1BD810D0420E4B5C0DE100EEAF
:10513000E8F010EE85F0040EE75204E0E6CFEEFF53
:10514000E82EFAD7EF6A0AD801D069D803012B2BD1
:10515000000E2C23362B000112D7120000EEE8F0CF
:1051600003011B51E926000EEA22EF500C6E000EDF
:105170000C52D8A4010E3C6E640E1B5D010ED8B01B
:10518000000E3C1600010EE000EEE8F003011B519A
:10519000E926000EEA22EF504B6E1B2B362B000146
:1051A0003ED8DCD71200FCEC46F076DE600E4B6E8B
:1051B00036D803011B6B000104EE0CF003011B51F8
:1051C000E926000EEA22EF500C6E0D0E0C5CD8A4FE
:1051D000010E3C6EC70E1B5D010ED8B0000E3C16D2
:1051E00000010FE004EE0CF003011B51E926000E54
:1051F000EA22EF504B6E000112D803011B2B000175
:10520000DAD7000E030111BD010E3C6E010E55539D
:10521000D8A4000E3C16000101E0ABDEC0D00301B3
:1052200011350001D8B092D0F29A486A080E485C55
:105230001FE20301188D4BA0189D00014CD84BB004
:1052400006D0476A03011689000114D80DD0030166
:105250001699472A00010ED8050E475C05E1476AFA
:1052600003011689000106D8D8904B32482ADEE3A4
:10527000F28A1200E86A030116BB010F16B9010A8F
:10528000D8B4169BD8A4168B030116510001E8BAB6
:1052900003D058C352FF02D059C352FF9EB219D057
:1052A000F76A57C3F6FF160EF626BA0EF722A66A5D
:1052B000A68E0800F5CF40FF7EA0FED70301572B36
:1052C0007E90170E575D000102E10301576B00014C
:1052D000E5D79E921200030118510001E8AC02D0FC
:1052E000010E4C1A0301188D4CA0189DD8904D3218
:1052F0004C3218510001E8BC01D01200080E4C1AC3
:10530000840E4D1A120003011135000101E3120051
:1053100003011A6B03011A511C5D000116E303011E
:1053200016890001A7DF486A060E485C06E2030101
:10533000169900019FDF482AF7E30301168900014F
:1053400099DF03011A2B0001E5E31200016A020E46
:10535000086E4B504FEC00F0200ED6EC01F003012C
:10536000532B100E535D000105E10301536B0D0E2D
:10537000D6EC01F00001120003011135000104E236
:10538000E2EC26F0B8EC25F05BEC46F04D684C689A
:1053900051C3BBFFBC6A9E9210C31CF3B4D7030178
:1053A0001135000104E30D0ED6EC01F011D0FF0E13
:1053B0004D180301526FFF0E4C184B6E00012FDF8A
:1053C00052C34BF02CDF54C31CF39DDF9EA2FED7CB
:1053D000C2EF25F00D0ED6EC01F0110EF76E200E87
:1053E000F66ECEEC01F0016A086A1A6A0E0E196EAA
:1053F00069EC00F02E0ED6EC01F0010E086E8C0E5A
:1054000067EC00F0110EF76E340EF66ECEEC01F084
:105410000D0ED6EC01F0130E096E880E026EAEEC86
:1054200001F0D8A038EF16F04A6E110EF76E3E0E5E
:10543000F66ECEEC01F00D0ED6EC01F0630ED6EC5C
:1054400001F06D0ED6EC01F0640ED6EC01F03E0ECC
:10545000D6EC01F004EE0CF00D0EEE6EEF6A03D800
:1054600082D8FBD8FCD73A0E096E980E026EAEECCD
:1054700001F0F9E34A6E030112510001E8A203D0E2
:105480004A50D6EC01F00D0E4A5C010ED8A4000E75
:105490003C6E0A0E4A5C010ED8A4000E3C1201E0DC
:1054A0001200010E496E4AC00CF43A0E096E980EB5
:1054B000026EAEEC01F0D8A045D04A6E0301125145
:1054C0000001E8A203D04A50D6EC01F0080E4A5C75
:1054D00004E1495201E04906E8D70D0E4A5C010E8D
:1054E000D8A4000E3C6E0A0E4A5C010ED8A4000E31
:1054F0003C124928010ED8A4000E3C1219E004EE1B
:105500000CF04950E926000EEA220D0EEF6E492AF2
:1055100004EE0CF04950E926000EEA22EF6A096A0F
:10552000960E026EAEEC01F001E34A6E120008D056
:1055300004EE0CF04950E926000EEA224AC0EFFFC3
:10554000492AB3D704EE0CF04950E926000EEA22AE
:105550000D0EEF6E492A04EE0CF04950E926000EBC
:10556000EA22EF6A120003011B6B000104EE0CF04B
:1055700003011B51E926000EEA22EF500C6E200EAB
:105580000C5CD8A4010E3C6E04EE0CF01B51E92615
:10559000000EEA22EF500C6E0D0E0C5CD8A4010E2A
:1055A0003C16FD0E1B5D010ED8B0000E3C1600012E
:1055B000D8B449D004EE0CF003011B51E926000ECB
:1055C000EA22EF500C6E610E0C5C000ED8B0010E9A
:1055D0003C6E04EE0CF01B51E926000EEA22EF505F
:1055E0000C6E7B0E0C5C000102E3000E01D0010E7C
:1055F0003C1614E004EE0CF003011B51E926000EEA
:10560000EA22EF500E6EDF0E0E140C6E04EE0CF05C
:105610001B51E926000EEA220CC0EFFF000104EE48
:105620000CF003011B51E926000EEA22EFCF0CF02B
:1056300000EEE8F01B51E926000EEA220CC0EFFF55
:105640001B2B000192D700EEE8F003011B51E92665
:10565000000EEA22EF6A00011200E8510C6E0A0EF9
:105660000C5C010ED8A4000E3C6EE8510C6E0D0EC1
:105670000C5C010ED8A4000E3C12E8510C6E010E19
:105680000C52D8A4000E3C1203E074CF1CF312009D
:10569000110EF76E520EF66E00EEE8F029EC04F0F3
:1056A00004E1CBEF30F077EF2EF0110EF76E580ECD
:1056B000F66E00EEE8F029EC04F009E0110EF76E4A
:1056C0005C0EF66E00EEE8F029EC04F004E196EFD3
:1056D00034F077EF2EF0110EF76E640EF66E00EEDA
:1056E000E8F029EC04F009E0110EF76E680EF66E92
:1056F00000EEE8F029EC04F004E13AEF34F077EF43
:105700002EF0110EF76E6E0EF66E00EEE8F029EC3C
:1057100004F009E0110EF76E720EF66E00EEE8F07E
:1057200029EC04F004E153EF34F077EF2EF0110E82
:10573000F76E7A0EF66E00EEE8F029EC04F009E060
:10574000110EF76E7E0EF66E00EEE8F029EC04F016
:1057500004E1E0EF34F077EF2EF0110EF76E860ED5
:10576000F66E00EEE8F029EC04F009E0110EF76E99
:105770008C0EF66E00EEE8F029EC04F004E11FEF69
:1057800036F077EF2EF0110EF76E940EF66E00EEF7
:10579000E8F029EC04F004E111EF41F077EF2EF08E
:1057A000110EF76E9A0EF66E00EEE8F029EC04F09A
:1057B00004E16DEF30F077EF2EF0110EF76EA20ED0
:1057C000F66E00EEE8F029EC04F004E124EF33F08B
:1057D00077EF2EF0110EF76EA80EF66E00EEE8F0E1
:1057E00029EC04F004E1C7EF32F077EF2EF0110E50
:1057F000F76EAE0EF66E00EEE8F029EC04F004E170
:10580000E1EF40F077EF2EF0110EF76EB60EF66E68
:1058100000EEE8F029EC04F009E0110EF76EBC0E82
:10582000F66E00EEE8F029EC04F004E193EF31F0BD
:1058300077EF2EF0110EF76EC40EF66E00EEE8F064
:1058400029EC04F009E0110EF76EC80EF66E00EEBA
:10585000E8F029EC04F003E1FAEF40F048D2110E31
:10586000F76ED00EF66E00EEE8F029EC04F009E0D9
:10587000110EF76ED40EF66E00EEE8F029EC04F08F
:1058800003E1A8EF3FF033D2110EF76EDC0EF66E97
:1058900000EEE8F029EC04F002E144D228D2110E27
:1058A000F76EE20EF66E00EEE8F029EC04F003E18C
:1058B000D4EF31F01CD2110EF76EE80EF66E00EE4A
:1058C000E8F029EC04F003E1EDEF31F010D2110E15
:1058D000F76EF00EF66E00EEE8F029EC04F009E049
:1058E000110EF76EF60EF66E00EEE8F029EC04F0FD
:1058F00003E16AEF32F0FBD1120EF76E000EF66E86
:1059000000EEE8F029EC04F009E0120EF76E040E48
:10591000F66E00EEE8F029EC04F003E193EF3BF0C3
:10592000E6D1120EF76E0E0EF66E00EEE8F029ECE0
:1059300004F003E163EF3CF0DAD1120EF76E140EBF
:10594000F66E00EEE8F029EC04F009E0120EF76EB6
:10595000180EF66E00EEE8F029EC04F003E151EFCA
:105960003EF0C5D1120EF76E220EF66E00EEE8F094
:1059700029EC04F009E0120EF76E280EF66E00EE28
:10598000E8F029EC04F003E180EF3EF0B0D1120E14
:10599000F76E2E0EF66E00EEE8F029EC04F003E14F
:1059A000AEEF3EF0A4D1120EF76E340EF66E00EE9E
:1059B000E8F029EC04F003E1D0EF3EF098D1120EAC
:1059C000F76E3A0EF66E00EEE8F029EC04F003E113
:1059D00051EF32F08CD1120EF76E400EF66E00EEE3
:1059E000E8F029EC04F003E106EF32F080D1120E6A
:1059F000F76E460EF66E00EEE8F029EC04F003E1D7
:105A00001FEF32F074D1120EF76E4E0EF66E00EEEE
:105A1000E8F029EC04F003E138EF32F068D1120E1F
:105A2000F76E560EF66E00EEE8F029EC04F009E091
:105A3000120EF76E5C0EF66E00EEE8F029EC04F044
:105A400003E136EF3FF053D1120EF76E620EF66EA1
:105A500000EEE8F029EC04F009E0120EF76E680E93
:105A6000F66E00EEE8F029EC04F003E103EF3FF0FE
:105A70003ED1110EF76E520EF66E00EEE8F029ECF4
:105A800004F003E1CBEF30F032D1120EF76E6E0E60
:105A9000F66E00EEE8F029EC04F009E0120EF76E65
:105AA000740EF66E00EEE8F029EC04F003E1E4EF8A
:105AB00030F01DD1120EF76E7E0EF66E00EEE8F09D
:105AC00029EC04F003E1FDEF30F011D1120EF76E76
:105AD000840EF66E00EEE8F029EC04F003E116EF18
:105AE00031F005D1120EF76E8A0EF66E00EEE8F078
:105AF00029EC04F003E12FEF31F0F9D0120EF76E2C
:105B0000900EF66E00EEE8F029EC04F009E0120EBB
:105B1000F76E940EF66E00EEE8F029EC04F003E167
:105B20007AEF31F0E4D0120EF76E9A0EF66E00EEB8
:105B3000E8F029EC04F003E148EF31F0D8D0120E80
:105B4000F76EA20EF66E00EEE8F029EC04F003E129
:105B500061EF31F0CCD0120EF76EA80EF66E00EEAB
:105B6000E8F029EC04F003E133EF3DF0C0D0110E72
:105B7000F76E940EF66E00EEE8F029EC04F003E107
:105B800011EF41F0B4D0120EF76EAC0EF66E00EECF
:105B9000E8F029EC04F003E1D9EF3FF0A8D0120EB1
:105BA000F76EB20EF66E00EEE8F029EC04F002E1BA
:105BB000D2D09DD0120EF76EB80EF66E00EEE8F061
:105BC00029EC04F003E19CEF32F091D0120EF76E55
:105BD000BE0EF66E00EEE8F029EC04F003E171EF82
:105BE00033F085D0120EF76EC80EF66E00EEE8F0B8
:105BF00029EC04F003E116EF40F079D0120EF76EB5
:105C0000CE0EF66E00EEE8F029EC04F003E1A1EF11
:105C100031F06DD0120EF76ED20EF66E00EEE8F097
:105C200029EC04F003E1BBEF31F061D0110EF76E07
:105C3000D00EF66E00EEE8F029EC04F003E1A8EFD8
:105C40003FF055D0120EF76ED80EF66E00EEE8F06B
:105C500029EC04F002E1B1D04AD0120EF76EDE0E4C
:105C6000F66E00EEE8F029EC04F002E18DD03FD0B2
:105C7000120EF76EE40EF66E00EEE8F029EC04F07A
:105C800003E103EF3EF033D0120EF76EEC0EF66E2A
:105C900000EEE8F029EC04F009E0120EF76EF00EC9
:105CA000F66E00EEE8F029EC04F002E1B8D01FD067
:105CB000120EF76EFA0EF66E00EEE8F029EC04F024
:105CC00009E0130EF76E000EF66E00EEE8F029EC18
:105CD00004F002E18BD00BD0130EF76E040EF66EBB
:105CE00000EEE8F029EC04F002E1C5EF3FF0130EFE
:105CF000F76E0A0EF66ECEEC01F00D0ED6EC01F04A
:105D0000630ED6EC01F06D0ED6EC01F0640ED6EC0D
:105D100001F03E0ED6EC01F0640ED7EC02F074CF29
:105D20001CF3120068EC46F0030118310001D8B0F2
:105D3000BAEF45F00301D89216B5D882D8B21281D5
:105D4000D8A21291AA6A240EA96E125159EC02F03F
:105D50000001E0EF45F068EC46F003011831000166
:105D6000D8B0BAEF45F00301D89216B5D882D8B2B0
:105D70001285D8A21295AA6A240EA96E125159EC66
:105D800002F00001E0EF45F068EC46F00301183145
:105D90000001D8B0BAEF45F00301D89216B5D88209
:105DA000D8B2128FD8A2129FAA6A240EA96E1251DD
:105DB00059EC02F00001E0EF45F068EC46F0030119
:105DC00018310001D8B0BAEF45F00301D89216B5EA
:105DD000D882D8B2148BD8A2149BAA6A260EA96EB8
:105DE000145159EC02F00001E0EF45F068EC46F088
:105DF000030118310001D8B0BAEF45F00301D89281
:105E000016B5D882D8B2148FD8A2149FAA6A260ECB
:105E1000A96E145159EC02F00001E0EF45F068EC76
:105E200046F0030118310001D8B0BAEF45F0030184
:105E3000D89216B5D882D8B2148DD8A2149DAA6A69
:105E4000260EA96E145159EC02F014510001E8AC71
:105E500042D1130EF76E200EF66ECEEC01F00D0E51
:105E6000D6EC01F0130EF76E580EF66ECEEC01F084
:105E70000D0ED6EC01F0130EF76EA40EF66ECEECFE
:105E800001F00D0ED6EC01F0130EF76ECA0EF66E91
:105E9000CEEC01F00601B051D6EC01F0200ED6ECAC
:105EA00001F03A0E096E980E026EAEEC01F00001A0
:105EB00023E303011C6F300E1C5D000ED8B0010EF1
:105EC0003C6E3A0E1C5D000102E3000E01D0010E93
:105ED0003C1612E01CC3B0F6AA6A480EA96E030174
:105EE0001C5159EC02F012510001E8A204D0030148
:105EF0001C51D6EC01F000010D0ED6EC01F0130E92
:105F0000F76ED20EF66ECEEC01F00601B151D6EC72
:105F100001F0200ED6EC01F03A0E096E980E026EDA
:105F2000AEEC01F0000123E303011C6F300E1C5D99
:105F3000000ED8B0010E3C6E3A0E1C5D000102E36B
:105F4000000E01D0010E3C1612E01CC3B1F6AA6A85
:105F5000490EA96E03011C5159EC02F012510001C7
:105F6000E8A204D003011C51D6EC01F000010D0E93
:105F7000D6EC01F0130EF76EDA0EF66ECEEC01F0F1
:105F80000601B251D6EC01F0200ED6EC01F03A0E2B
:105F9000096E980E026EAEEC01F0000123E30301DE
:105FA0001C6F300E1C5D000ED8B0010E3C6E3A0E18
:105FB0001C5D000102E3000E01D0010E3C1612E050
:105FC0001CC3B2F6AA6A4A0EA96E03011C5159EC11
:105FD00002F012510001E8A204D003011C51D6ECDA
:105FE00001F000010D0ED6EC01F0130EF76EE20E7B
:105FF000F66ECEEC01F00601B351D6EC01F0200EA6
:10600000D6EC01F03A0E096E980E026EAEEC01F07D
:10601000000123E303011C6F300E1C5D000ED8B09D
:10602000010E3C6E3A0E1C5D000102E3000E01D031
:10603000010E3C1612E01CC3B3F6AA6A4B0EA96E01
:1060400003011C5159EC02F012510001E8A204D0E6
:1060500003011C51D6EC01F000010D0ED6EC01F04D
:10606000130EF76EEA0EF66ECEEC01F00601B45197
:10607000D6EC01F0200ED6EC01F03A0E096E980E27
:10608000026EAEEC01F0000123E303011C6F300E41
:106090001C5D000ED8B0010E3C6E3A0E1C5D000176
:1060A00002E3000E01D0010E3C1612E01CC3B4F650
:1060B000AA6A4C0EA96E03011C5159EC02F0125150
:1060C0000001E8A204D003011C51D6EC01F000014C
:1060D0000D0ED6EC01F0E0EF45F0FEEC45F00601C8
:1060E0006551300A66116711681100010FE0060161
:1060F0006751681100010FE106016551C00A0001F6
:106100000AE106016651120A000105E1BC0E060112
:106110009B6F000136D006016551600A6611671158
:10612000681100010FE006016751681100010FE1DD
:1061300006016551800A00010AE106016651250A3F
:10614000000105E1550E06019B6F00011AD0060102
:106150006551C00A66116711681100010BE0060164
:1061600065516711681100010AE1060166514B0A89
:10617000000105E11E0E06019B6F000102D0BAEF7F
:1061800045F0AA6A3C0EA96E06019B5159EC02F03B
:106190000001E0EF45F068EC46F003011831000122
:1061A000D8B0BAEF45F00301D89216B5D882D8B26C
:1061B0001283D8A21293AA6A240EA96E125159EC26
:1061C00002F00001E0EF45F068EC46F00301183101
:1061D0000001D8B0BAEF45F00301D89216B5D882C5
:1061E000D8B21287D8A21297AA6A240EA96E1251A9
:1061F00059EC02F00001E0EF45F068EC46F00301D5
:1062000018310001D8B0BAEF45F00301D89216B5A5
:10621000D882D8B2138DD8A2139DAA6A250EA96E72
:10622000135159EC02F00001E0EF45F068EC46F044
:10623000030118310001D8B0BAEF45F00301D8923C
:1062400016B5D882D8B2138FD8A2139FAA6A250E8A
:10625000A96E135159EC02F00001E0EF45F068EC33
:1062600046F0030118310001D8B0BAEF45F0030140
:10627000D89216B5D882D8B21481D8A21491AA6A3D
:10628000260EA96E145159EC02F00001E0EF45F022
:1062900068EC46F0030118310001D8B0BAEF45F0C0
:1062A0000301D89216B5D882D8B21483D8A2149319
:1062B000AA6A260EA96E145159EC02F00001E0EF13
:1062C00045F068EC46F0030118310001D8B0BAEF90
:1062D00045F00301D89216B5D882D8B21489D8A255
:1062E0001499AA6A260EA96E145159EC02F0000105
:1062F000E0EF45F068EC46F0030118310001D8B03A
:10630000BAEF45F00301D89216B5D882D8B21487F7
:10631000D8A21497AA6A260EA96E145159EC02F05D
:106320000001E0EF45F0FEEC45F065C656F3AA6AC1
:106330002D0EA96E0301565159EC02F00001E0EF59
:1063400045F068EC46F0030118310001D8B0BAEF0F
:1063500045F0E86A030116B5010E010AD8B4129D92
:10636000D8A4128DAA6A240EA96E125159EC02F01B
:106370000001E0EF45F068EC46F003011831000140
:10638000D8B0BAEF45F00301D89216B5D882D8B28A
:106390001289D8A21299AA6A240EA96E125159EC38
:1063A00002F00001E0EF45F068EC46F0030118311F
:1063B0000001D8B0BAEF45F00301D89216B5D882E3
:1063C000D8B21381D8A21391AA6A250EA96E1351CF
:1063D00059EC02F00001E0EF45F068EC46F00301F3
:1063E00018310001D8B0BAEF45F00301D89216B5C4
:1063F000D882D8B21383D8A21393AA6A250EA96EA5
:10640000135159EC02F00001E0EF45F068EC46F062
:10641000030118310001D8B0BAEF45F00301D8925A
:1064200016B5D882D8B21387D8A21397AA6A250EB8
:10643000A96E135159EC02F00001E0EF45F068EC51
:1064400046F0030118310001D8B0BAEF45F003015E
:10645000D89216B5D882D8B21389D8A21399AA6A4D
:10646000250EA96E135159EC02F00001E0EF45F042
:1064700068EC46F0030118310001D8B0BAEF45F0DE
:106480000301D89216B5D882D8B2138BD8A2139B29
:10649000AA6A250EA96E135159EC02F00001E0EF33
:1064A00045F068EC46F0030118310001D8B0BAEFAE
:1064B00045F00301D89216B5D882D8B21385D8A278
:1064C0001395AA6A250EA96E135159EC02F000012A
:1064D000E0EF45F068EC46F0030118310001D8B058
:1064E000BAEF45F00301D89216B5D882D8B2128B14
:1064F000D8A2129BAA6A240EA96E125159EC02F07E
:106500000001E0EF45F068EC46F0030118310001AE
:10651000D8B0BAEF45F00301D89216B5D882D8B2F8
:106520001485D8A21495AA6A260EA96E145159ECA6
:1065300002F00001E0EF45F065EC45F004010C517C
:106540000C6E310E0C5C0001D8B4CAEF53F004019C
:106550000C510C6E320E0C5C0001D8B4A7EF54F055
:1065600004010C510C6E330E0C5C0001D8B49CEF8E
:1065700055F004010C510C6E340E0C5C000105E169
:106580000601B9890001E0EF45F0BAEF45F065EC8E
:1065900045F0B3EC2AF004010C510C6E450E0C5C76
:1065A00000011AE165EC45F004010C510C6E0F0E70
:1065B0000C140301556FAA6A2B0EA96E555159ECA4
:1065C00002F05553000104E10301119D000102D0C6
:1065D0000301118D00012ED004010C510C6E4F0EE1
:1065E0000C5C000125E104010D510C6E460E0C5CA3
:1065F000000104E10301119D000119D004010D51B6
:106600000C6E4E0E0C5C000110E10301118DAA6AA4
:106610002B0EA96E69EC02F0556F5553000103E192
:10662000050E0301556F000102D0BAEF45F002D00C
:10663000BAEF45F0AA6A230EA96E0301115159EC75
:1066400002F00001E0EF45F0040111510C6E0D0E57
:106650000C5C000101E1120065EC45F004010C51F5
:106660000C6E0D0E0C5C00010CE1AA6A780EA96E8E
:106670000D0E59EC02F00301119B119D17950001BD
:1066800025D003011A6B640E03011A5D00011AE2A2
:1066900004EE0CF003011A51E926000EEA22EF5035
:1066A0001C6FAA6A780E1A25A96ED8B0AA2A1C51A6
:1066B00059EC02F00D0E1C5D000104E003011A2BE1
:1066C0000001E1E30301118B118D17850001AA6A16
:1066D000230EA96E0301115159EC02F00001E0EF05
:1066E00045F00D0ED6EC01F0130EF76EF20EF66EBD
:1066F000CEEC01F00D0ED6EC01F0140EF76E000E8C
:10670000F66ECEEC01F00D0ED6EC01F0140EF76E25
:10671000240EF66ECEEC01F00D0ED6EC01F0030E59
:10672000166EE80ED8EC02F0B8EC25F00301576BBA
:106730009E9A000158C352FF9EBA1CD0170E030147
:10674000575D000113E2F76A57C3F6FF160EF626EF
:10675000BA0EF722A66AA68E0800F5CF40FF7EA0EB
:10676000FED77E900301572B0001E8D70301576B3A
:106770000001E2D7DF0EAE1403011C6F440E1C5D56
:10678000000109E1FF0E0301585D000102E203016F
:10679000582B0001CED7550E03011C5D000109E105
:1067A000650E0301585D000102E303015807000173
:1067B000C0D7450E03011C5D0001D8B456D0530E5E
:1067C00003011C5D0001D8A4B4D7AA6A2F0EA96EDC
:1067D0000301585159EC02F058510C0DF3CF23F33B
:1067E000F4CF24F33A6A396A300E386E830E376E6E
:1067F00024C334F023C333F078EC07F061EC06F0E7
:1068000036C022F335C021F334C020F333C01FF368
:1068100022C336F021C335F020C334F01FC333F058
:10682000C7EC05F0596FAA6A300EA96E595159ECA0
:1068300002F05851170DF3CF23F3F4CF24F33A6A43
:10684000396A386A840E376E24C334F023C333F0B8
:1068500078EC07F061EC06F0C7EC05F0516FAA6A1E
:106860002C0EA96E515159EC02F00001C2EC25F03A
:10687000E0EF45F068EC46F0030118310001D8B0B4
:10688000BAEF45F00301D89216B5D882D8B2118F6D
:10689000D8A2119FAA6A230EA96E115159EC02F0D9
:1068A0000001E0EF45F0FEEC45F00601665167118E
:1068B000681104E1650E655D000106E30601686B81
:1068C000676B666B640E656F000168C614F067C67F
:1068D00013F066C612F065C611F01C6A1B6A010E41
:1068E0001A6E800E196E9EEC03F014C028F013C0CF
:1068F00027F012C026F011C025F0800E25240601D5
:10690000656F000E2620666F000E2720676F000E51
:106910002820686F66C610F3AA6A270EA96E0301C5
:10692000105159EC02F00001E0EF45F065EC45F044
:10693000030116510001E8A60AD000EEE8F0EE6A65
:10694000EE6AEE6AEE6AEE6AEE6AEE6A02D098ECE1
:1069500043F003011A6B070E03011A5D00011EE2EA
:1069600000EEE8F003011A51E926000EEA22EFCF0B
:106970000CF000EE4FF01A510CC0EBFFAA6A1AC3DC
:10698000A9FF00EEE8F01A51E926000EEA22EF50C6
:1069900059EC02F003011A2B0001DDE3E86A030160
:1069A00016B7010E010AD8B41191D8A41181AA6AB0
:1069B000230EA96E115159EC02F00001E0EF45F0F1
:1069C00003011193119511971199000165EC45F0A0
:1069D000030116510001E8A60BD000EEE8F0EE6AC4
:1069E000EE6AEE6AEE6AEE6AEE6AEE6AEE6A02D06D
:1069F00098EC43F0030116510001E8B6BAEF45F0F8
:106A000003011A6B070E03011A5D000121E200EE7B
:106A1000E8F003011A51E926000EEA22EFCF0CF04C
:106A200000EE58F01A510CC0EBFFAA6A070E1A25A7
:106A3000A96ED8B0AA2A00EEE8F01A51E926000E95
:106A4000EA22EF5059EC02F003011A2B0001DAE3BD
:106A50005F6A0301118316310001D8B0D1D098ECE0
:106A600043F0030116510001E8B6BAEF45F0030107
:106A70001631000135E203011A6B070E03011A5D9E
:106A8000000121E200EEE8F003011A51E926000EB0
:106A9000EA22EFCF0CF000EE61F01A510CC0EBFFD0
:106AA000AA6A0E0E1A25A96ED8B0AA2A00EEE8F03E
:106AB0001A51E926000EEA22EF5059EC02F00301C8
:106AC0001A2B0001DAE3686B03011185000198ECD1
:106AD00043F0030116510001E8B6BAEF45F015D0B6
:106AE00003011A6B070E03011A5D00010EE2AA6A88
:106AF0000E0E03011A25A96ED8B0AA2A000E59EC71
:106B000002F003011A2B0001EDE30301163100012D
:106B100035E203011A6B070E03011A5D000121E241
:106B200000EEE8F003011A51E926000EEA22EFCF49
:106B30000CF000EE6AF01A510CC0EBFFAA6A150EB9
:106B40001A25A96ED8B0AA2A00EEE8F01A51E92653
:106B5000000EEA22EF5059EC02F003011A2B00015B
:106B6000DAE3716B03011187000198EC43F0030134
:106B700016510001E8B6BAEF45F015D003011A6BC3
:106B8000070E03011A5D00010EE2AA6A150E030149
:106B90001A25A96ED8B0AA2A000E59EC02F00301FA
:106BA0001A2B0001EDE303011A6B070E03011A5DB6
:106BB000000121E200EEE8F003011A51E926000E7F
:106BC000EA22EFCF0CF000EE73F01A510CC0EBFF8D
:106BD000AA6A1C0E1A25A96ED8B0AA2A00EEE8F0FF
:106BE0001A51E926000EEA22EF5059EC02F0030197
:106BF0001A2B0001DAE37A6B03011189000115D029
:106C000003011A6B070E03011A5D00010EE2AA6A66
:106C10001C0E03011A25A96ED8B0AA2A000E59EC41
:106C200002F003011A2B0001EDE3AA6A230EA96EFC
:106C30000301115159EC02F00001E0EF45F00D0E97
:106C4000D6EC01F0140EF76E4A0EF66ECEEC01F0A3
:106C50000301113100010EE300EEE8F010EE4FF0F9
:106C6000080EE75204E0E6CFEEFFE82EFAD7EF6A0F
:106C7000DCEC44F0AA6A310EA96E69EC02F0060160
:106C80003F6F69EC02F0406F69EC02F0416F69EC14
:106C900002F0426F0D0ED6EC01F0140EF76E520E9C
:106CA000F66ECEEC01F0016A9A5166EC00F0200E0F
:106CB000D6EC01F06D0ED6EC01F0570ED6EC01F0DB
:106CC0000D0ED6EC01F0140EF76E5E0EF66ECEECE5
:106CD00001F0016A086A46C628F045C627F044C696
:106CE00026F043C625F000EC01F0200ED6EC01F0B2
:106CF000480ED6EC01F07A0ED6EC01F00D0ED6EC73
:106D000001F0140EF76E700EF66ECEEC01F0016A13
:106D1000086A4AC628F049C627F048C626F047C682
:106D200025F000EC01F0200ED6EC01F0480ED6EC78
:106D300001F07A0ED6EC01F00D0ED6EC01F0140E37
:106D4000F76E860EF66ECEEC01F0016A086A42C656
:106D500028F041C627F040C626F03FC625F000ECDB
:106D600001F0200ED6EC01F0480ED6EC01F07A0EC0
:106D7000D6EC01F00D0ED6EC01F0140EF76E980E65
:106D8000F66ECEEC01F0030112350001D8A0E6D07A
:106D90004F0ED6EC01F04E0ED6EC01F00D0ED6ECF7
:106DA00001F0140EF76EA00EF66ECEEC01F0016A43
:106DB000086A50C61AF04FC619F069EC00F0200EB0
:106DC000D6EC01F0480ED6EC01F07A0ED6EC01F0CC
:106DD0000D0ED6EC01F0140EF76EAC0EF66ECEEC86
:106DE00001F0016A086A52C61AF051C619F069EC3E
:106DF00000F0200ED6EC01F0420ED6EC01F0640E4D
:106E0000D6EC01F00D0ED6EC01F0140EF76EB40EB8
:106E1000F66ECEEC01F0016A0601535166EC00F00B
:106E20000D0ED6EC01F0140EF76EC00EF66ECEEC21
:106E300001F0016A545166EC00F00D0ED6EC01F041
:106E4000140EF76ECC0EF66ECEEC01F0030113516A
:106E50000001E8A407D04F0ED6EC01F04E0ED6ECA0
:106E600001F008D04F0ED6EC01F0460ED6EC01F042
:106E7000D6EC01F00D0ED6EC01F0140EF76EDA0E22
:106E8000F66ECEEC01F003011431000107E34F0E62
:106E9000D6EC01F04E0ED6EC01F008D04F0ED6EC39
:106EA00001F0460ED6EC01F0D6EC01F00D0ED6EC5A
:106EB00001F0140EF76EEA0EF66ECEEC01F003014F
:106EC00013510001E8A607D04F0ED6EC01F04E0E8C
:106ED000D6EC01F008D04F0ED6EC01F0460ED6EC01
:106EE00001F0D6EC01F00D0ED6EC01F0140EF76EA9
:106EF000F80EF66ECEEC01F0030113510001E8A884
:106F000007D04F0ED6EC01F04E0ED6EC01F008D0B3
:106F10004F0ED6EC01F0460ED6EC01F0D6EC01F0A7
:106F20000D0ED6EC01F0150EF76E0E0EF66ECEECD1
:106F300001F0030113510001E8AA07D04F0ED6EC6F
:106F400001F04E0ED6EC01F008D04F0ED6EC01F059
:106F5000460ED6EC01F0D6EC01F008D04F0ED6EC80
:106F600001F0460ED6EC01F0D6EC01F00D0ED6EC99
:106F700001F0150EF76E240EF66ECEEC01F0030153
:106F80001231000109E24F0ED6EC01F0460ED6ECAC
:106F900001F0D6EC01F076D04F0ED6EC01F04E0E9B
:106FA000D6EC01F00D0ED6EC01F0150EF76E2C0E9E
:106FB000F66ECEEC01F0016A0601965166EC00F027
:106FC000200ED6EC01F0570ED6EC01F0500ED6ECA8
:106FD00001F04D0ED6EC01F00D0ED6EC01F0150EC1
:106FE000F76E340EF66ECEEC01F003011451000181
:106FF000E8A607D04F0ED6EC01F04E0ED6EC01F00D
:1070000008D04F0ED6EC01F0460ED6EC01F0D6ECCF
:1070100001F00D0ED6EC01F0150EF76E3C0EF66E7B
:10702000CEEC01F003011331000107E34F0ED6EC63
:1070300001F04E0ED6EC01F008D04F0ED6EC01F068
:10704000460ED6EC01F0D6EC01F00D0ED6EC01F0B8
:10705000150EF76E440EF66ECEEC01F003011351DF
:107060000001E8A207D04F0ED6EC01F04E0ED6EC90
:1070700001F008D04F0ED6EC01F0460ED6EC01F030
:10708000D6EC01F00D0ED6EC01F0150EF76E4E0E9B
:10709000F66ECEEC01F0030114510001E8A207D016
:1070A0004F0ED6EC01F04E0ED6EC01F008D04F0E8C
:1070B000D6EC01F0460ED6EC01F0D6EC01F00D0E48
:1070C000D6EC01F0150EF76E580EF66ECEEC01F010
:1070D000030114510001E8A807D04F0ED6EC01F0CF
:1070E0004E0ED6EC01F008D04F0ED6EC01F0460E55
:1070F000D6EC01F0D6EC01F00D0ED6EC01F0150E39
:10710000F76E600EF66ECEEC01F003011451000133
:10711000E8AA3CD14F0ED6EC01F04E0ED6EC01F0B1
:107120000D0ED6EC01F0150EF76E680EF66ECEEC75
:1071300001F0030111510001E8A274D000EEE8F063
:1071400010EE58F0080EE75204E0E6CFEEFFE82E0E
:10715000FAD7EF6ADCEC44F0030111510001E8A416
:107160001DD0200ED6EC01F0560ED6EC01F0690EC3
:10717000D6EC01F0610ED6EC01F0200ED6EC01F059
:1071800000EEE8F010EE61F0080EE75204E0E6CF02
:10719000EEFFE82EFAD7EF6ADCEC44F00301115160
:1071A0000001E8A61DD0200ED6EC01F0560ED6EC5C
:1071B00001F0690ED6EC01F0610ED6EC01F0200E64
:1071C000D6EC01F000EEE8F010EE6AF0080EE7529F
:1071D00004E0E6CFEEFFE82EFAD7EF6ADCEC44F0ED
:1071E000030111510001E8A81DD0200ED6EC01F0DA
:1071F000560ED6EC01F0690ED6EC01F0610ED6EC1D
:1072000001F0200ED6EC01F000EEE8F010EE73F085
:10721000080EE75204E0E6CFEEFFE82EFAD7EF6A59
:10722000DCEC44F003011051AB0DF3CF23F3F4CFAA
:1072300024F30D0ED6EC01F0150EF76E720EF66EFD
:10724000CEEC01F0016A245166EC00F00D0ED6EC94
:1072500001F0150EF76E7C0EF66ECEEC01F0016AB1
:10726000545166EC00F00D0ED6EC01F0150EF76EE1
:10727000860EF66ECEEC01F04F51D6EC01F0505177
:10728000D6EC01F0AA6A2D0EA96E69EC02F0566FD9
:107290000D0ED6EC01F0150EF76E900EF66ECEECDC
:1072A00001F0113500010DE3580ED6EC01F04D0E42
:1072B000D6EC01F0490ED6EC01F0540ED6EC01F0FC
:1072C00008D04F0ED6EC01F0460ED6EC01F0D6EC0D
:1072D00001F00D0ED6EC01F0150EF76E980EF66E5D
:1072E000CEEC01F0AA6A2B0EA96E69EC02F0030144
:1072F000556F11510001E8AC0DD0150EF76EA00EC0
:10730000F66ECEEC01F0016A0301555166EC00F017
:10731000000108D04F0ED6EC01F0460ED6EC01F07D
:10732000D6EC01F00D0ED6EC01F0150EF76EA80E9E
:10733000F66ECEEC01F0030111510001E8AA22D053
:107340000301246B780E236F366B640E0301365DE8
:10735000000117E224C3AAFF23C3A9FF69EC02F0CE
:1073600003011C6F1C51D6EC01F00D0E1C5D0001D9
:1073700008E00301232B000E24230301362B000118
:10738000E4E303D00D0ED6EC01F00BD04F0ED6EC9B
:1073900001F0460ED6EC01F0D6EC01F00D0ED6EC65
:1073A00001F0AA6A2D0EA96E69EC02F00301566F76
:1073B000150EF76EB00EF66ECEEC01F056530001CE
:1073C00007E1150EF76EBA0EF66ECEEC01F005D0A1
:1073D000016A0301565166EC00F000010D0ED6EC77
:1073E00001F0150EF76ED20EF66ECEEC01F0030131
:1073F00012510001E8A207D04F0ED6EC01F04E0E5C
:10740000D6EC01F008D04F0ED6EC01F0460ED6ECCB
:1074100001F0D6EC01F00D0ED6EC01F0150EF76E72
:10742000DA0EF66ECEEC01F0030112510001E8A66F
:1074300040D04F0ED6EC01F04E0ED6EC01F00D0E02
:10744000D6EC01F0150EF76EE20EF66ECEEC01F002
:10745000030113510001E8AC07D04F0ED6EC01F048
:107460004E0ED6EC01F008D04F0ED6EC01F0460ED1
:10747000D6EC01F0D6EC01F00D0ED6EC01F0150EB5
:10748000F76EF20EF66ECEEC01F00301133500013B
:1074900007E34F0ED6EC01F04E0ED6EC01F008D00B
:1074A0004F0ED6EC01F0460ED6EC01F0D6EC01F012
:1074B00008D04F0ED6EC01F0460ED6EC01F0D6EC1B
:1074C00001F00D0ED6EC01F0470ED6EC01F0500E97
:1074D000D6EC01F0530ED6EC01F03A0ED6EC01F0EA
:1074E000200ED6EC01F0030112510001E8AC09D0E6
:1074F0004F0ED6EC01F0460ED6EC01F0D6EC01F0C2
:107500001BD0030112510001E8A810D0550ED6EC93
:1075100001F0420ED6EC01F04C0ED6EC01F04F0E0D
:10752000D6EC01F0580ED6EC01F006D0160EF76E30
:10753000020EF66ECEEC01F00D0ED6EC01F0160E3A
:10754000F76E0A0EF66ECEEC01F003011251000147
:10755000E8AA07D04F0ED6EC01F04E0ED6EC01F0A3
:1075600008D04F0ED6EC01F0460ED6EC01F0D6EC6A
:1075700001F00D0ED6EC01F0160EF76E160EF66E3B
:10758000CEEC01F0030112510001E8A407D04F0E28
:10759000D6EC01F04E0ED6EC01F008D04F0ED6EC32
:1075A00001F0460ED6EC01F0D6EC01F0AA6A3C0ED2
:1075B000A96E69EC02F006019B6F0D0ED6EC01F08E
:1075C000160EF76E1E0EF66ECEEC01F0A10E9B5D50
:1075D000000106E3160EF76E280EF66ECEEC01F0F3
:1075E0004B0E06019B5D000102E2000E01D0010E70
:1075F0003C6E640E06019B5D010ED8B0000E3C1679
:10760000000106E0160EF76E300EF66ECEEC01F0BD
:107610002A0E06019B5D000106E2160EF76E380E7B
:10762000F66ECEEC01F00D0ED6EC01F0160EF76EF4
:10763000420EF66ECEEC01F0030114510001E8ACED
:1076400065D04F0ED6EC01F04E0ED6EC01F00D0ECB
:10765000D6EC01F0160EF76E4E0EF66ECEEC01F083
:1076600003011435000107E2160EF76E600EF66E88
:10767000CEEC01F009D0520ED6EC01F0410ED6EC62
:1076800001F0570ED6EC01F00D0ED6EC01F0430ED2
:10769000D6EC01F0680ED6EC01F0310ED6EC01F01C
:1076A0003A0ED6EC01F0200ED6EC01F0B0C6AFF6E3
:1076B0003BEC67F0160EF76E680EF66ECEEC01F03E
:1076C000B1C6AFF63BEC67F0160EF76E700EF66EB5
:1076D000CEEC01F0B2C6AFF63BEC67F0160EF76EDB
:1076E000780EF66ECEEC01F0B3C6AFF63BEC67F069
:1076F000160EF76E800EF66ECEEC01F0B4C6AFF645
:107700003BEC67F00D0ED6EC01F00BD04F0ED6EC33
:1077100001F0460ED6EC01F0D6EC01F00D0ED6ECE1
:1077200001F0E0EF45F0FEEC45F068C642F667C6B2
:1077300041F666C640F665C63FF6C00E06013F5DDF
:10774000CB0E4059170E4159070E42590001D8B0CF
:107750007AD003011A6B150E03011A5D000111E2C4
:1077600004EE0CF003011A51E926000EEA22EF5054
:107770000C6E0D0E0C5C000104E003011A2B0001DD
:10778000EAE3090E03011A5D00010CE204EE0CF0BD
:1077900003011A51E926000EEA22300EEF6E1A2B71
:1077A0000001EFD70D0E0401156F0601426B416B0E
:1077B000406B3F6B03011A6B090E03011A5D000158
:1077C000D8B041D0286A276A266A0A0E256E28C0DA
:1077D00014F027C013F026C012F025C011F042C6E5
:1077E0001CF041C61BF040C61AF03FC619F09EECD3
:1077F00003F014C028F013C027F012C026F011C007
:1078000025F004EE0CF003011A51E926000EEA22DD
:10781000EF500C6E2C6A2B6A2A6A0CC029F00F0EEE
:1078200029162950252406013F6F2A502620406F33
:107830002B502720416F2C502820426F03011A2B18
:107840000001D8A0B9D7070E0601425D000114E37C
:1078500011E1170E0601415D00010EE30BE1CB0EB5
:107860000601405D000108E305E1C00E06013F5D31
:10787000000102E3000E01D0010E3C6E810E0601F4
:107880003F5DD90E40599F0E4159380E42590001B3
:1078900002E2000E01D0010E3C1202E0BAEF45F008
:1078A000AA6A310EA96E06013F5159EC02F040510F
:1078B00059EC02F0415159EC02F0425159EC02F0FE
:1078C0000001E0EF45F0FEEC45F068C64AF667C6F9
:1078D00049F666C648F665C647F6C00E0601475D1E
:1078E000CB0E4859170E4959070E4A590001D8B016
:1078F0007AD003011A6B150E03011A5D000111E223
:1079000004EE0CF003011A51E926000EEA22EF50B2
:107910000C6E0D0E0C5C000104E003011A2B00013B
:10792000EAE3090E03011A5D00010CE204EE0CF01B
:1079300003011A51E926000EEA22300EEF6E1A2BCF
:107940000001EFD70D0E0401156F06014A6B496B5C
:10795000486B476B03011A6B090E03011A5D0001A6
:10796000D8B041D0286A276A266A0A0E256E28C038
:1079700014F027C013F026C012F025C011F04AC63B
:107980001CF049C61BF048C61AF047C619F09EEC19
:1079900003F014C028F013C027F012C026F011C065
:1079A00025F004EE0CF003011A51E926000EEA223C
:1079B000EF500C6E2C6A2B6A2A6A0CC029F00F0E4D
:1079C0002916295025240601476F2A502620486F82
:1079D0002B502720496F2C5028204A6F03011A2B67
:1079E0000001D8A0B9D7070E06014A5D000114E3D3
:1079F00011E1170E0601495D00010EE30BE1CB0E0C
:107A00000601485D000108E305E1C00E0601475D7F
:107A1000000102E3000E01D0010E3C6E810E060152
:107A2000475DD90E48599F0E4959380E4A590001F1
:107A300002E2000E01D0010E3C1202E0BAEF45F066
:107A4000AA6A3E0EA96E0601475159EC02F0485150
:107A500059EC02F0495159EC02F04A5159EC02F04C
:107A60000001E0EF45F0FEEC45F068C646F667C65B
:107A700045F666C644F665C643F6800E0601435DCC
:107A8000960E4459980E4559000E46590001D8B03B
:107A90007AD003011A6B150E03011A5D000111E281
:107AA00004EE0CF003011A51E926000EEA22EF5011
:107AB0000C6E0D0E0C5C000104E003011A2B00019A
:107AC000EAE3080E03011A5D00010CE204EE0CF07B
:107AD00003011A51E926000EEA22300EEF6E1A2B2E
:107AE0000001EFD70D0E0401156F0601466B456BC3
:107AF000446B436B03011A6B090E03011A5D00010D
:107B0000D8B041D0286A276A266A0A0E256E28C096
:107B100014F027C013F026C012F025C011F046C69D
:107B20001CF045C61BF044C61AF043C619F09EEC83
:107B300003F014C028F013C027F012C026F011C0C3
:107B400025F004EE0CF003011A51E926000EEA229A
:107B5000EF500C6E2C6A2B6A2A6A0CC029F00F0EAB
:107B60002916295025240601436F2A502620446FE8
:107B70002B502720456F2C502820466F03011A2BCD
:107B80000001D8A0B9D7000E0601465D000114E33C
:107B900011E1980E0601455D00010EE30BE1960E22
:107BA0000601445D000108E305E1800E0601435D26
:107BB000000102E3000E01D0010E3C6EC10E060171
:107BC000435D0E0E4459160E4559020E46590001EA
:107BD00002E2000E01D0010E3C1202E0BAEF45F0C5
:107BE000AA6A360EA96E0601435159EC02F04451BF
:107BF00059EC02F0455159EC02F0465159EC02F0B3
:107C00000001E0EF45F065EC45F00301306B2F6BB0
:107C10001A6B000104EE0CF003011A51E926000E64
:107C2000EA22EF500C6E0D0E0C5C00012DE004EE0C
:107C30000CF003011A51E926000EEA22EF501C6FE6
:107C4000266A0A0E256E26C012F02550116E2F03EB
:107C5000F3CF25F0F4CF26F012502F03F350262651
:107C600011503003F35026261CC329F02A6A0F0E48
:107C70002916000E2A16295025242F6F2A50262057
:107C8000306F1A2B0001C5D7AA6A3A0EA96E0301FC
:107C90002F5159EC02F0305159EC02F00001E0EFA5
:107CA00045F0FEEC45F066C650F665C64FF6030E8D
:107CB0000601505D000117E305E1E90E06014F5D85
:107CC000000111E3160EF76E880EF66ECEEC01F091
:107CD0000D0ED6EC01F0030E0601506F520E4F6FE1
:107CE0000001BAEF45F0AA6A420EA96E06014F5193
:107CF00059EC02F0505159EC02F00001E0EF45F070
:107D0000FEEC45F066C652F665C651F6030E060156
:107D1000525D000116E305E1E90E0601515D000127
:107D200010E3160EF76EA20EF66ECEEC01F00D0EFD
:107D3000D6EC01F00601526B640E516F0001BAEFF0
:107D400045F0AA6A440EA96E0601515159EC02F0A1
:107D5000525159EC02F00001E0EF45F0FEEC45F025
:107D600065C653F6090E0601535D00010FE3160EBA
:107D7000F76EBA0EF66ECEEC01F00D0ED6EC01F0F9
:107D8000070E0601536F0001BAEF45F0AA6A460ECE
:107D9000A96E0601535159EC02F00001E0EF45F0E5
:107DA000FEEC45F065C654F6030E0601545D000175
:107DB00002E2000E01D0010E3C6E0F0E0601545D72
:107DC000D8A4010E3C16010E5453D8A4000E3C1644
:107DD00000010FE0160EF76ECE0EF66ECEEC01F03F
:107DE0000D0ED6EC01F0020E0601546F0001BAEF41
:107DF00045F0AA6A470EA96E0601545159EC02F0EB
:107E00000001E0EF45F0FEEC45F065C696F6030193
:107E10001A6B0F0E03011A5D00011BE204EE0CF059
:107E200003011A51E926000EEA22EF501C6F0D0ED5
:107E30001C5D00010EE0AA6A3D0E03011A25A96E21
:107E4000D8B0AA2A1C5159EC02F003011A2B0001E8
:107E5000E0E3AA6A3D0E03011A25A96ED8B0AA2A4A
:107E6000FF0E59EC02F00001E0EF45F0FEEC45F0AA
:107E700065C69AF6650E06019A5D000103E3640E7D
:107E800006019A6F0001AA6A350EA96E06019A5181
:107E900059EC02F09A5176EC07F032EC04F036C05F
:107EA0002CF035C02BF034C02AF033C029F0366AEC
:107EB000356A200E346E820E336E2CC03AF02BC021
:107EC00039F02AC038F029C037F0C7EC06F036C0C8
:107ED00022F335C021F334C020F333C01FF322C393
:107EE00036F021C335F020C334F01FC333F0C7ECA4
:107EF00005F003011C6F150E1C5D000103E3140E59
:107F000003011C6F03011C51040D1508000114E34B
:107F1000F86AFC0EF324F66E230EF420F76E0900C7
:107F2000F5CF11F00900F5CF12F00900F550090066
:107F3000F2EC02F011C061F6AA6A4D0EA96E0601BC
:107F4000615159EC02F0000199EC25F0E0EF45F0A9
:107F50000D0ED6EC01F0160EF76EE20EF66ECEECBC
:107F600001F0016A086A1A6A0E0E196E69EC00F0D7
:107F70002E0ED6EC01F0010E086E8C0E67EC00F0B0
:107F80000D0ED6EC01F0E0EF45F04F0ED6EC01F00F
:107F90004B0ED6EC01F00D0ED6EC01F0010E166E74
:107FA000F40ED8EC02F089EC47F078EC68F038EF8A
:107FB00016F0C2EC4AF00601B9510001E8B234D023
:107FC00068EC4BF0160EF76EF40EF66ECEEC01F088
:107FD000016A8AC628F089C627F088C626F087C6B7
:107FE00025F0020EA2EC00F0560ED6EC01F0200EA9
:107FF000D6EC01F0D6EC01F0160EF76EFC0EF66E24
:10800000CEEC01F0016A82C628F081C627F080C656
:1080100026F07FC625F0010EA2EC00F0430ED6EC50
:1080200001F00D0ED6EC01F0E9EF45F0AA6A4D0E15
:10803000A96E69EC02F00601616F170EF76E040E6F
:10804000F66ECEEC01F0016A9A5166EC00F00D0E6E
:10805000D6EC01F06E0ED6EC01F03A0ED6EC01F043
:10806000200ED6EC01F0016A615166EC00F00D0EB5
:10807000D6EC01F0170EF76E140EF66ECEEC01F092
:108080000D0ED6EC01F0939A8A8A0001E2EC26F0FC
:10809000D6EC25F0750E096E300E026EAEEC01F0D6
:1080A000F9E303011C6F440E1C5D010ED8A4000E01
:1080B0003C6E640E1C5D010ED8A4000E3C12000143
:1080C00020E0060161510001E8BE06D006016153BF
:1080D000000102E00601610700016E0ED6EC01F01E
:1080E000200ED6EC01F03D0ED6EC01F0200ED6ECC1
:1080F00001F0016A0601615166EC00F00D0ED6EC4C
:1081000001F0550E03011C5D010ED8A4000E3C6E5B
:10811000750E1C5D010ED8A4000E3C1200011EE07D
:10812000060161BF04D07F0E615D000102E206011D
:10813000612B00016E0ED6EC01F0200ED6EC01F0A2
:108140003D0ED6EC01F0200ED6EC01F0016A0601DE
:10815000615166EC00F00D0ED6EC01F0450E030106
:108160001C5D010ED8A4000E3C6E650E1C5D010E58
:10817000D8A4000E3C12000104E0C2EC25F0E0EFB0
:1081800045F0530E03011C5D010ED8A4000E3C6E99
:10819000730E1C5D010ED8A4000E3C1200010EE00F
:1081A000C2EC25F0AA6A4D0EA96E0601615159EC88
:1081B00002F061C62CF60001E0EF45F099EC25F0E5
:1081C00069D765EC45F004010C5103014F6F0401C0
:1081D0000D510301506FAA6A290EA96E4F5159EC37
:1081E00002F0AA6A2A0EA96E505159EC02F0000161
:1081F000E0EF45F0FEEC45F065C654F3020E0301D6
:10820000545D000103E2020E0301546F0001AA6AEB
:108210002E0EA96E0301545159EC02F00001E0EF5B
:1082200045F00D0ED6EC01F0170EF76E420EF66E0D
:10823000CEEC01F00D0ED6EC01F00D0ED6EC01F0F7
:10824000170EF76E5C0EF66ECEEC01F00D0ED6EC4E
:1082500001F0170EF76E7C0EF66ECEEC01F00D0EEF
:10826000D6EC01F0170EF76E9A0EF66ECEEC01F01A
:108270000D0ED6EC01F0170EF76EC40EF66ECEECB6
:1082800001F00D0ED6EC01F0170EF76EEE0EF66E45
:10829000CEEC01F00D0ED6EC01F0180EF76E140EB8
:1082A000F66ECEEC01F00D0ED6EC01F0180EF76E66
:1082B000480EF66ECEEC01F00D0ED6EC01F0180E65
:1082C000F76E7E0EF66ECEEC01F00D0ED6EC01F0E0
:1082D000180EF76EA40EF66ECEEC01F00D0ED6EC75
:1082E00001F0180EF76ECE0EF66ECEEC01F00D0E0C
:1082F000D6EC01F0180EF76EE40EF66ECEEC01F03F
:108300000D0ED6EC01F0180EF76EFA0EF66ECEECEE
:1083100001F00D0ED6EC01F0190EF76E160EF66E8A
:10832000CEEC01F00D0ED6EC01F0190EF76E420EF8
:10833000F66ECEEC01F00D0ED6EC01F0190EF76ED4
:10834000620EF66ECEEC01F00D0ED6EC01F0190EB9
:10835000F76E8A0EF66ECEEC01F00D0ED6EC01F043
:10836000190EF76EBE0EF66ECEEC01F00D0ED6ECC9
:1083700001F0190EF76EF20EF66ECEEC01F00D0E56
:10838000D6EC01F01A0EF76E280EF66ECEEC01F068
:108390000D0ED6EC01F01A0EF76E620EF66ECEECF4
:1083A00001F00D0ED6EC01F01A0EF76E9C0EF66E73
:1083B000CEEC01F00D0ED6EC01F01A0EF76EBC0EED
:1083C000F66ECEEC01F00D0ED6EC01F01B0EF76E42
:1083D000020EF66ECEEC01F00D0ED6EC01F01B0E87
:1083E000F76E280EF66ECEEC01F00D0ED6EC01F015
:1083F0001B0EF76E5C0EF66ECEEC01F00D0ED6EC99
:1084000001F01B0EF76E820EF66ECEEC01F00D0E33
:10841000D6EC01F01B0EF76EAC0EF66ECEEC01F052
:108420000D0ED6EC01F01B0EF76EDE0EF66ECEECE6
:1084300001F00D0ED6EC01F01C0EF76E0C0EF66E70
:10844000CEEC01F00D0ED6EC01F01C0EF76E360EE0
:10845000F66ECEEC01F00D0ED6EC01F01C0EF76EB0
:10846000700EF66ECEEC01F00D0ED6EC01F01C0E87
:10847000F76E9A0EF66ECEEC01F00D0ED6EC01F012
:108480001C0EF76EDC0EF66ECEEC01F00D0ED6EC87
:1084900001F01D0EF76E0A0EF66ECEEC01F00D0E19
:1084A000D6EC01F01D0EF76E360EF66ECEEC01F036
:1084B0000D0ED6EC01F01D0EF76E600EF66ECEECD2
:1084C00001F00D0ED6EC01F01D0EF76E760EF66E75
:1084D000CEEC01F00D0ED6EC01F01D0EF76EA60EDF
:1084E000F66ECEEC01F00D0ED6EC01F01D0EF76E1F
:1084F000E40EF66ECEEC01F00D0ED6EC01F01E0E81
:10850000F76E020EF66ECEEC01F00D0ED6EC01F019
:108510001E0EF76E300EF66ECEEC01F00D0ED6ECA0
:1085200001F01E0EF76E7A0EF66ECEEC01F00D0E17
:10853000D6EC01F01E0EF76E980EF66ECEEC01F042
:108540000D0ED6EC01F01E0EF76EC00EF66ECEECE0
:1085500001F00D0ED6EC01F01F0EF76E0C0EF66E4C
:10856000CEEC01F00D0ED6EC01F01F0EF76E320EC0
:10857000F66ECEEC01F00D0ED6EC01F01F0EF76E8C
:10858000460EF66ECEEC01F00D0ED6EC01F01F0E8D
:10859000F76E660EF66ECEEC01F00D0ED6EC01F025
:1085A0001F0EF76E860EF66ECEEC01F00D0ED6ECB9
:1085B00001F01F0EF76EA60EF66ECEEC01F00D0E5A
:1085C000D6EC01F01F0EF76EC60EF66ECEEC01F083
:1085D0000D0ED6EC01F01F0EF76EEC0EF66ECEEC23
:1085E00001F00D0ED6EC01F0200EF76E120EF66EB5
:1085F000CEEC01F00D0ED6EC01F0200EF76E3A0E27
:10860000F66ECEEC01F00D0ED6EC01F0200EF76EFA
:10861000540EF66ECEEC01F00D0ED6EC01F0200EED
:10862000F76E860EF66ECEEC01F00D0ED6EC01F074
:10863000200EF76EB60EF66ECEEC01F00D0ED6ECF7
:1086400001F0200EF76ED40EF66ECEEC01F00D0E9A
:10865000D6EC01F0200EF76EEA0EF66ECEEC01F0CD
:108660000D0ED6EC01F0210EF76E160EF66ECEEC66
:1086700001F00D0ED6EC01F0210EF76E360EF66EFF
:10868000CEEC01F00D0ED6EC01F0210EF76E4E0E81
:10869000F66ECEEC01F00D0ED6EC01F0210EF76E69
:1086A000680EF66ECEEC01F00D0ED6EC01F0210E48
:1086B000F76E820EF66ECEEC01F00D0ED6EC01F0E8
:1086C000210EF76E960EF66ECEEC01F00D0ED6EC86
:1086D00001F0210EF76EAA0EF66ECEEC01F00D0E33
:1086E000D6EC01F0210EF76EC00EF66ECEEC01F066
:1086F0000D0ED6EC01F0210EF76ED60EF66ECEEC16
:1087000001F00D0ED6EC01F0210EF76EE80EF66EBC
:10871000CEEC01F00D0ED6EC01F0210EF76EFE0E40
:10872000F66ECEEC01F00D0ED6EC01F0E0EF45F068
:10873000030116970001B3EC2AF0030116911A6B9E
:10874000000104EE0CF003011A51E926000EEA22A2
:10875000EF500C6E2D0E0C5CD8A4010E3C6E04EE96
:108760000CF01A51E926000EEA22EF500C6E200E92
:108770000C5CD8A4010E3C1604EE0CF01A51E9264C
:10878000000EEA22EF500C6E0D0E0C5CD8A4010E08
:108790003C160A0E1A5D010ED8B0000E3C16000100
:1087A00014E004EE0CF003011A51E926000EEA224F
:1087B000EFCF0CF000EEE8F01A51E926000EEA22A5
:1087C0000CC0EFFF1A2B0001BBD7060E03011A5D88
:1087D000000113E21AC31BF3060E03011B5D000127
:1087E0000CE200EEE8F003011B51E926000EEA223C
:1087F000200EEF6E1B2B0001EFD704EE0CF00301EF
:108800001A51E926000EEA22EF500C6E200E0C5C85
:10881000000101E1EE6B04EE0CF003011A51E926B0
:10882000000EEA22EF500C6E0D0E0C5C000105E10B
:10883000030116810001EE6B120004EE0CF003013F
:108840001A51E926000EEA22EF500C6E2D0E0C5C38
:108850000001D8A46AD003011A2B04EE0CF01A51BF
:10886000E926000EEA22EF500C6E0F0E0C144E6E2D
:108870001A2B04EE0CF01A51E926000EEA22EF50F2
:108880000C6E300E0C5C000ED8B0010E3C6E04EE87
:108890000CF01A51E926000EEA22EF500C6E3A0E47
:1088A0000C5C000102E3000E01D0010E3C1629E031
:1088B000266A0A0E256E26C011F04E502502F3CF0F
:1088C00025F0F4CF26F01102F350262604EE0CF02A
:1088D00003011A51E926000EEA22EF500C6E2A6AB3
:1088E0000CC029F00F0E2916000E2A162550292437
:1088F0004E6E100E4E5C000102E30F0E4E6E030131
:108900001A2B00014EC0EEF004EE0CF003011A51D8
:10891000E926000EEA22EF500C6E0D0E0C5C0001F1
:1089200004E1030116810001120003011A2B04EE79
:108930000CF01A51E926000EEA22EF500C6E560E8A
:108940000C5C010ED8A4000E3C6E04EE0CF01A5123
:10895000E926000EEA22EF500C6E760E0C5C010E3A
:10896000D8A4000E3C12000103E0AFD8AED802D06C
:10897000030116870001120003011A6B070E0301A1
:108980001A5D000118E200EEE8F003011A51E92631
:10899000000EEA22EF500C6ED8900C344B6E060E8F
:1089A0001A5D000102E14E504B120FEC29F0030159
:1089B0001A2B0001E3E3120003011A6B000100EE21
:1089C000E8F003011A51E926000EEA22EF500C6E7E
:1089D000200E0C5CD8A4010E3C6E060E1A5D010E32
:1089E000D8B0000E3C1600010DE000EEE8F00301E7
:1089F0001A51E926000EEA22EF50D6EC01F01A2BAC
:108A00000001DCD7EE510C6E0C5207E02D0ED6ECB7
:108A100001F0016AEE5166EC00F0120003011A6BDE
:108A2000000100EE4FF003011A51EB500C6E200EC6
:108A30000C5CD8A4010E3C6E060E1A5D010ED8B077
:108A4000000E3C1600010EE000EE4FF003011A513B
:108A5000EBCF0CF005EEADF01A510CC0EBFF1A2B6A
:108A60000001DED7F36A05EEADF003011A51F3CF32
:108A7000EBFF00EEE8F0240EEE6EEE6EEE6EEE6EA4
:108A800015EEADF0320EE75204E0E6CFEEFFE82E31
:108A9000FAD7EF6A55500C6E0C52000115E000EE4B
:108AA000E8F0EE50FEE1ED522D0EEE6E020E016E7C
:108AB000EACF0DF0E9CF0CF055500DC0EAFF0CC025
:108AC000E9FF66EC00F0EF6A120003011697366BBF
:108AD000000104EE0CF003013651E926000EEA22F3
:108AE000EF500C6E200E0C5CD8A4010E3C6EFD0EF7
:108AF000365D010ED8B0000E3C16000115E004EE04
:108B00000CF003013651E926000EEA22EF500C6EFC
:108B10000D0E0C5C000104E1030116870001120038
:108B20000301362B0001D4D70301362B3651FF0841
:108B30000B6E1B6B03011B510B5C00011AE303015D
:108B40001B5136250E6E0F6A0F360E500C0FE96E54
:108B5000040E0F20EA6EEFCF0CF004EE0CF01B5168
:108B6000E926000EEA220CC0EFFF03011B2B0001D7
:108B7000E1E31200450ED6EC01F0520ED6EC01F006
:108B8000D6EC01F04F0ED6EC01F0520ED6EC01F00F
:108B90000D0ED6EC01F0630ED6EC01F06D0ED6ECA6
:108BA00001F0640ED6EC01F03E0ED6EC01F0AECF33
:108BB0001CF300EEE8F0EF6A04EE0CF0EF6A12002E
:108BC0004F0ED6EC01F04B0ED6EC01F00D0ED6ECAC
:108BD00001F0630ED6EC01F06D0ED6EC01F0640EE0
:108BE000D6EC01F03E0ED6EC01F0AECF1CF300EE59
:108BF000E8F0EF6A04EE0CF0EF6A120066DF010E97
:108C000003011A6F04010C510C6E0F0B0601686B07
:108C1000676B666B656F000104EE0CF003011A517F
:108C2000E926000EEA22EF500C6E0D0E0C5C0001DE
:108C3000D8B440D0286A276A266A0A0E256E28C052
:108C400014F027C013F026C012F025C011F068C63A
:108C50001CF067C61BF066C61AF065C619F09EECDC
:108C600003F014C028F013C027F012C026F011C082
:108C700025F004EE0CF003011A51E926000EEA2259
:108C8000EF500C6E2C6A2B6A2A6A0CC029F00F0E6A
:108C90002916295025240601656F2A502620666F63
:108CA0002B502720676F2C502820686F03011A2B48
:108CB0000001B1D71200476A486A496A4B6A4D6A97
:108CC0004C6A4E6A0301536B168B576B00011200FE
:108CD000FCDEB3EC2AF00301189104010C510C6E78
:108CE0004F0E0C5C010ED8A4000E3C6E0D510C6EA4
:108CF0004E0E0C5C010ED8A4000E3C16000104E0E0
:108D000003011685000158D004010C510C6E590E58
:108D10000C5C010ED8A4000E3C6E0D510C6E450E7D
:108D20000C5C010ED8A4000E3C160E510C6E530EB6
:108D30000C5C010ED8A4000E3C16000104E00301F7
:108D40001685000139D004010C510C6E4F0E0C5CDD
:108D5000010ED8A4000E3C6E0D510C6E460E0C5C3C
:108D6000010ED8A4000E3C160E510C6E460E0C5C83
:108D7000010ED8A4000E3C16000104E00301169574
:108D800000011AD004010C510C6E4E0E0C5C010E49
:108D9000D8A4000E3C6E0D510C6E4F0E0C5C010EF3
:108DA000D8A4000E3C16000104E003011695000152
:108DB00002D0030118810001120003011A6B070E93
:108DC00003011A5D000116E203011A512325A96E61
:108DD000000E2421AA6E69EC02F00C6E00EEE8F0A1
:108DE0001A51E926000EEA220CC0EFFF03011A2BEC
:108DF0000001E5E3EF6B1200030111510001E8AA45
:108E000087D003011B6B1897189B0601B981630E6D
:108E100003011B5D0001D8B07BD0AA6A780E030164
:108E20001B25A96ED8B0AA2A69EC02F01C6F0D0EA2
:108E30001C5D0001D8B46CD05C0E03011C5D000108
:108E4000D8A462D0030118871B2BAA6A780E1B25B1
:108E5000A96ED8B0AA2A69EC02F01C6F1C9B550EB3
:108E60001C5D000102E161EC52F0560E03011C5D35
:108E7000010ED8A4000E3C6E570E1C5D010ED8A446
:108E8000000E3C12000102E0CBEC4BF0540E03014B
:108E90001C5D000102E11FEC51F0580E03011C5D46
:108EA000000102E1C0EC51F0420E03011C5D000123
:108EB0000CE100EE85F015EEA7F0050EE75204E098
:108EC000E6CFEEFFE82EFAD7EF6A03011251000158
:108ED000E8A603D023EC53F009D000EE8AF0200E70
:108EE000EE6EEF6A00EE90F0EE6EEF6A500E030148
:108EF0001C5D000109E10601B9510001E8B402D08E
:108F000017EC5DF0C2EC5DF003011B2B00017FD775
:108F10001200AA6A230EA96E69EC02F00301116F18
:108F2000AA6A240EA96E69EC02F0126FAA6A250ED5
:108F3000A96E69EC02F0136FAA6A260EA96E69EC9D
:108F400002F0146FAA6A270EA96E69EC02F0106F86
:108F50000001B1DEAA6A2C0EA96E69EC02F00301D1
:108F6000516FAA6A2F0EA96E69EC02F0586FAA6AB7
:108F7000300EA96E69EC02F0596FCD80AA6A290EF5
:108F8000A96E69EC02F04F6FAA6A2A0EA96E69EC0D
:108F900002F0506FAA6A2E0EA96E69EC02F0546FAF
:108FA000556BAA6A2D0EA96E69EC02F0566F11314D
:108FB000000111E30301246B236B0001FEDE00EED0
:108FC0004FF010EEE8F0960EE75204E0E6CFEEFF29
:108FD000E82EFAD7EF6A030111510001E8A212D07E
:108FE0000301246B070E236F0001E7DE00EE58F04B
:108FF00010EEE8F0960EE75204E0E6CFEEFFE82E22
:10900000FAD7EF6A030111510001E8A412D003015D
:10901000246B0E0E236F0001D0DE00EE61F010EE27
:10902000E8F0960EE75204E0E6CFEEFFE82EFAD71E
:10903000EF6A030111510001E8A612D00301246B6D
:10904000150E236F0001B9DE00EE6AF010EEE8F0B5
:10905000960EE75204E0E6CFEEFFE82EFAD7EF6A6D
:10906000030111510001E8A812D00301246B1C0E6A
:10907000236F0001A2DE00EE73F010EEE8F0960E12
:10908000E75204E0E6CFEEFFE82EFAD7EF6AAA6ACD
:10909000310EA96E69EC02F006013F6F69EC02F037
:1090A000406F69EC02F0416F69EC02F0426F070E0D
:1090B000425D000114E311E1170E0601415D00015C
:1090C0000EE30BE1CB0E0601405D000108E305E174
:1090D000C00E06013F5D000102E3000E01D0010E4B
:1090E0003C6E810E06013F5DD90E40599F0E4159DD
:1090F000380E4259000102E2000E01D0010E3C126E
:1091000008E0080E0601426FA10E416F790E406F14
:109110003F6B0001AA6A3E0EA96E69EC02F00601DF
:10912000476F69EC02F0486F69EC02F0496F69EC37
:1091300002F04A6F070E4A5D000114E311E1170EB9
:109140000601495D00010EE30BE1CB0E0601485D0F
:10915000000108E305E1C00E0601475D000102E3DE
:10916000000E01D0010E3C6E810E0601475DD90E46
:1091700048599F0E4959380E4A59000102E2000E23
:1091800001D0010E3C1209E0080E06014A6F9E0E46
:10919000496F6B0E486FC00E476F960E0601956FB4
:1091A000AA6A350EA96E69EC02F09A6FAA6A4D0E92
:1091B000A96E69EC02F02C6F650E9A5D000103E365
:1091C000640E06019A6F06019A5176EC07F032ECB4
:1091D00004F036C02CF035C02BF034C02AF033C078
:1091E00029F0366A356A200E346E820E336E2CC03A
:1091F0003AF02BC039F02AC038F029C037F0C7EC5C
:1092000006F036C022F335C021F334C020F333C05A
:109210001FF322C336F021C335F020C334F01FC33F
:1092200033F0C7EC05F003011C6F150E1C5D000147
:1092300003E3140E03011C6F03011C51040D1508F8
:10924000000114E3F86A540EF324F66E240EF420A1
:10925000F76E0900F5CF11F00900F5CF12F0090003
:10926000F5500900F2EC02F011C08EF606018E51A5
:109270002C5D000103E02CC661F602D08EC661F6BB
:10928000320E06019A5D000125E2030E03011C2740
:10929000150E1C5D000103E3140E03011C6F030196
:1092A0001C51040D1508000114E3F86AAC0EF324F8
:1092B000F66E240EF420F76E0900F5CF11F00900C8
:1092C000F5CF12F00900F5500900F2EC02F011C0E0
:1092D00097F603D07F0E0601976F06018D6B140E73
:1092E0008C6FAA6A3D0EA96E69EC02F0966F140E9F
:1092F000965D000103E2140E0601966F790E0601D9
:10930000965D000103E3780E0601966F0001040EDE
:10931000126EB00E116E166A96C615F04CEC03F084
:1093200006018C6F12C08DF68CC691F6AA6A360EB5
:10933000A96E69EC02F0436F69EC02F0446F69ECCE
:1093400002F0456F69EC02F0466F000E465D0001C9
:1093500014E311E1980E0601455D00010EE30BE1F7
:10936000960E0601445D000108E305E1800E06014A
:10937000435D000102E3000E01D0010E3C6E410E80
:109380000601435D8A0E4459F70E4559010E4659B0
:10939000000102E2000E01D0010E3C1209E0010EB4
:1093A0000601466FC90E456FC30E446F800E436FB2
:1093B0000001AA6A3C0EA96E69EC02F006019B6FDF
:1093C000AA6A420EA96E69EC02F04F6F69EC02F0D6
:1093D000506F030E505D00010BE305E1E90E06013D
:1093E0004F5D000105E3030E0601506F520E4F6FF3
:1093F0000001AA6A440EA96E69EC02F00601516FE1
:1094000069EC02F0526F030E525D00010AE305E1C0
:10941000E90E0601515D000104E30601526B640E82
:10942000516F0001AA6A460EA96E69EC02F00601AE
:10943000536F090E535D000103E3070E0601536FDE
:109440000001AA6A470EA96E69EC02F00601546F8A
:10945000030E545D000102E2000E01D0010E3C6ECD
:109460000F0E0601545DD8A4010E3C16000103E066
:10947000020E0601546F000105EEA7F0EF6A060127
:10948000996B01EEAFF0300EEE6E2E0EEE6E300EDA
:10949000EE6EEF6A0501A46BA36BA66BA56B146A55
:1094A0000F0E136E420E126E400E116E51C619F061
:1094B00052C61AF01B6A1C6A1EEC03F012C06CF64E
:1094C00011C06BF60F0E0601545D00010CE00601A1
:1094D00054516B03F3CF6DF6F4CF6EF66C03F3507B
:1094E0006E2700010BD0D89006016C31266E6B31CF
:1094F000256E6B256D6F26506C216E6F0001AA6A78
:10950000480EA96E69EC02F00601B06FAA6A490E16
:10951000A96E69EC02F0B16FAA6A4A0EA96E69ECF5
:1095200002F0B26FAA6A4B0EA96E69EC02F0B36F3B
:10953000AA6A4C0EA96E69EC02F0B46F080EB05D19
:10954000010ED8A4000E3C6E080EB15D010ED8A429
:10955000000E3C12080EB25D010ED8A4000E3C12A3
:10956000080EB35D010ED8A4000E3C12080EB45DC7
:10957000010ED8A4000E3C12000102E00301128B80
:109580000001120081940601B993949E8B9E810E76
:10959000026E010E096E810E036E040E046E010E42
:1095A0000A6E116EAEEC02F0949E8B8E03015B6B23
:1095B0005A6B000181B618D003015A2B000E5B23B1
:1095C0005B5304E1FB0E5A5D00010DE3220EF76EC2
:1095D000140EF66ECEEC01F00D0ED6EC01F0060185
:1095E000B98300011200E5D7949E8B9E03015B6B4B
:1095F0005A6B0001810E026E010E096E810E036E20
:10960000040E046E010E0A6E440E116EAEEC02F0F2
:10961000810E026E020E096E810E036E040E046E40
:109620000A6A85EC02F011C01CF303011C29000139
:1096300023E0949E8B8E010ED7EC02F0949E8B9EBD
:1096400003015A2B000E5B23610E5B5D000113E3E7
:1096500005E1A90E03015A5D00010DE3220EF76E2C
:109660002E0EF66ECEEC01F00D0ED6EC01F00601DA
:10967000B98300011200BDD7810E026E020E096E81
:10968000810E036E040E046E0A6A85EC02F011C0AE
:109690009CF685EC02F011C09DF685EC02F011C03D
:1096A0009EF685EC02F011C09FF685EC02F011C029
:1096B000A0F685EC02F011C0A1F685EC02F011C015
:1096C000A2F685EC02F011C0A3F6949E8B8E1200D8
:1096D000220EF76E4E0EF66ECEEC01F0016A060118
:1096E0009C5166EC00F00D0ED6EC01F0220EF76EE8
:1096F0005E0EF66ECEEC01F0016A020E086E9D5110
:109700004FEC00F0020E086E9E514FEC00F00D0E73
:10971000D6EC01F0220EF76E680EF66ECEEC01F07C
:10972000016A020E086E9F514FEC00F00D0ED6EC50
:1097300001F0220EF76E780EF66ECEEC01F0016AA3
:10974000020E086EA0514FEC00F0020E086EA151FF
:109750004FEC00F00D0ED6EC01F0220EF76E8C0EE1
:10976000F66ECEEC01F0016A020E086EA2514FECCB
:1097700000F00D0ED6EC01F0220EF76E9C0EF66E88
:10978000CEEC01F0016A020E086EA3514FEC00F01E
:109790000D0ED6EC01F0030E0501E06F140EE16F23
:1097A000180EE26FE36B060EE46F00018EEC50F0D2
:1097B0000501E2510301246F0501E3510301236F09
:1097C00023C333F024C334F078EC07F03A6A396AE3
:1097D000400E386E800E376EC7EC06F036C028F0AB
:1097E00035C027F034C026F033C025F03A6A396A14
:1097F000200E386E890E376E28C036F027C035F03F
:1098000026C034F025C033F061EC06F036C08AF68D
:1098100035C089F634C088F633C087F6000E14BF11
:10982000010E3C6E010E0601B9B1000E3C1600019E
:1098300025E0366A356A480E346E850E336E8AC668
:109840003AF089C639F088C638F087C637F0C7ECD9
:1098500006F015EC07F00301236F34C024F300EE8B
:10986000B1F0020E016E030E086E24C31AF023C37A
:1098700019F069EC00F0EF6A00010FD000EEB1F0D2
:10988000020E016E8AC628F089C627F088C626F027
:1098900087C625F0A2EC00F0EF6A0501E451030150
:1098A000246F0501E5510301236F340E226F330E3F
:1098B000216F630E206F7C0E1F6F24C334F023C30F
:1098C00033F070EC07F022C33AF021C339F020C323
:1098D00038F01FC337F0C7EC06F036C028F035C0AB
:1098E00027F034C026F033C025F03A6A800E396E76
:1098F000140E386E870E376E28C036F027C035F04C
:1099000026C034F025C033F0D1EC05F036C082F625
:1099100035C081F634C080F633C07FF6000E14BF28
:10992000010E3C6E010E0601B9B1000E3C1600019D
:109930003DE0366A356A200E346E840E336E82C680
:109940003AF081C639F080C638F07FC637F0D3ECE4
:1099500005F036C028F035C027F034C026F033C0FB
:1099600025F0366A356A200E346E820E336E28C0BA
:109970003AF027C039F026C038F025C037F0C7ECE0
:1099800006F015EC07F00301236F34C024F300EE5A
:10999000BCF0020E016E030E086E24C31AF023C33E
:1099A00019F069EC00F0EF6A000110D000EEBCF095
:1099B000020E016E82C628F081C627F080C626F00E
:1099C0007FC625F0010EA2EC00F0EF6A1200030141
:1099D0001B6B000101EC27F0266A0A0E256E0501BB
:1099E000AD510C6E2A6A0CC029F00F0E2916000E1C
:1099F0002A1626C01EF025C01DF02AC016F029C068
:109A000015F0DFEC03F0256E1AC026F0AE510E6E95
:109A10002A6A0EC029F00F0E2916000E2A162550AC
:109A200029240601A56F266A0A0E256E0501AF518D
:109A30000C6E2A6A0CC029F00F0E2916000E2A1689
:109A400026C01EF025C01DF02AC016F029C015F052
:109A5000DFEC03F0256E1AC026F0B0510E6E2A6AB4
:109A60000EC029F00F0E2916000E2A1625502924A3
:109A70000601A66F3A6A396A700E386E840E376E28
:109A8000A65176EC07F061EC06F036C028F035C040
:109A900027F034C026F033C025F0A55176EC07F04E
:109AA00028C03AF027C039F026C038F025C037F07A
:109AB000D3EC05F036C022F335C021F334C020F3D7
:109AC00033C01FF3266A0A0E256E0501B2510C6ED3
:109AD0002A6A0CC029F00F0E2916000E2A1626C07D
:109AE0001EF025C01DF02AC016F029C015F0DFECCD
:109AF00003F0256E1AC026F0B3510E6E2A6A0EC00E
:109B000029F00F0E2916000E2A16255029240601C9
:109B1000AA6F03011B6B000100EC27F005EEADF00E
:109B2000EECFF3FFEFCFF4FFF3504E0AF41005E150
:109B30005A0E0601A527000115D00601A5515A08A5
:109B4000A56FA65300010EE00601A507A6513C082B
:109B5000A66FAA53000105E00601A607AA516408F2
:109B6000AA6F0001D8900601A637D890AA37030142
:109B70001B6B0001FFEC26F0266A640E256E0501C2
:109B8000AD510C6E2A6A0CC029F00F0E2916000E7A
:109B90002A1626C01EF025C01DF02AC016F029C0C6
:109BA00015F0DFEC03F0256E1AC026F02A6A0A0EC3
:109BB000296EAE510E6E2E6A0EC02DF00F0E2D16B0
:109BC000000E2E162AC01EF029C01DF02EC016F061
:109BD0002DC015F0DFEC03F0296E1AC02AF02950D1
:109BE00025262A502622AF51106E2A6A10C029F06D
:109BF0000F0E2916000E2A16295025240601A76FDC
:109C00002A502620A86F266A0A0E256E0501B0513B
:109C10000C6E2A6A0CC029F00F0E2916000E2A16A7
:109C200026C01EF025C01DF02AC016F029C015F070
:109C3000DFEC03F0256E1AC026F0B1510E6E2A6AD1
:109C40000EC029F00F0E2916000E2A1625502924C1
:109C50000601A96F3A6A396A700E386E840E376E43
:109C6000A95176EC07F061EC06F036C028F035C05B
:109C700027F034C026F033C025F0A7C633F0A8C6BD
:109C800034F078EC07F028C03AF027C039F026C04D
:109C900038F025C037F0D3EC05F036C022F335C0DC
:109CA00021F334C020F333C01FF3266A0A0E256E59
:109CB0000501B3510C6E2A6A0CC029F00F0E29164B
:109CC000000E2A1626C01EF025C01DF02AC016F070
:109CD00029C015F0DFEC03F0256E1AC026F0B45150
:109CE0000E6E2A6A0EC029F00F0E2916000E2A16D3
:109CF000255029240601AB6F03011B6B0001FEEC0C
:109D000026F005EEADF0EECFF3FFEFCFF4FFF3500A
:109D1000450AF41007E1B40E0601A727000EA82398
:109D200000011AD00601A751B408A76F000EA8556C
:109D3000A86FA953000110E00601A707000EA85B59
:109D4000A9513C08A96FAB53000105E00601A90722
:109D5000AB516408AB6F000105EEADF0EF6AA8C629
:109D600012F0A7C611F0166A140E156E4CEC03F033
:109D7000256E12C026F0410E252403011C6F05EE4E
:109D8000ADF0EE50FEE1ED521CC3EEFFEF6AA5C64A
:109D900011F00A0E49EC03F0256E266A410E2524C7
:109DA0001C6F05EEADF0EE50FEE1ED521CC3EEFF70
:109DB000EF6A266A300E256EA8C62AF0A7C629F0DB
:109DC0002AC012F029C011F0166A140E156E4CEC60
:109DD00003F01AC02AF019C029F0D8902A3229328B
:109DE000255029241C6F05EEADF0EE50FEE1ED523A
:109DF0001CC3EEFFEF6A126AA5C611F0166A0A0EBE
:109E0000156E4CEC03F01AC026F019C025F0300E88
:109E100025241C6F05EEADF0EE50FEE1ED521CC3A3
:109E2000EEFFEF6A266A410E256E000E0601A7B10D
:109E3000010E2A6A296E2A503C0DF3CF2AF02950D0
:109E40003C0DF3CF29F0F4502A26A9512926000E03
:109E50002A222AC012F029C011F0166A050E156ECA
:109E60004CEC03F0296E12C02AF02550292403017E
:109E70001C6F05EEADF0EE50FEE1ED521CC3EEFF9F
:109E8000EF6AA6C611F0050E49EC03F0256E266AAE
:109E9000410E25241C6F05EEADF0EE50FEE1ED52B3
:109EA0001CC3EEFFEF6A000E14B9010E3C6E000EEB
:109EB00017B1010E3C120001D8B4E8D03C0E0601E7
:109EC000A7A1000E256EA7A1000E266EA95125247C
:109ED0000301236F000E2620246F24C312F023C336
:109EE00011F0166A050E156E4CEC03F019C01CF348
:109EF0001C51640DF3CF25F0F4CF26F00601AB51D1
:109F000025240301236F000E2620246F24C312F0A2
:109F100023C311F0166A320E156E4CEC03F0256E59
:109F200012C026F0300E25241C6F05EEADF0EE5069
:109F3000FEE1ED521CC3EEFFEF6A24C312F023C30F
:109F400011F0166A320E156E4CEC03F019C0ABF628
:109F5000126AA6C611F0166A050E156E4CEC03F0D7
:109F600019C01CF31C51640DF3CF25F0F4CF26F07B
:109F70000601AA5125240301236F000E2620246F19
:109F800024C312F023C311F0166A320E156E4CEC86
:109F900003F0256E12C026F0300E25241C6F24C35A
:109FA00012F023C311F0166A320E156E4CEC03F05A
:109FB00019C0AAF605EEADF0EE50FEE1ED521CC35D
:109FC000EEFFEF6ADF0E3A6E4F0E396E050E386EF9
:109FD000800E376E0601AB5176EC07F061EC06F0AF
:109FE00036C028F035C027F034C026F033C025F045
:109FF000366A356A020E346E850E336E28C03AF02A
:10A0000027C039F026C038F025C037F0D3EC05F072
:10A0100015EC07F003011C6F05EEADF0EE50FEE10C
:10A02000ED521CC3EEFFEF6ADF0E3A6E4F0E396E33
:10A03000050E386E800E376E0601AA5176EC07F0D9
:10A0400061EC06F036C028F035C027F034C026F0A9
:10A0500033C025F0366A356A020E346E850E336ED3
:10A0600028C03AF027C039F026C038F025C037F0B4
:10A07000D3EC05F015EC07F003011C6F05EEADF015
:10A08000EE50FEE1ED521CC3EEFFEF6A000112003C
:10A0900003015B6B5A6B000181B61AD003015A2B86
:10A0A000000E5B23090E5B5D000111E305E1C50EA7
:10A0B00003015A5D00010BE3220EF76E140EF66EDB
:10A0C000CEEC01F00D0ED6EC01F000011200E3D74A
:10A0D000949E8B9E0501E0510B6E010E0601AC6F44
:10A0E0000601AC510B5C000116E3810E026E010EFD
:10A0F000096E810E036E040E046E010E0A6E05EEEB
:10A10000E0F00601AC51EB50116EAEEC02F006012E
:10A11000AC2B0001E5E3949E8B8E12008194B8DF96
:10A1200003015B6B5A6B000181B61AD003015A2BF5
:10A13000000E5B23610E5B5D000111E305E1A90EDA
:10A1400003015A5D00010BE3220EF76E2E0EF66E30
:10A15000CEEC01F00D0ED6EC01F000011200E3D7B9
:10A16000949E8B9E03015B6B5A6B0001810E026E05
:10A17000010E096E810E036E040E046E010E0A6E4E
:10A18000440E116EAEEC02F0810E026E020E096EEC
:10A19000810E036E040E046E0A6A85EC02F011C093
:10A1A0001CF303011C29000121E0949E8B8E010EFB
:10A1B000D7EC02F0949E8B9E03015A2B000E5B237A
:10A1C000610E5B5D000111E305E1A90E03015A5D1B
:10A1D00000010BE3220EF76E2E0EF66ECEEC01F0B0
:10A1E0000D0ED6EC01F000011200BFD705EEE0F035
:10A1F0000601AC51EB500C6E0C0403011C6F060100
:10A20000AC6B0601AC5103011C5D000115E3810E2E
:10A21000026E020E096E810E036E040E046E0A6A4F
:10A2200085EC02F005EEE0F00601AC5111C0EBFF49
:10A230000601AC2B0001E5E3949E8B8E1200030116
:10A24000266B256B1A6B0A0E03011A5D00010FE2E3
:10A25000010E70EC02F00C6E26C00DF00C500301E4
:10A2600025270D50262303011A2B0001ECE325C3FB
:10A2700033F026C334F078EC07F03A6A400E396EBA
:10A280001C0E386E8A0E376ED1EC05F036C028F001
:10A2900035C027F034C026F033C025F03A6A396A59
:10A2A000480E386E840E376E28C036F027C035F061
:10A2B00026C034F025C033F061EC06F036C07EF6DF
:10A2C00035C07DF634C07CF633C07BF6000E03014A
:10A2D00014BF010E3C6E010E0601B9B1000E3C1612
:10A2E00000013DE0366A356A200E346E840E336E0E
:10A2F0007EC63AF07DC639F07CC638F07BC637F0B2
:10A30000D3EC05F036C028F035C027F034C026F075
:10A3100033C025F0366A356A200E346E820E336EF5
:10A3200028C03AF027C039F026C038F025C037F0F1
:10A33000C7EC06F015EC07F00301236F34C024F3DB
:10A3400000EE9BF0020E016E030E086E24C31AF09D
:10A3500023C319F069EC00F0EF6A000110D000EEA1
:10A360009BF0020E016E7EC628F07DC627F07CC6EB
:10A3700026F07BC625F0010EA2EC00F0EF6A120079
:10A380000301246B236B1A6B0A0E03011A5D000193
:10A390000FE2000E70EC02F00C6E26C00DF00C50B7
:10A3A000030123270D50242303011A2B0001ECE3A2
:10A3B00023C333F024C334F078EC07F03A6A400E3C
:10A3C000396E1C0E386E8A0E376ED1EC05F036C031
:10A3D00028F035C027F034C026F033C025F03A6AA3
:10A3E000396A480E386E840E376E28C036F027C0A2
:10A3F00035F026C034F025C033F061EC06F036C0ED
:10A4000086F635C085F634C084F633C083F6000E78
:10A41000030114BF010E3C6E010E0601B9B1000E1E
:10A420003C1600013DE0366A356A200E346E840E1B
:10A43000336E86C63AF085C639F084C638F083C6D6
:10A4400037F0D3EC05F036C028F035C027F034C023
:10A4500026F033C025F0366A356A200E346E820E3F
:10A46000336E28C03AF027C039F026C038F025C036
:10A4700037F0C7EC06F015EC07F00301236F34C08A
:10A4800024F300EEC7F0020E016E030E086E24C323
:10A490001AF023C319F069EC00F0EF6A000110D044
:10A4A00000EEC7F0020E016E86C628F085C627F0C2
:10A4B00084C626F083C625F0010EA2EC00F0EF6AF8
:10A4C00012000301246B236B1A6B0A0E03011A5D41
:10A4D00000010FE2030E70EC02F00C6E26C00DF0CE
:10A4E0000C50030123270D50242303011A2B0001D4
:10A4F000ECE33A6A400E396E1C0E386E8B0E376EE6
:10A5000024C334F023C333F078EC07F061EC06F099
:10A5100036C074F635C073F634C072F633C071F6C7
:10A52000000E030114BF010E3C6E010E0601B9B10D
:10A53000000E3C16000116E000EEA6F0020E016EC1
:10A54000030E086E24C312F023C311F0166A0A0E1C
:10A55000156E4CEC03F0196E12C01AF069EC00F0A5
:10A56000EF6A0FD000EEA6F0020E016E74C628F05E
:10A5700073C627F072C626F071C625F0A2EC00F073
:10A58000EF6A12000301246B236B1A6B0A0E03019E
:10A590001A5D00010FE20F0E70EC02F00C6E26C087
:10A5A0000DF00C50030123270D50242303011A2B17
:10A5B0000001ECE33A6A400E396E1C0E386E8B0EC9
:10A5C000376E24C334F023C333F078EC07F061EC2A
:10A5D00006F036C078F635C077F634C076F633C06C
:10A5E00075F6000E030114BF010E3C6E010E06014C
:10A5F000B9B1000E3C16000116E000EE90F0020E1C
:10A60000016E030E086E24C312F023C311F0166A04
:10A610000A0E156E4CEC03F0196E12C01AF069ECBC
:10A6200000F0EF6A0FD000EE90F0020E016E78C6D7
:10A6300028F077C627F076C626F075C625F0A2EC7E
:10A6400000F0EF6A12000301266B256B246B236B6D
:10A650001A6B0A0E03011A5D000119E2040E70EC78
:10A6600002F00C6E26C00DF00C50030125270D5092
:10A6700026230F0E70EC02F00C6E26C00DF00C506D
:10A6800023270D50242303011A2B0001E2E30301C9
:10A690002551235D0601796F0301265124590601D6
:10A6A0007A6F7AC620F079C61FF01A6A0B0E196EFF
:10A6B00063EC03F0796F12C07AF63A6A400E396E95
:10A6C0001C0E386E8B0E376E24C334F023C333F068
:10A6D00078EC07F061EC06F036C078F635C077F616
:10A6E00034C076F633C075F6000E030114BF010EB8
:10A6F0003C6E010E0601B9B1000E3C1600012EE0C1
:10A70000640E060179250301256F000E06017A21EA
:10A710000301266F00EE8AF0020E016E030E086E32
:10A7200026C31AF025C319F069EC00F0EF6A00EEB9
:10A7300090F0020E016E030E086E24C312F023C3C4
:10A7400011F0166A320E156E4CEC03F0196E12C041
:10A750001AF069EC00F0EF6A00011BD000EE8AF0FD
:10A76000020E016E086A7AC61AF079C619F064EC16
:10A7700000F0EF6A00EE90F0020E016E78C628F04D
:10A7800077C627F076C626F075C625F0A2EC00F055
:10A79000EF6A1200949A8B8A030112510001E8B803
:10A7A0001ED0800E026E400E096E226A9BC621F0FA
:10A7B000066A056A200E016EA66AA68E0F0EF76E57
:10A7C0006E0EF66E0900F55003E066EC01F0FAD764
:10A7D0000D0E66EC01F00A0E66EC01F03BD0800E27
:10A7E000026E400E096E226A9BC621F0066A056A57
:10A7F000200E016EB50E66EC01F0620E66EC01F003
:10A80000060E66EC01F0570E66EC01F0080E66ECE1
:10A8100001F0000E66EC01F0010E66EC01F0000E96
:10A8200066EC01F0000E66EC01F0000E66EC01F043
:10A83000500E66EC01F04F0E66EC01F0540E66EC23
:10A8400001F0530E66EC01F0AC0E66EC01F0850EE3
:10A8500066EC01F0A20ED36ED2889B9CC2904B0E88
:10A86000D7EC02F09B8CD298F40ED36EC280949AEF
:10A870008B9A030112510001E8B81ED0800E026EBF
:10A88000400E096E226A9BC621F0066A056A200EF8
:10A89000016EA66AA68E220EF76EA80EF66E09004D
:10A8A000F55003E066EC01F0FAD70D0E66EC01F00E
:10A8B0000A0E66EC01F03BD0800E026E400E096E6F
:10A8C000226A9BC621F0066A056A200E016EB50E4B
:10A8D00066EC01F0620E66EC01F0060E66EC01F02B
:10A8E000570E66EC01F0080E66EC01F0000E66EC07
:10A8F00001F0010E66EC01F0000E66EC01F0000EB6
:10A9000066EC01F0000E66EC01F0200E66EC01F042
:10A910004E0E66EC01F0550E66EC01F0520E66EC40
:10A9200001F07B0E66EC01F0C30E66EC01F0130E35
:10A93000166E880ED8EC02F0096A010E026EAEECBB
:10A9400001F0D8A027D703011C6F000123D79BC6B5
:10A9500049F004EE0CF0240EEE6E470EEE6EEF6A38
:10A96000800E026E800E096E226A9BC621F00B0ECD
:10A97000066EB80E056E27EC01F0D8A0D3D02408DF
:10A98000FAE127EC01F0D8A0CDD003011C6F020E34
:10A990001A6F510E03011A5D00011BE2800E026E58
:10A9A000800E096E226A9BC621F043EC01F0030180
:10A9B0001C6F04EE0CF01A51E926000EEA221CC3AB
:10A9C000EFFF0D0E1C5D000104E003011A2B0001D6
:10A9D000E0E30D6A03011A290C6ED8B40D2A0C505D
:10A9E0000C0FE96E040E0D20EA6EEF6A1B6B03017B
:10A9F0001B511A5D00010EE304EE0CF003011B5124
:10AA0000E926000EEA22EF50D6EC01F003011B2BE1
:10AA10000001EDE3030E096EE80E026EAEEC01F0EC
:10AA2000D8A095D703011C6F550E1C5D010ED8A44C
:10AA3000000E3C6E750E1C5D010ED8A4000E3C127B
:10AA4000000109E006019B2B016A9B5166EC00F0B6
:10AA50000D0ED6EC01F0440E03011C5D010ED8A4CE
:10AA6000000E3C6E640E1C5D010ED8A4000E3C125C
:10AA7000000109E006019B07016A9B5166EC00F0AA
:10AA80000D0ED6EC01F0530E03011C5D010ED8A48F
:10AA9000000E3C6E730E1C5D010ED8A4000E3C121D
:10AAA00000011AE0AA6A3C0EA96E06019B5159ECFE
:10AAB00002F00D0ED6EC01F0220EF76EB40EF66E1B
:10AAC000CEEC01F0016A9B5166EC00F00D0ED6EC65
:10AAD00001F00001E0EF45F0450E03011C5D010EA1
:10AAE000D8A4000E3C6E650E1C5D010ED8A4000EAD
:10AAF0003C12000116E049C09BF60D0ED6EC01F0A9
:10AB0000220EF76EBC0EF66ECEEC01F0016A060165
:10AB10009B5166EC00F00D0ED6EC01F00001E0EF69
:10AB200045F017D7220EF76ED80EF66ECEEC01F078
:10AB30000D0ED6EC01F06ED7939A8A8AE2EC26F0DD
:10AB4000C2EC25F0010E0601561B080E0501E06F50
:10AB5000110EE16F400EE26F040EE36FE46B58C616
:10AB6000E5F557C6E6F556C6E7F555C6E8F5000122
:10AB700048EC50F0640ED7EC02F0D6EC25F0130E42
:10AB8000096E880E026EAEEC01F0DAE303011C6F71
:10AB9000450E1C5D010ED8A4000E3C6E650E1C5DBA
:10ABA000010ED8A4000E3C12000104E0EFEC25F0E9
:10ABB000E0EF45F0C5D703011131000101E21200B9
:10ABC00004EE0CF0220EF76EEA0EF66E18EC04F0AE
:10ABD000020E016E086A1A6A0E0E196E69EC00F018
:10ABE0002E0EEE6E020E016E010E086E8C0E67ECDC
:10ABF00000F0EF6ABCEC29F000EEE8F0410EEE6EDA
:10AC0000500EEE6E420EEE6E430EEE6E020E016EB2
:10AC1000086E8C0E67EC00F0EF6A800E4E6EBCEC96
:10AC200044F000EEE8F010EE4FF0080EE75204E0BA
:10AC3000E6CFEEFFE82EFAD7EF6A610E4E6EBCEC5F
:10AC400044F0030E4B6E0FEC29F0F00E4B6E0FEC40
:10AC500029F003011A6B640E03011A5D000112E270
:10AC600004EE0CF003011A51E926000EEA22EF501F
:10AC70004B6E4B52000106E00FEC29F003011A2B3A
:10AC80000001E9E3CFEC29F003011797010E166EDE
:10AC9000F40ED8EC02F000011200080E0601426F1B
:10ACA000A10E416F790E406F3F6B2BC636F02AC65E
:10ACB00035F029C634F028C633F03A6A396AA80E4E
:10ACC000386E860E376E4FEC05F03C6E2BC636F0B4
:10ACD0002AC635F029C634F028C633F03A6A396AF4
:10ACE000C80E386E840E376E8BEC05F03C160001F2
:10ACF00009E0080E0601426F9B0E416F370E406F50
:10AD0000700E3F6F000127C636F026C635F025C607
:10AD100034F024C633F0CD0E3A6ECC0E396E8B0E65
:10AD2000386E840E376E4FEC05F03C6E27C636F059
:10AD300026C635F025C634F024C633F08F0E3A6EA1
:10AD4000C20E396E650E386E810E376E8BEC05F0D3
:10AD50003C162BC636F02AC635F029C634F028C674
:10AD600033F08F0E3A6E420E396E980E386E850EA5
:10AD7000376E4FEC05F03C162BC636F02AC635F080
:10AD800029C634F028C633F0140E3A6EAE0E396E72
:10AD9000D30E386E830E376E8BEC05F03C1609E04F
:10ADA000080E0601426FAD0E416F380E406FD00E97
:10ADB0003F6F000127C636F026C635F025C634F0B1
:10ADC00024C633F03D0E3A6E0A0E396E6B0E386EA5
:10ADD000830E376E4FEC05F03C6E27C636F026C664
:10ADE00035F025C634F024C633F0660E3A6E396E5F
:10ADF0003C0E386E840E376E8BEC05F03C162BC67D
:10AE000036F02AC635F029C634F028C633F0EC0EE9
:10AE10003A6E510E396E7E0E386E850E376E4FECDF
:10AE200005F03C162BC636F02AC635F029C634F09C
:10AE300028C633F0290E3A6E9C0E396E190E386E04
:10AE4000860E376E8BEC05F03C1609E0080E060105
:10AE5000426F9F0E416F560E406F200E3F6F0001F4
:10AE600027C636F026C635F025C634F024C633F0A2
:10AE7000480E3A6EE10E396E0E0E386E830E376E46
:10AE80004FEC05F03C6E27C636F026C635F025C6D9
:10AE900034F024C633F0C30E3A6EF50E396E560EFA
:10AEA000386E840E376E8BEC05F03C162BC636F0F0
:10AEB0002AC635F029C634F028C633F09A0E3A6E09
:10AEC000190E396E120E386E850E376E4FEC05F086
:10AED0003C162BC636F02AC635F029C634F028C6F3
:10AEE00033F08F0E3A6EC20E396E060E386E860E35
:10AEF000376E8BEC05F03C1608E0080E0601426F39
:10AF00009F0E416F080E406F3F6B000127C636F061
:10AF100026C635F025C634F024C633F0850E3A6EC9
:10AF2000EB0E396E290E386E840E376E4FEC05F03D
:10AF30003C6E27C636F026C635F025C634F024C64A
:10AF400033F0E10E3A6E7A0E396E4E0E386E840E84
:10AF5000376E8BEC05F03C162BC636F02AC635F062
:10AF600029C634F028C633F00A0E3A6ED70E396E71
:10AF7000300E386E850E376E4FEC05F03C162BC642
:10AF800036F02AC635F029C634F028C633F0E10E73
:10AF90003A6E7A0E396E6D0E386E850E376E8BEC0A
:10AFA00005F03C1608E0080E0601426FA10E416F45
:10AFB000790E406F3F6B000127C636F026C635F08C
:10AFC00025C634F024C633F0710E3A6E3D0E396E4C
:10AFD000420E386E810E376E4FEC05F03C6E27C680
:10AFE00036F026C635F025C634F024C633F0290ED7
:10AFF0003A6E5C0E396E230E386E830E376E8BEC14
:10B0000005F03C162BC636F02AC635F029C634F0BA
:10B0100028C633F0D70E3A6EA30E396E420E386E44
:10B02000850E376E4FEC05F03C162BC636F02AC65F
:10B0300035F029C634F028C633F0CD0E3A6E4C0EEA
:10B04000396E520E386E850E376E8BEC05F03C165D
:10B0500009E0080E0601426FAC0E416F890E406F89
:10B06000080E3F6F000127C636F026C635F025C60C
:10B0700034F024C633F0F60E3A6E280E396EDA0E2E
:10B08000386E840E376E4FEC05F03C6E27C636F0F6
:10B0900026C635F025C634F024C633F0520E3A6E7B
:10B0A000B80E396E810E386E840E376E8BEC05F05B
:10B0B0003C162BC636F02AC635F029C634F028C611
:10B0C00033F0B80E3A6E9E0E396E210E386E860E33
:10B0D000376E4FEC05F03C162BC636F02AC635F01D
:10B0E00029C634F028C633F0710E3A6EFD0E396E63
:10B0F000330E386E860E376E8BEC05F03C1609E089
:10B10000080E0601426F9E0E416F0A0E406F180E28
:10B110003F6F000127C636F026C635F025C634F04D
:10B1200024C633F0140E3A6EAE0E396EC80E386E69
:10B13000840E376E4FEC05F03C6E27C636F026C6FF
:10B1400035F025C634F024C633F05C0E3A6E8F0E0F
:10B15000396E8A0E386E820E376E8BEC05F03C1617
:10B160002BC636F02AC635F029C634F028C633F08F
:10B170009A0E3A6E990E396E530E386E850E376EF2
:10B180004FEC05F03C162BC636F02AC635F029C622
:10B1900034F028C633F0B80E3A6E9E0E396E210E8A
:10B1A000386E860E376E8BEC05F03C1609E0080E03
:10B1B0000601426FA70E416F310E406FD80E3F6FF0
:10B1C000000127C636F026C635F025C634F024C661
:10B1D00033F0EC0E3A6E510E396EA80E386E820EB8
:10B1E000376E4FEC05F03C6E27C636F026C635F0BC
:10B1F00025C634F024C633F05C0E3A6E8F0E396EDD
:10B20000420E386E810E376E8BEC05F03C162BC665
:10B2100036F02AC635F029C634F028C633F0F60ECB
:10B220003A6EA80E396E3D0E386E850E376E4FECB5
:10B2300005F03C162BC636F02AC635F029C634F088
:10B2400028C633F03A6A396A160E386E860E376EA3
:10B250008BEC05F03C1609E0080E0601426F9B0ED0
:10B26000416F370E406F700E3F6F000127C636F0FA
:10B2700026C635F025C634F024C633F01F0E3A6ECC
:10B28000850E396E040E386E840E376E4FEC05F065
:10B290003C6E27C636F026C635F025C634F024C6E7
:10B2A00033F01F0E3A6E850E396E1A0E386E840E0C
:10B2B000376E8BEC05F03C162BC636F02AC635F0FF
:10B2C00029C634F028C633F08F0E3A6E420E396E1E
:10B2D0007A0E386E850E376E4FEC05F03C162BC695
:10B2E00036F02AC635F029C634F028C633F01F0ED2
:10B2F0003A6EC50E396E010E386E860E376E8BECC7
:10B3000005F03C1609E0080E0601426F9E0E416FE3
:10B31000B90E406FE00E3F6F000127C636F026C61B
:10B3200035F025C634F024C633F0520E3A6EB80E0E
:10B33000396ECF0E386E840E376E4FEC05F03C6ED2
:10B3400027C636F026C635F025C634F024C633F0BD
:10B35000F60E3A6E280E396E9A0E386E830E376EE0
:10B360008BEC05F03C162BC636F02AC635F029C604
:10B3700034F028C633F09A0E3A6E190E396E8E0EDE
:10B38000386E850E376E4FEC05F03C162BC636F046
:10B390002AC635F029C634F028C633F03A6A396A2D
:10B3A000D60E386E840E376E8BEC05F03C1609E035
:10B3B000080E0601426FA30E416F740E406FD00E4F
:10B3C0003F6F000127C636F026C635F025C634F09B
:10B3D00024C633F03A6A396A386A820E376E4FEC07
:10B3E00005F03C6E27C636F026C635F025C634F08B
:10B3F00024C633F0B80E3A6E1E0E396E310E386E1A
:10B40000820E376E8BEC05F03C162BC636F02AC642
:10B4100035F029C634F028C633F0330E3A6EB30E39
:10B42000396EAB0E386E850E376E4FEC05F03C165C
:10B430002BC636F02AC635F029C634F028C633F0BC
:10B440009A0E3A6E990E396EA50E386E850E376ECD
:10B450008BEC05F03C1608E0080E0601426FA10EC9
:10B46000416F790E406F3F6B000127C636F026C64C
:10B4700035F025C634F024C633F09A0E3A6E990E94
:10B48000396E790E386E7F0E376E4FEC05F03C6EDC
:10B4900027C636F026C635F025C634F024C633F06C
:10B4A000480E3A6EE10E396E4A0E386E820E376ED5
:10B4B0008BEC05F03C162BC636F02AC635F029C6B3
:10B4C00034F028C633F01F0E3A6E850E396E8F0E9B
:10B4D000386E850E376E4FEC05F03C162BC636F0F5
:10B4E0002AC635F029C634F028C633F05C0E3A6E11
:10B4F0008F0E396EF20E386E840E376E8BEC05F0BF
:10B500003C1609E0080E0601426FA40E416FAD0E15
:10B51000406F500E3F6F000127C636F026C635F04B
:10B5200025C634F024C633F00A0E3A6ED70E396EB3
:10B53000630E386E810E376E4FEC05F03C6E27C6F9
:10B5400036F026C635F025C634F024C633F0E10EB9
:10B550003A6E7A0E396E1C0E386E820E376E8BEC98
:10B5600005F03C162BC636F02AC635F029C634F055
:10B5700028C633F0520E3A6EB80E396EA50E386EEC
:10B58000850E376E4FEC05F03C162BC636F02AC6FA
:10B5900035F029C634F028C633F05C0E3A6E8F0EB3
:10B5A000396E9A0E386E850E376E8BEC05F03C16B0
:10B5B00009E0080E0601426FA40E416FAD0E406F08
:10B5C000500E3F6F0001AA6A310EA96E69EC02F0BD
:10B5D0000601656F69EC02F0666F69EC02F0676F57
:10B5E00069EC02F0686F3F51655D0AE14051665DAC
:10B5F00007E14151675D04E14251685D000112E0DD
:10B60000AA6A310EA96E06013F5159EC02F0405171
:10B6100059EC02F0415159EC02F0425159EC02F060
:10B62000000101D81200010E0501E06FE16F080E64
:10B63000E26F00018EEC50F0030116930501E25118
:10B640000C6E640E0C5C000102E10301168306011E
:10B650003E6B020E3D6F030116510001E8B292D01D
:10B660001F0E0601425D000114E311E14A0E0601BE
:10B67000415D00010EE30BE1DD0E0601405D0001BE
:10B6800008E305E1400E06013F5D000102E3000E04
:10B6900001D0010E3C6E010E06013F5DB10E405916
:10B6A000080E4159190E4259000102E2000E01D064
:10B6B000010E3C1605E0040E06013D6F020E3E6FC2
:10B6C000140E0601425D000114E311E1DC0E0601D7
:10B6D000415D00010EE30BE1930E0601405D0001A8
:10B6E00008E305E1800E06013F5D000102E3000E64
:10B6F00001D0010E3C6E010E06013F5D7F0E4059E8
:10B70000ED0E4159100E4259000102E2000E01D027
:10B71000010E3C1605E0060E06013D6F030E3E6F5E
:10B720000A0E0601425D000114E311E16E0E0601EE
:10B73000415D00010EE30BE1490E0601405D000191
:10B7400008E305E1C00E06013F5D000102E3000EC3
:10B7500001D0010E3C6E810E06013F5DBF0E4059C7
:10B76000760E4159080E4259000102E2000E01D046
:10B77000010E3C1605E00C0E06013D6F050E3E6FF6
:10B78000000151D0400E06013F5D720E4059050E7A
:10B7900041592A0E4259000105E2030E06013D6F90
:10B7A000010E3E6FC00E06013F5DEC0E40594F0E7C
:10B7B00041591C0E4259000105E2040E06013D6F7D
:10B7C000020E3E6F400E06013F5D5A0E40590A0EB2
:10B7D0004159150E4259000105E2060E06013D6F62
:10B7E000030E3E6FC00E06013F5DD90E40593E0E5E
:10B7F00041590E0E4259000105E2080E06013D6F47
:10B80000040E3E6F400E06013F5DCE0E40598C0E79
:10B8100041590A0E4259000105E20C0E06013D6F26
:10B82000050E3E6F0001146A080E136E126A116A4B
:10B830001C6A1B6A1A6A3DC619F09EEC03F014C01C
:10B8400068F613C067F612C066F611C065F646C604
:10B8500036F045C635F044C634F043C633F07AECD2
:10B8600007F036C03AF035C039F034C038F033C094
:10B8700037F068C636F067C635F066C634F065C680
:10B8800033F07AEC07F061EC06F036C038F635C0DC
:10B8900037F634C036F633C035F646C614F045C622
:10B8A00013F044C612F043C611F01C6A1B6A1A6AF0
:10B8B0003DC619F01EEC03F014C030F613C02FF68D
:10B8C00012C02EF611C02DF642C614F041C613F078
:10B8D00040C612F03FC611F030C61CF02FC61BF058
:10B8E0002EC61AF02DC619F01EEC03F014C028F075
:10B8F00013C027F012C026F011C025F02504060160
:10B90000586F42C614F041C613F040C612F03FC64D
:10B9100011F030C61CF02FC61BF02EC61AF02DC633
:10B9200019F01EEC03F032C068F631C067F630C083
:10B9300066F62FC065F630C636F02FC635F02EC637
:10B9400034F02DC633F07AEC07F036C03AF035C04B
:10B9500039F034C038F033C037F068C636F067C607
:10B9600035F066C634F065C633F07AEC07F061EC6A
:10B9700006F036C034F635C033F634C032F633C084
:10B9800031F6366A356A346A7F0E336E34C63AF061
:10B9900033C639F032C638F031C637F0D3EC05F093
:10B9A00036C034F635C033F634C032F633C031F623
:10B9B000366A356A346A920E336E34C63AF033C64C
:10B9C00039F032C638F031C637F0C7EC06F015EC66
:10B9D00007F0396F34C03AF635C03BF636C03CF656
:10B9E0003BC657F63AC656F639C655F6080E050157
:10B9F000E06F110EE16F400EE26F040EE36FE46B37
:10BA000058C6E5F557C6E6F556C6E7F555C6E8F556
:10BA1000000148EF50F00F13171A1C1E1E1D1B18B3
:10BA200015110D0906030100000204070B0F719E9A
:10BA30000601F16BF06BEF6BEE6BF56BF46BF36B78
:10BA4000F26B4CEC02F0EE0E16EC02F0AA0E16ECC5
:10BA500002F0FAEC01F0BB6FFAEC01F0BA6FFAEC0D
:10BA600001F0BD6FFAEC01F0BC6FFAEC01F0BF6FB2
:10BA7000FAEC01F0BE6FFAEC01F0C16FFAEC01F0E4
:10BA8000C06FFAEC01F0C36FFAEC01F0C26FFAEC90
:10BA900001F0C56FF8EC01F0C46F29EC02F04CEC3A
:10BAA00002F0EE0E16EC02F0B60E16EC02F0FAEC16
:10BAB00001F0C76FFAEC01F0C66FFAEC01F0C96F44
:10BAC000FAEC01F0C86FFAEC01F0E16FFAEC01F06A
:10BAD000E06FFAEC01F0E36FFAEC01F0E26FFAECE0
:10BAE00001F0E56FF8EC01F0E46F29EC02F0B985A4
:10BAF000000112004CEC02F0EE0E16EC02F0F40E17
:10BB000016EC02F02E0E14EC02F0050ED7EC02F04B
:10BB1000EE0E16EC02F0F60E16EC02F0FAEC01F066
:10BB20000601FF6FF8EC01F0FE6F29EC02F0FFC692
:10BB3000EFF6FEC6EEF64CEC02F0EE0E16EC02F05E
:10BB4000F40E16EC02F0340E14EC02F0050ED7ECF5
:10BB500002F0EE0E16EC02F0F60E16EC02F0FAEC25
:10BB600001F00701006FFAEC01F00601FF6FF8EC3D
:10BB700001F0FE6F29EC02F000C7F3F6FFC6F2F603
:10BB800000011200719E03011C6B030E03011C5D7A
:10BB9000000119E2AFDF0601F251E627F351E72376
:10BBA000F451E823F551E923EE51EA27EF51EB2355
:10BBB000F051EC23F151ED23C80ED7EC02F0030154
:10BBC0001C2B0001E2E3E9C614F0E8C613F0E7C657
:10BBD00012F0E6C611F01C6A1B6A1A6A030E196E8F
:10BBE0001EEC03F014C0F5F613C0F4F612C0F3F621
:10BBF00011C0F2F6EDC614F0ECC613F0EBC612F06D
:10BC0000EAC611F01C6A1B6A1A6A030E196E1EEC52
:10BC100003F014C0F1F613C0F0F612C0EFF611C035
:10BC2000EEF60601C451EE5D336EC551EF59346E28
:10BC3000000EC5BFFF0EF059356E000EC5BFFF0EDA
:10BC4000F159366E7CEC07F036C028F035C027F08D
:10BC500034C026F033C025F0C3C634F0C2C633F07A
:10BC600070EC07F028C03AF027C039F026C038F051
:10BC700025C037F0C7EC06F036C022F335C021F3FB
:10BC800034C020F333C01FF322C304F721C303F7EA
:10BC900020C302F70F0E03011F5D02E23F84000E76
:10BCA0000701016FE3C634F0E2C633F070EC07F031
:10BCB00036C028F035C027F034C026F033C025F058
:10BCC0000B0E252402E33F82FF0E0001256E04C700
:10BCD0002CF003C72BF002C72AF001C729F0E5C6F4
:10BCE00034F0E4C633F070EC07F02CC03AF02BC00F
:10BCF00039F02AC038F029C037F0D3EC05F036C04F
:10BD00002CF035C02BF034C02AF033C029F028C005
:10BD100036F027C035F026C034F025C033F02CC0F3
:10BD20003AF02BC039F02AC038F029C037F061EC66
:10BD300006F036C008F735C007F734C006F733C041
:10BD400005F704C73AF003C739F002C738F001C756
:10BD500037F008C736F007C735F006C734F005C717
:10BD600033F0D3EC05F036C018F735C017F734C000
:10BD700016F733C015F7366A356A346A820E336EA9
:10BD800018C73AF017C739F016C738F015C737F09B
:10BD9000D3EC05F036C028F035C027F034C026F0CB
:10BDA00033C025F03A6A396A386A830E376E28C084
:10BDB00036F027C035F026C034F025C033F061ECF2
:10BDC00006F015EC07F00601F66F34C0F7F635C043
:10BDD000F8F636C0F9F63A6A396A200E386E820EE5
:10BDE000376EF9C636F0F8C635F0F7C634F0F6C649
:10BDF00033F07CEC07F061EC06F036C024F735C078
:10BE000023F734C022F733C021F7000E030114BF1B
:10BE1000010E3C6E010E0601B9B1000E3C16000188
:10BE20003DE0366A356A200E346E840E336E24C7C8
:10BE30003AF023C739F022C738F021C737F0D3ECE6
:10BE400005F036C028F035C027F034C026F033C0E6
:10BE500025F0366A356A200E346E820E336E28C0A5
:10BE60003AF027C039F026C038F025C037F0C7ECCB
:10BE700006F015EC07F00301236F34C024F300EE45
:10BE8000DDF0020E016E030E086E24C31AF023C308
:10BE900019F069EC00F0EF6A000110D000EEDDF05F
:10BEA000020E016E24C728F023C727F022C726F010
:10BEB00021C725F0010EA2EC00F0EF6A3A6A396A58
:10BEC0007A0E386E8A0E376E18C736F017C735F0FF
:10BED00016C734F015C733F0D1EC05F036C01CF7A7
:10BEE00035C01BF734C01AF733C019F71CC73AF036
:10BEF0001BC739F01AC738F019C737F01CC736F01E
:10BF00001BC735F01AC734F019C733F0C7EC06F079
:10BF100036C028F035C027F034C026F033C025F0F5
:10BF200028C022F327C021F326C020F30C0E255C85
:10BF300002E23F84000E03011F6FC9C634F0C8C679
:10BF400033F070EC07F022C33AF021C339F020C37C
:10BF500038F01FC337F0C7EC06F036C004F735C021
:10BF600003F734C002F733C001F7BDC634F0BCC6D6
:10BF700033F070EC07F01CC73AF01BC739F01AC752
:10BF800038F019C737F0C7EC06F036C008F735C0EF
:10BF900007F734C006F733C005F704C73AF003C704
:10BFA00039F002C738F001C737F008C736F007C7C5
:10BFB00035F006C734F005C733F0D3EC05F036C0D2
:10BFC00028F035C027F034C026F033C025F028C053
:10BFD0000CF727C00BF726C00AF70B0E255C02E210
:10BFE0003F84000E0701096FBBC634F0BAC633F0B8
:10BFF00070EC07F036C028F035C027F034C026F0CA
:10C0000033C025F0020E252402E33F82FF0E00011B
:10C01000256E28C03AF027C039F026C038F025C078
:10C0200037F00CC736F00BC735F00AC734F009C734
:10C0300033F0D3EC05F036C028F035C027F034C01B
:10C0400026F033C025F0366A356A346A800E336EC6
:10C0500028C03AF027C039F026C038F025C037F0A4
:10C06000D3EC05F036C028F035C027F034C026F0F8
:10C0700033C025F028C010F727C00FF726C00EF7F1
:10C08000020E255C02E23F84000E07010D6FBFC661
:10C0900034F0BEC633F070EC07F01CC73AF01BC793
:10C0A00039F01AC738F019C737F0C7EC06F036C0B8
:10C0B00028F035C027F034C026F033C025F028C062
:10C0C00004F727C003F726C002F70D0E255C02E235
:10C0D0003F84000E0701016FC7C634F0C6C633F0B7
:10C0E00070EC07F022C33AF021C339F020C338F0D6
:10C0F0001FC337F0C7EC06F036C028F035C027F074
:10C1000034C026F033C025F028C008F727C007F751
:10C1100026C006F7100E255C02E23F84000E0701E0
:10C12000056F04C728F003C727F002C726F001C730
:10C1300025F028C03AF027C039F026C038F025C0D5
:10C1400037F008C736F007C735F006C734F005C723
:10C1500033F0D3EC05F036C028F035C027F034C0FA
:10C1600026F033C025F0366A356A346A800E336EA5
:10C1700028C03AF027C039F026C038F025C037F083
:10C18000D3EC05F036C028F035C027F034C026F0D7
:10C1900033C025F028C00CF727C00BF726C00AF7DC
:10C1A000020E255C02E23F84000E0701096FC1C642
:10C1B00034F0C0C633F070EC07F036C028F035C05C
:10C1C00027F034C026F033C025F00CC72CF00BC785
:10C1D0002BF00AC72AF009C729F0366A356A346A93
:10C1E0008E0E336E2CC03AF02BC039F02AC038F0D6
:10C1F00029C037F0D3EC05F036C02CF035C02BF059
:10C2000034C02AF033C029F028C03AF027C039F0F2
:10C2100026C038F025C037F02CC036F02BC035F0E2
:10C220002AC034F029C033F0C7EC06F036C028F03D
:10C2300035C027F034C026F033C025F028C014F7ED
:10C2400027C013F726C012F70F0E255C02E23F84C9
:10C25000000E0701116FF5C636F0F4C635F0F3C6CF
:10C2600034F0F2C633F07CEC07F010C73AF00FC799
:10C2700039F00EC738F00DC737F0D1EC05F036C0F5
:10C2800028F035C027F034C026F033C025F0366AD8
:10C29000500E356E430E346E8E0E336E28C03AF05B
:10C2A00027C039F026C038F025C037F0C7EC06F0BB
:10C2B00015EC07F00601DA6F34C0DBF635C0DCF6AA
:10C2C00036C0DDF6DDC636F0DCC635F0DBC634F050
:10C2D000DAC633F07CEC07F03A6A396A386A800EC5
:10C2E000376EC7EC06F036C028F035C027F034C0F2
:10C2F00026F033C025F028C036F027C035F026C020
:10C3000034F025C033F014C73AF013C739F012C720
:10C3100038F011C737F061EC06F036C020F735C0B1
:10C320001FF734C01EF733C01DF720C722F31FC705
:10C3300021F31EC720F3080E07011D5D02E23F84B2
:10C34000000E03011F6F22C33AF021C339F020C34E
:10C3500038F01FC337F022C336F021C335F020C3B5
:10C3600034F01FC333F0C7EC06F036C004F735C015
:10C3700003F734C002F733C001F7366AE00E356EBA
:10C380003D0E346E8A0E336E04C73AF003C739F09F
:10C3900002C738F001C737F0C7EC06F036C028F006
:10C3A00035C027F034C026F033C025F028C004F78C
:10C3B00027C003F726C002F7100E255C02E23F8477
:10C3C000000E0701016F366AE80E356EE50E346E19
:10C3D0008B0E336E20C73AF01FC739F01EC738F0F6
:10C3E0001DC737F0C7EC06F036C028F035C027F07F
:10C3F00034C026F033C025F028C008F727C007F75F
:10C4000026C006F7100E255C02E23F84000E0701ED
:10C41000056F20C728F01FC727F01EC726F01DC7CD
:10C4200025F004C72CF003C72BF002C72AF001C780
:10C4300029F02CC03AF02BC039F02AC038F029C0BE
:10C4400037F008C736F007C735F006C734F005C720
:10C4500033F0D3EC05F036C02CF035C02BF034C0EF
:10C460002AF033C029F0366AF00E356E6C0E346E49
:10C470008A0E336E2CC03AF02BC039F02AC038F047
:10C4800029C037F0D3EC05F036C02CF035C02BF0C6
:10C4900034C02AF033C029F0040E295E02E23F8442
:10C4A000296A000128C03AF027C039F026C038F0C8
:10C4B00025C037F02CC036F02BC035F02AC034F040
:10C4C00029C033F0D3EC05F015EC07F00601FA6F44
:10C4D00034C0FBF635C0FCF636C0FDF63A6A396A60
:10C4E000480E386E850E376EFDC636F0FCC635F048
:10C4F000FBC634F0FAC633F07CEC07F061EC06F0D2
:10C5000036C020F735C01FF734C01EF733C01DF703
:10C51000000E030114BF010E3C6E010E0601B9B1FD
:10C52000000E3C16000125E03A6A396A480E386E62
:10C53000840E376E20C736F01FC735F01EC734F0A3
:10C540001DC733F0D1EC05F015EC07F00301236FA4
:10C5500034C024F300EED2F0020E016E030E086E1A
:10C5600024C31AF023C319F069EC00F0EF6A00014C
:10C5700010D000EED2F0020E016E20C728F01FC7C7
:10C5800027F01EC726F01DC725F0010EA2EC00F013
:10C59000EF6A718E1200B50E0501E06F620EE16F59
:10C5A000060EE26F240EE36FE46FE56BE669E76960
:10C5B000080EE86F030EE96FEA6BEB6BEC6BED6B4B
:10C5C000100EEE6F270EEF6FF06BF16B050EF26F32
:10C5D000F36BFA0EF46FF56BF66FF76B640EF86F92
:10C5E000F96B2C0EFA6F010EFB6FFC6B3C0EFD6FAE
:10C5F000FE6BFF6B0601006B016BC80E026F036BD5
:10C60000046B056B066B076B086B096B1C0E0A6FDE
:10C610006C0E0B6FB50E0C6F620E0D6F060E0E6F6B
:10C62000240E0F6F106B116B2A0E126F840E136F96
:10C6300003011A6B340E03011A5D000116E2800E2D
:10C64000026E400E096E226A9BC621F0066A056AD8
:10C65000200E016E05EEE0F003011A51EB5066EC7E
:10C6600001F003011A2B0001E5E312000B0E060195
:10C67000945D000106E307E1B90E0601935D000138
:10C6800002E2000E01D0010E3C6E74C636F073C695
:10C6900035F072C634F071C633F09A0E3A6E990EC8
:10C6A000396E190E386E7F0E376E4FEC05F03C1662
:10C6B000000109E0070E166ED00ED8EC02F097C606
:10C6C00061F699EC25F0BBEC26F00601986BB98178
:10C6D000000E030113B5010E3C6E000E13B3010EE4
:10C6E0003C12000102E061EC52F0000E030113B9AC
:10C6F000010E3C6E000E14B1010E3C12000104E06C
:10C70000E5EC25F0CBEC4BF00601B9510001E8B89F
:10C71000A2D103011A6B060E03011A5D00010EE29D
:10C7200000EE4FF003011A51EB500C6E200E0C5C22
:10C73000000104E003011A2B0001EDE300EEE8F034
:10C740000D0EEE6E240EEE6EEE6EEE6EEE6E10EED2
:10C750004FF003011A510001E6CFEEFFE82EFBD7A0
:10C76000EF6A00EEE8F0EE50FEE1ED522F0EEE6EB5
:10C77000410EEE6E4D0EEE6E2C0EEE6E15EEA7F027
:10C78000050EE75204E0E6CFEEFFE82EFAD72C0EB6
:10C79000EE6E11EE7FF00F0EE75204E0E6CFEEFFF3
:10C7A000E82EFAD72C0EEE6E11EE8FF00F0EE75238
:10C7B00004E0E6CFEEFFE82EFAD72C0EEE6E11EE77
:10C7C0009FF00F0EE75204E0E6CFEEFFE82EFAD717
:10C7D000EF6A030117310001D8B0EFD000EEE8F0A6
:10C7E000EE50FEE1ED522C0EEE6E11EEAFF00F0E9C
:10C7F000E75204E0E6CFEEFFE82EFAD7EF6A030136
:10C8000012510001E8AA17D0C2EC5DF000EEE8F08A
:10C81000EE50FEE1ED522C0EEE6E020E016E20C7C0
:10C8200028F01FC727F01EC726F01DC725F0010EF0
:10C83000A2EC00F0EF6A030114510001E8A41CD03F
:10C8400000EEE8F0EE50FEE1ED522C0EEE6E020E20
:10C85000016E086AA4C51AF0A3C519F069EC00F0CE
:10C860002C0EEE6E020E016E086AA6C51AF0A5C562
:10C8700019F069EC00F0EF6A030113510001E8A61A
:10C8800013D01FEC51F000EEE8F0EE50FEE1ED5257
:10C890002C0EEE6E10EE9BF00A0EE75204E0E6CF8F
:10C8A000EEFFE82EFAD7EF6A030113510001E8A862
:10C8B00011D000EEE8F0EE50FEE1ED522C0EEE6EDF
:10C8C00010EEBCF00A0EE75204E0E6CFEEFFE82ED1
:10C8D000FAD7EF6A030113510001E8AA13D0C0ECA4
:10C8E00051F000EEE8F0EE50FEE1ED522C0EEE6E4F
:10C8F00010EEC7F00A0EE75204E0E6CFEEFFE82E96
:10C90000FAD7EF6A03011431000111E300EEE8F0F9
:10C91000EE50FEE1ED522C0EEE6E10EEB1F00A0E6E
:10C92000E75204E0E6CFEEFFE82EFAD7EF6A030104
:10C9300013510001E8A411D000EEE8F0EE50FEE142
:10C94000ED522C0EEE6E10EEA6F00A0EE75204E049
:10C95000E6CFEEFFE82EFAD7EF6A0301125100018D
:10C96000E8A62BD0030113510001E8AC11D000EE72
:10C97000E8F0EE50FEE1ED522C0EEE6E10EE90F06F
:10C980000A0EE75204E0E6CFEEFFE82EFAD7EF6A90
:10C9900003011335000111E300EEE8F0EE50FEE173
:10C9A000ED522C0EEE6E10EE8AF0050EE75204E00A
:10C9B000E6CFEEFFE82EFAD7EF6A0301145100012B
:10C9C000E8A213D0E7EC4CF000EEE8F0EE50FEE108
:10C9D000ED522C0EEE6E15EEADF0320EE75204E085
:10C9E000E6CFEEFFE82EFAD7EF6A06018F6B00EE76
:10C9F000E8F0E86AEE5202E0E83EFCD70B6E050E66
:10CA000003011B6F03011B510B5C00010FE300EEE0
:10CA1000E8F003011B51E926000EEA22EF500C6EEC
:10CA200006018F1B03011B2B0001ECE300EEE8F075
:10CA3000EE50FEE1ED522A0EEE6E020E016E086E11
:10CA400006018F514FEC00F00D0EEE6E0A0EEE6EE9
:10CA5000EF6A000129D000EEE8F0240EEE6E13EE2E
:10CA600060F0550EE75204E0E6CFEEFFE82EFAD76D
:10CA7000EF6A1AD800EEE8F0240EEE6E13EEB6F070
:10CA8000550EE75204E0E6CFEEFFE82EFAD7EF6A44
:10CA90000BD8640ED7EC02F0EFEC25F08EC661F6F1
:10CAA00099EC25F0C2EF25F0939A8A8A6CEC25F078
:10CAB000B8EC25F0640ED7EC02F003011A6B00010C
:10CAC00000EEE8F003011A51E926000EEA22EF50C9
:10CAD0000C6E000E0C52D8A4010E3C6E960E1A5D20
:10CAE000010ED8B0000E3C16000136E000EEE8F072
:10CAF00003011A51E926000EEA22EF500601906F59
:10CB0000939A8A9A6CC612F06B51E5EC02F0010E12
:10CB100003011C6F03011C510601535D000110E36A
:10CB2000060190B1818A90A1819A6CC612F06B5176
:10CB3000E5EC02F0D890903303011C2B0001EAE3EE
:10CB4000939A8A8A6EC612F006016D51E5EC02F0E6
:10CB500003011A2B0001B3D7640ED7EC02F00601D3
:10CB6000B9510001E8B808D0EFEC25F08EC661F6A7
:10CB700099EC25F0C2EC25F0800E026E800E096E55
:10CB8000226A9BC621F00B0E066EB80E056E27ECCE
:10CB900001F009E32408FBE127EC01F004E30301C1
:10CBA0001C6F0001120082949494640ED7EC02F082
:10CBB0009484030E166EE80ED8EF02F00601B991C8
:10CBC00004EE0CF0540EEE6E230EEE6E020E016EAD
:10CBD000030E086EB8C61AF0B7C619F069EC00F07B
:10CBE000EF6AB0C6AFF6000170D804EE0CF0EE505C
:10CBF000FEE1ED522C0EEE6E11EEBFF00A0EE75282
:10CC000004E0E6CFEEFFE82EFAD7EF6AB1C6AFF642
:10CC10005CD804EE0CF0EE50FEE1ED522C0EEE6E00
:10CC200011EEBFF00A0EE75204E0E6CFEEFFE82E69
:10CC3000FAD7EF6AB2C6AFF648D804EE0CF0EE5061
:10CC4000FEE1ED522C0EEE6E11EEBFF00A0EE75231
:10CC500004E0E6CFEEFFE82EFAD7EF6AB3C6AFF6F0
:10CC600034D804EE0CF0EE50FEE1ED522C0EEE6ED8
:10CC700011EEBFF00A0EE75204E0E6CFEEFFE82E19
:10CC8000FAD7EF6AB4C6AFF620D804EE0CF0EE5037
:10CC9000FEE1ED522C0EEE6E11EEBFF00A0EE752E1
:10CCA00004E0E6CFEEFFE82EFAD7EF6A04EE0CF0D0
:10CCB000EE50FEE1ED52220EF76EF40EF66E18EC19
:10CCC00004F00D0EEE6EEE6A120003011251000127
:10CCD000E8A603D023EC53F00ED000EE8AF0310E1C
:10CCE000EE6E300EEE6EEE6EEF6A00EE90F0EE6ECF
:10CCF000EE6EEE6EEF6A300E0601AF5D000106E1EA
:10CD000001EEBFF0300EEE6EEF6AB4D0310E0601C8
:10CD1000AF5D00010FE11FEC51F001EEBFF010EE2E
:10CD20009BF00A0EE75204E0E6CFEEFFE82EFAD7BA
:10CD3000EF6AA0D0320E0601AF5D00010FE1C0EC3A
:10CD400051F001EEBFF010EEC7F00A0EE75204E01A
:10CD5000E6CFEEFFE82EFAD7EF6A8CD0330E06014D
:10CD6000AF5D00010FE1CBEC4BF001EEBFF010EE38
:10CD7000BCF00A0EE75204E0E6CFEEFFE82EFAD749
:10CD8000EF6A78D0340E0601AF5D00010FE161EC6F
:10CD900052F001EEBFF010EEA6F00A0EE75204E0EA
:10CDA000E6CFEEFFE82EFAD7EF6A64D0350E060123
:10CDB000AF5D00010FE1CBEC4BF001EEBFF010EEE8
:10CDC000B1F00A0EE75204E0E6CFEEFFE82EFAD704
:10CDD000EF6A50D0360E0601AF5D00010DE101EEA5
:10CDE000BFF010EE90F00A0EE75204E0E6CFEEFF3F
:10CDF000E82EFAD7EF6A3ED0370E0601AF5D00018C
:10CE00000DE101EEBFF010EE8AF0050EE75204E0EE
:10CE1000E6CFEEFFE82EFAD7EF6A2CD0380E0601E7
:10CE2000AF5D000116E10601B9510001E8B402D07E
:10CE300017EC5DF0C2EC5DF001EEBFF010EED2F049
:10CE40000A0EE75204E0E6CFEEFFE82EFAD7EF6ACB
:10CE500011D0390E0601AF5D00010CE101EEBFF00B
:10CE600015EEA7F0050EE75204E0E6CFEEFFE82E40
:10CE7000FAD7EF6A1200300E0601AF5D000107E13C
:10CE8000220EF76EFE0EF66ECEEC01F06BD0310E78
:10CE90000601AF5D000107E1230EF76E060EF66E88
:10CEA000CEEC01F05FD0320E0601AF5D000107E16C
:10CEB000230EF76E100EF66ECEEC01F053D0330E4B
:10CEC0000601AF5D000107E1230EF76E1A0EF66E44
:10CED000CEEC01F047D0340E0601AF5D000107E152
:10CEE000230EF76E220EF66ECEEC01F03BD0350E1F
:10CEF0000601AF5D000107E1230EF76E2C0EF66E02
:10CF0000CEEC01F02FD0360E0601AF5D000107E137
:10CF1000230EF76E360EF66ECEEC01F023D0370EF0
:10CF20000601AF5D000107E1230EF76E400EF66EBD
:10CF3000CEEC01F017D0380E0601AF5D000107E11D
:10CF4000230EF76E4A0EF66ECEEC01F00BD0390EC2
:10CF50000601AF5D000106E1230EF76E540EF66E7A
:10CF6000CEEC01F012002ADE4CEC27F003011C6B22
:10CF7000000104EE0CF003011C51E926000EEA2228
:10CF8000EF500C6E0D0E0C5CD8A4010E3C6EFF0E23
:10CF90001C5D010ED8B0000E3C16000110E004EE3E
:10CFA0000CF003011C51E926000EEA22EF504B6EF3
:10CFB00000010FEC29F003011C2B0001D9D7CFECA5
:10CFC00029F0010E0601B725256E000EB821266E48
:10CFD00026C012F025C011F0030E166EE80E156E75
:10CFE0004CEC03F01AC0B8F619C0B7F600011200F5
:10CFF0000601B55300010DE104EE0CF011EECAF08C
:10D00000500EE75204E0E6CFEEFFE82EFAD7EF6AC3
:10D0100035D0010E0601B55D00010DE104EE0CF006
:10D0200012EE1BF0500EE75204E0E6CFEEFFE82EC2
:10D03000FAD7EF6A23D0020E0601B55D00010DE1BB
:10D0400004EE0CF012EE6CF0500EE75204E0E6CF66
:10D05000EEFFE82EFAD7EF6A11D0030E0601B55D98
:10D0600000010CE104EE0CF012EEBDF0500EE752A0
:10D0700004E0E6CFEEFFE82EFAD7EF6A0601B52B03
:10D08000030EB51704EE0CF0EE50FEE1ED520D0E5E
:10D09000EE6EEF6A00014CEC27F003011C6B0001FF
:10D0A00004EE0CF003011C51E926000EEA22EF50B9
:10D0B0000C6E0D0E0C5CD8A4010E3C6EFF0E1C5DB8
:10D0C000010ED8B0000E3C16000110E004EE0CF08A
:10D0D00003011C51E926000EEA22EF504B6E0001BD
:10D0E0000FEC29F003011C2B0001D9D7CFEF29F059
:10D0F00003011A6B000100EE4FF003011A51EB50CF
:10D100000C6E210E0C5C000111E300EE4FF00301E8
:10D110001A51EBCF0CF000EEE8F01A51E926000EA0
:10D12000EA220CC0EFFF1A2B0001E4D700EEE8F072
:10D1300003011A51E926000EEA22EF6A55500C6EDF
:10D140000C52000115E000EEE8F0EE50FEE1ED5269
:10D150002D0EEE6E020E016EEACF0DF0E9CF0CF04F
:10D1600055500DC0EAFF0CC0E9FF66EC00F0EF6A15
:10D1700000EEE8F0E86AEE5202E0E83EFCD70C6E02
:10D18000090E0C5C09E200EEE8F0EE50FEE1ED5213
:10D19000200EEE6EEF6AECD701EECAF03A0EEE6E9C
:10D1A00010EEE8F0960EE75204E0E6CFEEFFE82E30
:10D1B000FAD7230EF76E600EF66E18EC04F0EF6AE5
:10D1C00002EE1BF03A0EEE6E10EEE8F0960EE7520D
:10D1D00004E0E6CFEEFFE82EFAD7230EF76E680ED6
:10D1E000F66E18EC04F0EF6A02EE6CF03A0EEE6E9A
:10D1F00010EEE8F0960EE75204E0E6CFEEFFE82EE0
:10D20000FAD7230EF76E700EF66E18EC04F0EF6A84
:10D2100002EEBDF03A0EEE6E10EEE8F0960EE7521A
:10D2200004E0E6CFEEFFE82EFAD7230EF76E780E75
:10D23000F66E18EC04F0EF6AB0C61CF32DD874EC4F
:10D240006BF0B1C61CF328D874EC6BF0B2C61CF3BB
:10D2500023D874EC6BF0B3C61CF31ED874EC6BF0DF
:10D26000B4C61CF319D801EECAF0EE50FEE1ED523F
:10D27000230EF76E9A0EF66E18EC04F0EF6A02EECB
:10D280001BF0EE50FEE1ED52230EF76E9A0EF66E95
:10D2900018EC04F0EF6A1200300E03011C5D00016F
:10D2A00023E101EECAF0EE50FEE1ED524E0EEE6EBD
:10D2B000430EEE6EEF6A02EE1BF0EE50FEE1ED5211
:10D2C000200EEE6EEF6A02EE6CF0EE50FEE1ED52D3
:10D2D000300EEE6E2C0EEE6E310EEE6E2C0EEE6EED
:10D2E000300EEE6EEF6AFFD1310E03011C5D0001BE
:10D2F00036E101EECAF0EE50FEE1ED52230EF76E7C
:10D30000B40EF66E18EC04F0EF6A02EE1BF0EE506D
:10D31000FEE1ED52430EEE6EEF6A0301143500019B
:10D320000DE302EE6CF0EE50FEE1ED52230EF76ECF
:10D33000BC0EF66E18EC04F0EF6A10D002EE6CF042
:10D34000EE50FEE1ED52300EEE6E2C0EEE6E310E12
:10D35000EE6E2C0EEE6E300EEE6EEF6AC4D1320E13
:10D3600003011C5D000136E101EECAF0EE50FEE162
:10D37000ED52230EF76EC60EF66E18EC04F0EF6A4F
:10D3800002EE1BF0EE50FEE1ED52430EEE6EEF6A40
:10D390000301143500010DE302EE6CF0EE50FEE1E6
:10D3A000ED52230EF76EBC0EF66E18EC04F0EF6A29
:10D3B00010D002EE6CF0EE50FEE1ED52300EEE6E4B
:10D3C0002C0EEE6E310EEE6E2C0EEE6E300EEE6EFC
:10D3D000EF6A89D1330E03011C5D000136E101EED5
:10D3E000CAF0EE50FEE1ED52230EF76ECE0EF66E51
:10D3F00018EC04F0EF6A02EE1BF0EE50FEE1ED5285
:10D40000430EEE6EEF6A0301143500010DE302EEE8
:10D410006CF0EE50FEE1ED52230EF76EBC0EF66E90
:10D4200018EC04F0EF6A10D002EE6CF0EE50FEE162
:10D43000ED52300EEE6E2C0EEE6E310EEE6E2C0EA8
:10D44000EE6E300EEE6EEF6A4ED1340E03011C5DAF
:10D45000000138E101EECAF0EE50FEE1ED52550E4A
:10D46000EE6E620EEE6E610EEE6E740EEE6EEF6A92
:10D4700002EE1BF0EE50FEE1ED52560EEE6EEF6A3C
:10D480000301143500010DE302EE6CF0EE50FEE1F5
:10D49000ED52230EF76ED60EF66E18EC04F0EF6A1E
:10D4A00010D002EE6CF0EE50FEE1ED52300EEE6E5A
:10D4B0002C0EEE6E310EEE6E2C0EEE6E300EEE6E0B
:10D4C000EF6A11D1350E03011C5D000138E101EE58
:10D4D000CAF0EE50FEE1ED52550EEE6E730EEE6E9A
:10D4E000790EEE6E730EEE6EEF6A02EE1BF0EE50EA
:10D4F000FEE1ED52560EEE6EEF6A030114350001A7
:10D500000DE302EE6CF0EE50FEE1ED52230EF76EED
:10D51000E00EF66E18EC04F0EF6A10D002EE6CF03C
:10D52000EE50FEE1ED52300EEE6E2C0EEE6E310E30
:10D53000EE6E2C0EEE6E300EEE6EEF6AD4D0360E1E
:10D5400003011C5D000138E101EECAF0EE50FEE17E
:10D55000ED52550EEE6E730EEE6E6F0EEE6E6C0E9D
:10D56000EE6EEF6A02EE1BF0EE50FEE1ED52560E4B
:10D57000EE6EEF6A0301143500010DE302EE6CF06C
:10D58000EE50FEE1ED52230EF76ED60EF66E18EC5D
:10D5900004F0EF6A10D002EE6CF0EE50FEE1ED52B6
:10D5A000300EEE6E2C0EEE6E310EEE6E2C0EEE6E1A
:10D5B000300EEE6EEF6A97D0370E03011C5D00014E
:10D5C00025E101EECAF0EE50FEE1ED52490EEE6E9D
:10D5D000730EEE6E6F0EEE6E6C0EEE6EEF6A02EE76
:10D5E0001BF0EE50FEE1ED526D0EEE6E410EEE6E52
:10D5F000EF6A02EE6CF0EE50FEE1ED52230EF76E94
:10D60000EA0EF66E18EC04F0EF6A6DD0380E0301E6
:10D610001C5D00013DE101EECAF0EE50FEE1ED526D
:10D62000230EF76E4A0EF66E18EC04F0EF6A02EE67
:10D630001BF0EE50FEE1ED52680EEE6E500EEE6EF7
:10D64000610EEE6EEF6A0301143500010DE302EE88
:10D650006CF0EE50FEE1ED52230EF76EF40EF66E16
:10D6600018EC04F0EF6A10D002EE6CF0EE50FEE120
:10D67000ED52300EEE6E2C0EEE6E310EEE6E2C0E66
:10D68000EE6E300EEE6EEF6A0301128B00012BD0AE
:10D69000390E03011C5D000126E101EECAF0EE50D7
:10D6A000FEE1ED52530EEE6E410EEE6E540EEE6E36
:10D6B000730EEE6EEF6A02EE1BF0EE50FEE1ED52DD
:10D6C000200EEE6EEF6A02EE6CF0EE50FEE1ED52CF
:10D6D000300EEE6E2C0EEE6E310EEE6E2C0EEE6EE9
:10D6E000300EEE6EEF6A120001EECAF0EE50FEE16F
:10D6F000ED522C0EEE6EEF6A02EE1BF0EE50FEE1E4
:10D70000ED522C0EEE6EEF6A02EE6CF0EE50FEE182
:10D71000ED522C0EEE6EEF6A120003011251000161
:10D72000E8AC01D0120003011A6B189103011A2B07
:10D730000B0E1A5D000104E30301188100011200C1
:10D74000240E03011C5D000112E0800E026E800EAB
:10D75000096E226A9BC621F0030E066EE80E056E66
:10D7600027EC01F0E3E303011C6F0001E9D7800E11
:10D77000026E800E096E226A9BC621F0010E066EB3
:10D780002C0E056E27EC01F0D1E303011C6F470E50
:10D790001C5D0001CBE1800E026E800E096E226AD4
:10D7A0009BC621F0010E066E2C0E056E27EC01F0D3
:10D7B000D8A0BCD703011C6F500E1C5DD8A4010E6D
:10D7C0003C6E4E0E1C5DD8A4010E3C16000101E01B
:10D7D000ADD7800E026E800E096E226A9BC621F0C4
:10D7E000010E066E2C0E056E27EC01F0D8A09ED718
:10D7F00003011C6F560E1C5D0001D8A497D7800E44
:10D80000026E800E096E226A9BC621F0010E066E22
:10D810002C0E056E27EC01F0D8A088D703011C6FF1
:10D82000540E1C5D0001D8A481D7120006018F6B35
:10D83000010E03011A6F800E026E400E096E226AFD
:10D840009BC621F0066A056A200E016E240E66EC66
:10D8500001F0000100EEE8F003011A51E926000E84
:10D86000EA22EF500C6E2A0E0C5CD8A4010E3C6E1E
:10D870004F0E1A5D010ED8B0000E3C16000123E0D9
:10D88000800E026E400E096E226A9BC621F0066A67
:10D89000056A200E016E00EEE8F003011A51E92638
:10D8A000000EEA22EF5066EC01F000EEE8F01A51AB
:10D8B000E926000EEA22EF500C6E06018F1B0301D1
:10D8C0001A2B0001C6D7800E026E400E096E226A26
:10D8D0009BC621F0066A056A200E016E2A0E66ECD0
:10D8E00001F0020E086E06018F514FEC00F00D0E94
:10D8F00066EC01F00A0E66EC01F0000112007BEC10
:10D9000025F0BCEC26F0030E166EE80ED8EC02F003
:08D91000FCEF24F0FFD7FFD764
:020000040030CA
:03000100D8103CD8
:020005003D803C
:0600080008C00FE00F40EC
:0200000400F00A
:100000004E4F43414C4C0B4243504C313400574906
:1000100044453120010000000000000057494445DC
:1000200032200177860080280F2F4F028A0302C0FA
:10003000690079A1086407F82401F4015414C06B25
:100040009E0852036400373231343536377F6A29CF
:100050003F3E3C3830202123272F475501310611E0
:10006000150902140B10041E0D1207050F161B0AAA
:1000700008030C180E191D134243545241434B20E0
:10008000762E5C5A202D20556261743D205C755699
:0A0090002C2054313D205C54430D38
:00000001FF
